 AutoWrap

 Timestamp is 57a0e29a (Tue Aug  2 21:12:42 2016)

 Preferred load address is 0000000180000000

 Start         Length     Name                   Class
 0001:00000000 00000010H .00cfg                  CODE
 0001:00000010 00000008H .CRT$XCA                CODE
 0001:00000018 00000008H .CRT$XCZ                CODE
 0001:00000020 00000008H .CRT$XIA                CODE
 0001:00000028 00000018H .CRT$XIC                CODE
 0001:00000040 00000008H .CRT$XIZ                CODE
 0001:00000048 00000008H .CRT$XPA                CODE
 0001:00000050 00000010H .CRT$XPX                CODE
 0001:00000060 00000008H .CRT$XPXA               CODE
 0001:00000068 00000008H .CRT$XPZ                CODE
 0001:00000070 00000008H .CRT$XTA                CODE
 0001:00000078 00000008H .CRT$XTZ                CODE
 0001:00000080 000074f8H .rdata                  CODE
 0001:00007578 000001f8H .rdata$r                CODE
 0001:00007770 00000010H .rdata$zETW0            CODE
 0001:00007780 00000077H .rdata$zETW1            CODE
 0001:000077f7 0000002cH .rdata$zETW2            CODE
 0001:00007823 00000001H .rdata$zETW9            CODE
 0001:00007824 0000034cH .rdata$zzzdbg           CODE
 0001:00007b70 00000008H .rtc$IAA                CODE
 0001:00007b78 00000008H .rtc$IZZ                CODE
 0001:00007b80 00000008H .rtc$TAA                CODE
 0001:00007b88 00000008H .rtc$TZZ                CODE
 0001:00007b90 000001e0H .text                   CODE
 0001:00007d70 0000c5f0H .text$mn                CODE
 0001:00014360 00000020H .text$mn$00             CODE
 0001:00014380 00000260H .text$x                 CODE
 0001:000145e0 00000c38H .xdata                  CODE
 0001:00015218 000000f8H .xdata$x                CODE
 0001:00015310 000000afH .edata                  CODE
 0002:00000000 00000940H .data                   DATA
 0002:00000940 000000a0H .data$r                 DATA
 0002:000009e0 00001c68H .bss                    DATA
 0003:00000000 00000fa8H .pdata                  DATA
 0004:00000000 00000248H .idata$5                DATA
 0004:00000248 00000028H .idata$2                DATA
 0004:00000270 00000018H .idata$3                DATA
 0004:00000288 00000248H .idata$4                DATA
 0004:000004d0 00000546H .idata$6                DATA
 0005:00000000 00000080H .gfids$x                DATA
 0005:00000080 00000038H .gfids$y                DATA
 0006:00000000 00000060H .rsrc$01                DATA
 0006:00000060 00000370H .rsrc$02                DATA

  Address         Publics by Value              Rva+Base               Lib:Object

 0000:00000000       __guard_iat_table          0000000000000000     <absolute>
 0000:00000000       __dynamic_value_reloc_table 0000000000000000     <absolute>
 0000:00000000       __guard_iat_count          0000000000000000     <absolute>
 0000:00000000       __guard_longjmp_table      0000000000000000     <absolute>
 0000:00000000       __guard_longjmp_count      0000000000000000     <absolute>
 0000:00000000       __guard_fids_count         0000000000000000     <absolute>
 0000:00000000       ___safe_se_handler_table   0000000000000000     <absolute>
 0000:00000000       ___safe_se_handler_count   0000000000000000     <absolute>
 0000:00000000       __guard_fids_table         0000000000000000     <absolute>
 0000:00000100       __guard_flags              0000000000000100     <absolute>
 0000:00000000       __ImageBase                0000000180000000     <linker-defined>
 0001:00000000       __guard_check_icall_fptr   0000000180001000     LIBCMT:guard_support.obj
 0001:00000008       __guard_dispatch_icall_fptr 0000000180001008     LIBCMT:guard_support.obj
 0001:00000010       __xc_a                     0000000180001010     LIBCMT:initializers.obj
 0001:00000018       __xc_z                     0000000180001018     LIBCMT:initializers.obj
 0001:00000020       __xi_a                     0000000180001020     LIBCMT:initializers.obj
 0001:00000028       __acrt_multibyte_initializer 0000000180001028     libucrt:multibyte_initializer.obj
 0001:00000030       __acrt_stdio_initializer   0000000180001030     libucrt:stdio_initializer.obj
 0001:00000038       __acrt_tran_fma3_initializer 0000000180001038     libucrt:fma3_initializer.obj
 0001:00000040       __xi_z                     0000000180001040     LIBCMT:initializers.obj
 0001:00000048       __xp_a                     0000000180001048     LIBCMT:initializers.obj
 0001:00000050       __acrt_locale_terminator   0000000180001050     libucrt:locale_initializer.obj
 0001:00000058       __dcrt_console_output_terminator 0000000180001058     libucrt:console_output_initializer.obj
 0001:00000060       __acrt_stdio_terminator    0000000180001060     libucrt:stdio_initializer.obj
 0001:00000068       __xp_z                     0000000180001068     LIBCMT:initializers.obj
 0001:00000070       __xt_a                     0000000180001070     LIBCMT:initializers.obj
 0001:00000078       __xt_z                     0000000180001078     LIBCMT:initializers.obj
 0001:00000080       MainGuid                   0000000180001080     AutoWrap.obj
 0001:00000090       MenuGuid                   0000000180001090     AutoWrap.obj
 0001:000000a0       DialogGuid                 00000001800010a0     AutoWrap.obj
 0001:000000b0       ??_7?$DialogItemBinding@UFarDialogItem@@@@6B@ 00000001800010b0     AutoWrap.obj
 0001:000000c0       ??_7PluginCheckBoxBinding@@6B@ 00000001800010c0     AutoWrap.obj
 0001:000000d0       ??_7PluginRadioButtonBinding@@6B@ 00000001800010d0     AutoWrap.obj
 0001:000000e0       ??_7PluginEditFieldBinding@@6B@ 00000001800010e0     AutoWrap.obj
 0001:000000f0       ??_7PluginIntEditFieldBinding@@6B@ 00000001800010f0     AutoWrap.obj
 0001:00000100       ??_C@_15EFLNJKHH@?$AA?$CF?$AAu?$AA?$AA@ 0000000180001100     AutoWrap.obj
 0001:00000108       ??_7PluginUIntEditFieldBinding@@6B@ 0000000180001108     AutoWrap.obj
 0001:00000118       ??_7?$DialogBuilderBase@UFarDialogItem@@@@6B@ 0000000180001118     AutoWrap.obj
 0001:00000160       ??_7PluginDialogBuilder@@6B@ 0000000180001160     AutoWrap.obj
 0001:000001a8       ??_C@_11LOCGONAA@?$AA?$AA@ 00000001800011a8     AutoWrap.obj
 0001:000001b0       ??_C@_1BC@NMCLCAKE@?$AAA?$AAu?$AAt?$AAo?$AAW?$AAr?$AAa?$AAp?$AA?$AA@ 00000001800011b0     AutoWrap.obj
 0001:000001c8       ??_C@_1DE@LDAHMEKD@?$AAA?$AAu?$AAt?$AAo?$AA?5?$AAw?$AAr?$AAa?$AAp?$AA?5?$AAf?$AAo?$AAr?$AA?5?$AAF?$AAa?$AAr?$AA?5?$AAM?$AAa?$AAn?$AAa?$AAg?$AAe?$AAr?$AA?$AA@ 00000001800011c8     AutoWrap.obj
 0001:00000200       ??_C@_1DE@BGKMIKPD@?$AAE?$AAu?$AAg?$AAe?$AAn?$AAe?$AA?5?$AAR?$AAo?$AAs?$AAh?$AAa?$AAl?$AA?5?$AA?$CG?$AA?5?$AAF?$AAa?$AAr?$AA?5?$AAG?$AAr?$AAo?$AAu?$AAp?$AA?$AA@ 0000000180001200     AutoWrap.obj
 0001:00000238       ??_C@_19BFPOADG@?$AAW?$AAr?$AAa?$AAp?$AA?$AA@ 0000000180001238     AutoWrap.obj
 0001:00000248       ??_C@_1BI@JMKBMFLI@?$AAR?$AAi?$AAg?$AAh?$AAt?$AAM?$AAa?$AAr?$AAg?$AAi?$AAn?$AA?$AA@ 0000000180001248     AutoWrap.obj
 0001:00000260       ??_C@_17ECHFBE@?$AA?$CK?$AA?4?$AA?$CK?$AA?$AA@ 0000000180001260     AutoWrap.obj
 0001:00000268       ??_C@_1BE@GBKLIJMP@?$AAF?$AAi?$AAl?$AAe?$AAM?$AAa?$AAs?$AAk?$AAs?$AA?$AA@ 0000000180001268     AutoWrap.obj
 0001:00000280       ??_C@_1CC@MHEGACBP@?$AAE?$AAx?$AAc?$AAl?$AAu?$AAd?$AAe?$AAF?$AAi?$AAl?$AAe?$AAM?$AAa?$AAs?$AAk?$AAs?$AA?$AA@ 0000000180001280     AutoWrap.obj
 0001:000002b0       __xmm@ffffffffffffffff0000000000000002 00000001800012b0     AutoWrap.obj
 0001:000002c0       __xmm@ffffffffffffffffffffffffffffffff 00000001800012c0     AutoWrap.obj
 0001:000002d0       _pRawDllMain               00000001800012d0     LIBCMT:dll_dllmain.obj
 0001:000002d0       _pDefaultRawDllMain        00000001800012d0     LIBCMT:dll_dllmain.obj
 0001:000002e0       ??_7exception@std@@6B@     00000001800012e0     LIBCMT:throw_bad_alloc.obj
 0001:000002f0       ??_C@_0BC@EOODALEL@Unknown?5exception?$AA@ 00000001800012f0     LIBCMT:throw_bad_alloc.obj
 0001:00000310       ??_7bad_alloc@std@@6B@     0000000180001310     LIBCMT:throw_bad_alloc.obj
 0001:00000320       ??_C@_0P@GHFPNOJB@bad?5allocation?$AA@ 0000000180001320     LIBCMT:throw_bad_alloc.obj
 0001:00000338       ??_7bad_array_new_length@std@@6B@ 0000000180001338     LIBCMT:throw_bad_alloc.obj
 0001:00000348       ??_C@_0BF@KINCDENJ@bad?5array?5new?5length?$AA@ 0000000180001348     LIBCMT:throw_bad_alloc.obj
 0001:00000368       ??_7type_info@@6B@         0000000180001368     LIBCMT:std_type_info_static.obj
 0001:00000370       _Microsoft_CRTProvider     0000000180001370     libvcruntime:telemetry.obj
 0001:00000378       ??_C@_00CNPNBAHC@?$AA@     0000000180001378     libvcruntime:telemetry.obj
 0001:00000380       ??_C@_0O@JEOPJOMI@Main?5Invoked?4?$AA@ 0000000180001380     libvcruntime:telemetry.obj
 0001:00000390       ??_C@_0P@NEAEIBDO@Main?5Returned?4?$AA@ 0000000180001390     libvcruntime:telemetry.obj
 0001:00000400       ??_C@_1BC@DNHGCMLG@?$AAa?$AAd?$AAv?$AAa?$AAp?$AAi?$AA3?$AA2?$AA?$AA@ 0000000180001400     libvcruntime:winapi_downlevel.obj
 0001:00000418       ??_C@_1DM@KHCHBNEB@?$AAa?$AAp?$AAi?$AA?9?$AAm?$AAs?$AA?9?$AAw?$AAi?$AAn?$AA?9?$AAc?$AAo?$AAr?$AAe?$AA?9?$AAf?$AAi?$AAb?$AAe?$AAr?$AAs?$AA?9?$AAl?$AA1?$AA?9?$AA1?$AA?9?$AA1?$AA?$AA@ 0000000180001418     libvcruntime:winapi_downlevel.obj
 0001:00000458       ??_C@_1DK@LPPGFMPP@?$AAa?$AAp?$AAi?$AA?9?$AAm?$AAs?$AA?9?$AAw?$AAi?$AAn?$AA?9?$AAc?$AAo?$AAr?$AAe?$AA?9?$AAs?$AAy?$AAn?$AAc?$AAh?$AA?9?$AAl?$AA1?$AA?9?$AA2?$AA?9?$AA0?$AA?$AA@ 0000000180001458     libvcruntime:winapi_downlevel.obj
 0001:00000498       ??_C@_1BC@GDMECMAK@?$AAk?$AAe?$AAr?$AAn?$AAe?$AAl?$AA3?$AA2?$AA?$AA@ 0000000180001498     libvcruntime:winapi_downlevel.obj
 0001:000004b0       ??_C@_0O@BAMBGLIE@EventRegister?$AA@ 00000001800014b0     libvcruntime:winapi_downlevel.obj
 0001:000004c8       ??_C@_0BE@BJEEGHGK@EventSetInformation?$AA@ 00000001800014c8     libvcruntime:winapi_downlevel.obj
 0001:000004e0       ??_C@_0BA@FAKLIPIC@EventUnregister?$AA@ 00000001800014e0     libvcruntime:winapi_downlevel.obj
 0001:000004f8       ??_C@_0BD@PKLHJPHD@EventWriteTransfer?$AA@ 00000001800014f8     libvcruntime:winapi_downlevel.obj
 0001:00000518       ??_C@_08KNHFBNJ@FlsAlloc?$AA@ 0000000180001518     libvcruntime:winapi_downlevel.obj
 0001:00000530       ??_C@_07PEJMOBNF@FlsFree?$AA@ 0000000180001530     libvcruntime:winapi_downlevel.obj
 0001:00000540       ??_C@_0M@GDNOONDI@FlsGetValue?$AA@ 0000000180001540     libvcruntime:winapi_downlevel.obj
 0001:00000558       ??_C@_0M@JCPCPOEF@FlsSetValue?$AA@ 0000000180001558     libvcruntime:winapi_downlevel.obj
 0001:00000570       ??_C@_0BM@HCFOFFN@InitializeCriticalSectionEx?$AA@ 0000000180001570     libvcruntime:winapi_downlevel.obj
 0001:000008b0       ??_C@_08EHJDFFNH@__based?$CI?$AA@ 00000001800018b0     libvcruntime:undname.obj
 0001:000008c0       ??_C@_07KOLFKCDI@__cdecl?$AA@ 00000001800018c0     libvcruntime:undname.obj
 0001:000008c8       ??_C@_08GHMPAG@__pascal?$AA@ 00000001800018c8     libvcruntime:undname.obj
 0001:000008d8       ??_C@_09IFJBGAPI@__stdcall?$AA@ 00000001800018d8     libvcruntime:undname.obj
 0001:000008e8       ??_C@_0L@NPHFGOKO@__thiscall?$AA@ 00000001800018e8     libvcruntime:undname.obj
 0001:000008f8       ??_C@_0L@JMKHOMEK@__fastcall?$AA@ 00000001800018f8     libvcruntime:undname.obj
 0001:00000908       ??_C@_0N@BCKKPABJ@__vectorcall?$AA@ 0000000180001908     libvcruntime:undname.obj
 0001:00000918       ??_C@_09HIJEGCPM@__clrcall?$AA@ 0000000180001918     libvcruntime:undname.obj
 0001:00000924       ??_C@_06GHPCKEAG@__eabi?$AA@ 0000000180001924     libvcruntime:undname.obj
 0001:00000930       ??_C@_07JOMMBBKO@__ptr64?$AA@ 0000000180001930     libvcruntime:undname.obj
 0001:00000938       ??_C@_0L@PILCLIHE@__restrict?$AA@ 0000000180001938     libvcruntime:undname.obj
 0001:00000948       ??_C@_0M@GFIIJFMG@__unaligned?$AA@ 0000000180001948     libvcruntime:undname.obj
 0001:00000958       ??_C@_09DHDLOLLB@restrict?$CI?$AA@ 0000000180001958     libvcruntime:undname.obj
 0001:00000964       ??_C@_04NIHEBCM@?5new?$AA@ 0000000180001964     libvcruntime:undname.obj
 0001:00000970       ??_C@_07FPCDHGMM@?5delete?$AA@ 0000000180001970     libvcruntime:undname.obj
 0001:00000978       ??_C@_01NEMOKFLO@?$DN?$AA@ 0000000180001978     libvcruntime:undname.obj
 0001:0000097c       ??_C@_02GPIOPFAK@?$DO?$DO?$AA@ 000000018000197c     libvcruntime:undname.obj
 0001:00000980       ??_C@_02FODMEDOG@?$DM?$DM?$AA@ 0000000180001980     libvcruntime:undname.obj
 0001:00000984       ??_C@_01DCLJPIOD@?$CB?$AA@ 0000000180001984     libvcruntime:undname.obj
 0001:00000988       ??_C@_02EGOFBIJA@?$DN?$DN?$AA@ 0000000180001988     libvcruntime:undname.obj
 0001:0000098c       ??_C@_02FDNJECIE@?$CB?$DN?$AA@ 000000018000198c     libvcruntime:undname.obj
 0001:00000990       ??_C@_02GPECMEKF@?$FL?$FN?$AA@ 0000000180001990     libvcruntime:undname.obj
 0001:00000998       ??_C@_08LHJFAFGD@operator?$AA@ 0000000180001998     libvcruntime:undname.obj
 0001:000009a4       ??_C@_02HBOOOICD@?9?$DO?$AA@ 00000001800019a4     libvcruntime:undname.obj
 0001:000009a8       ??_C@_01NBENCBCI@?$CK?$AA@ 00000001800019a8     libvcruntime:undname.obj
 0001:000009ac       ??_C@_02ECNGHCIF@?$CL?$CL?$AA@ 00000001800019ac     libvcruntime:undname.obj
 0001:000009b0       ??_C@_02BAABKJLB@?9?9?$AA@ 00000001800019b0     libvcruntime:undname.obj
 0001:000009b4       ??_C@_01JOAMLHOP@?9?$AA@   00000001800019b4     libvcruntime:undname.obj
 0001:000009b8       ??_C@_01MIFGBAGJ@?$CL?$AA@ 00000001800019b8     libvcruntime:undname.obj
 0001:000009bc       ??_C@_01HNPIGOCE@?$CG?$AA@ 00000001800019bc     libvcruntime:undname.obj
 0001:000009c0       ??_C@_03MNHNFDLC@?9?$DO?$CK?$AA@ 00000001800019c0     libvcruntime:undname.obj
 0001:000009c4       ??_C@_01KMDKNFGN@?1?$AA@   00000001800019c4     libvcruntime:undname.obj
 0001:000009c8       ??_C@_01FGNFDNOH@?$CF?$AA@ 00000001800019c8     libvcruntime:undname.obj
 0001:000009cc       ??_C@_01MNNFJEPP@?$DM?$AA@ 00000001800019cc     libvcruntime:undname.obj
 0001:000009d0       ??_C@_02EHCHHCKH@?$DM?$DN?$AA@ 00000001800019d0     libvcruntime:undname.obj
 0001:000009d4       ??_C@_01PPODPGHN@?$DO?$AA@ 00000001800019d4     libvcruntime:undname.obj
 0001:000009d8       ??_C@_02EEKDKGMJ@?$DO?$DN?$AA@ 00000001800019d8     libvcruntime:undname.obj
 0001:000009dc       ??_C@_01IHBHIGKO@?0?$AA@   00000001800019dc     libvcruntime:undname.obj
 0001:000009e0       ??_C@_02HCKGKOFO@?$CI?$CJ?$AA@ 00000001800019e0     libvcruntime:undname.obj
 0001:000009e4       ??_C@_01PJKLJHI@?$HO?$AA@  00000001800019e4     libvcruntime:undname.obj
 0001:000009e8       ??_C@_01JKBOJNNK@?$FO?$AA@ 00000001800019e8     libvcruntime:undname.obj
 0001:000009ec       ??_C@_01DNKMNLPK@?$HM?$AA@ 00000001800019ec     libvcruntime:undname.obj
 0001:000009f0       ??_C@_02PPKAJPJL@?$CG?$CG?$AA@ 00000001800019f0     libvcruntime:undname.obj
 0001:000009f4       ??_C@_02NONPIBCD@?$HM?$HM?$AA@ 00000001800019f4     libvcruntime:undname.obj
 0001:000009f8       ??_C@_02FPIMKNGF@?$CK?$DN?$AA@ 00000001800019f8     libvcruntime:undname.obj
 0001:000009fc       ??_C@_02FOEOMHFC@?$CL?$DN?$AA@ 00000001800019fc     libvcruntime:undname.obj
 0001:00000a00       ??_C@_02FKMDLLOA@?9?$DN?$AA@ 0000000180001a00     libvcruntime:undname.obj
 0001:00000a04       ??_C@_02FJEHGPIO@?1?$DN?$AA@ 0000000180001a04     libvcruntime:undname.obj
 0001:00000a08       ??_C@_02FENAOKFI@?$CF?$DN?$AA@ 0000000180001a08     libvcruntime:undname.obj
 0001:00000a0c       ??_C@_03IKFCCPFF@?$DO?$DO?$DN?$AA@ 0000000180001a0c     libvcruntime:undname.obj
 0001:00000a10       ??_C@_03CDNPDDLA@?$DM?$DM?$DN?$AA@ 0000000180001a10     libvcruntime:undname.obj
 0001:00000a14       ??_C@_02FGJGFEAB@?$CG?$DN?$AA@ 0000000180001a14     libvcruntime:undname.obj
 0001:00000a18       ??_C@_02DHLNPPGH@?$HM?$DN?$AA@ 0000000180001a18     libvcruntime:undname.obj
 0001:00000a1c       ??_C@_02MHEGNOJ@?$FO?$DN?$AA@ 0000000180001a1c     libvcruntime:undname.obj
 0001:00000a20       ??_C@_09IFPLHPGF@?$GAvftable?8?$AA@ 0000000180001a20     libvcruntime:undname.obj
 0001:00000a30       ??_C@_09BLBHBJP@?$GAvbtable?8?$AA@ 0000000180001a30     libvcruntime:undname.obj
 0001:00000a40       ??_C@_07FEEIOKP@?$GAvcall?8?$AA@ 0000000180001a40     libvcruntime:undname.obj
 0001:00000a48       ??_C@_08LLFFHHDJ@?$GAtypeof?8?$AA@ 0000000180001a48     libvcruntime:undname.obj
 0001:00000a58       ??_C@_0BF@KDPPACIK@?$GAlocal?5static?5guard?8?$AA@ 0000000180001a58     libvcruntime:undname.obj
 0001:00000a70       ??_C@_08OBABFOLI@?$GAstring?8?$AA@ 0000000180001a70     libvcruntime:undname.obj
 0001:00000a80       ??_C@_0BD@JDLKDPAB@?$GAvbase?5destructor?8?$AA@ 0000000180001a80     libvcruntime:undname.obj
 0001:00000a98       ??_C@_0BN@DEGPLNFK@?$GAvector?5deleting?5destructor?8?$AA@ 0000000180001a98     libvcruntime:undname.obj
 0001:00000ab8       ??_C@_0BO@OBMKPJIG@?$GAdefault?5constructor?5closure?8?$AA@ 0000000180001ab8     libvcruntime:undname.obj
 0001:00000ad8       ??_C@_0BN@IMDCHIKM@?$GAscalar?5deleting?5destructor?8?$AA@ 0000000180001ad8     libvcruntime:undname.obj
 0001:00000af8       ??_C@_0BO@PFGOCPJJ@?$GAvector?5constructor?5iterator?8?$AA@ 0000000180001af8     libvcruntime:undname.obj
 0001:00000b18       ??_C@_0BN@LFPFMEDL@?$GAvector?5destructor?5iterator?8?$AA@ 0000000180001b18     libvcruntime:undname.obj
 0001:00000b38       ??_C@_0CE@IKBNEHA@?$GAvector?5vbase?5constructor?5iterat@ 0000000180001b38     libvcruntime:undname.obj
 0001:00000b60       ??_C@_0BL@NILFHHPC@?$GAvirtual?5displacement?5map?8?$AA@ 0000000180001b60     libvcruntime:undname.obj
 0001:00000b80       ??_C@_0CB@JONCMFFK@?$GAeh?5vector?5constructor?5iterator?8@ 0000000180001b80     libvcruntime:undname.obj
 0001:00000ba8       ??_C@_0CA@GCEOPDGL@?$GAeh?5vector?5destructor?5iterator?8?$AA@ 0000000180001ba8     libvcruntime:undname.obj
 0001:00000bc8       ??_C@_0CH@OOJPLCPH@?$GAeh?5vector?5vbase?5constructor?5ite@ 0000000180001bc8     libvcruntime:undname.obj
 0001:00000bf0       ??_C@_0BL@LLKPOHJI@?$GAcopy?5constructor?5closure?8?$AA@ 0000000180001bf0     libvcruntime:undname.obj
 0001:00000c10       ??_C@_0BA@KBCDOMBN@?$GAudt?5returning?8?$AA@ 0000000180001c10     libvcruntime:undname.obj
 0001:00000c20       ??_C@_03KLGMFNMG@?$GAEH?$AA@ 0000000180001c20     libvcruntime:undname.obj
 0001:00000c24       ??_C@_05KHLCHHI@?$GARTTI?$AA@ 0000000180001c24     libvcruntime:undname.obj
 0001:00000c30       ??_C@_0BA@KKLDJDLB@?$GAlocal?5vftable?8?$AA@ 0000000180001c30     libvcruntime:undname.obj
 0001:00000c40       ??_C@_0CE@IIHCMGGL@?$GAlocal?5vftable?5constructor?5closu@ 0000000180001c40     libvcruntime:undname.obj
 0001:00000c64       ??_C@_06FHBGPFGH@?5new?$FL?$FN?$AA@ 0000000180001c64     libvcruntime:undname.obj
 0001:00000c70       ??_C@_09LBNFPBCA@?5delete?$FL?$FN?$AA@ 0000000180001c70     libvcruntime:undname.obj
 0001:00000c80       ??_C@_0P@HJKNJFNN@?$GAomni?5callsig?8?$AA@ 0000000180001c80     libvcruntime:undname.obj
 0001:00000c90       ??_C@_0BL@CNOONJFP@?$GAplacement?5delete?5closure?8?$AA@ 0000000180001c90     libvcruntime:undname.obj
 0001:00000cb0       ??_C@_0BN@CKNJLHMB@?$GAplacement?5delete?$FL?$FN?5closure?8?$AA@ 0000000180001cb0     libvcruntime:undname.obj
 0001:00000cd0       ??_C@_0CG@CFDHKGGD@?$GAmanaged?5vector?5constructor?5iter@ 0000000180001cd0     libvcruntime:undname.obj
 0001:00000cf8       ??_C@_0CF@IMGKMJNO@?$GAmanaged?5vector?5destructor?5itera@ 0000000180001cf8     libvcruntime:undname.obj
 0001:00000d20       ??_C@_0CG@HLDDJMAG@?$GAeh?5vector?5copy?5constructor?5iter@ 0000000180001d20     libvcruntime:undname.obj
 0001:00000d48       ??_C@_0CM@FCBBDIGB@?$GAeh?5vector?5vbase?5copy?5constructo@ 0000000180001d48     libvcruntime:undname.obj
 0001:00000d78       ??_C@_0BL@CLIPGLGB@?$GAdynamic?5initializer?5for?5?8?$AA@ 0000000180001d78     libvcruntime:undname.obj
 0001:00000d98       ??_C@_0CB@PDBIFEP@?$GAdynamic?5atexit?5destructor?5for?5?8@ 0000000180001d98     libvcruntime:undname.obj
 0001:00000dc0       ??_C@_0CD@CGAJBKEJ@?$GAvector?5copy?5constructor?5iterato@ 0000000180001dc0     libvcruntime:undname.obj
 0001:00000de8       ??_C@_0CJ@GJELGAMM@?$GAvector?5vbase?5copy?5constructor?5i@ 0000000180001de8     libvcruntime:undname.obj
 0001:00000e18       ??_C@_0CL@FGIJHLCE@?$GAmanaged?5vector?5copy?5constructor@ 0000000180001e18     libvcruntime:undname.obj
 0001:00000e48       ??_C@_0BM@PMGGMLDN@?$GAlocal?5static?5thread?5guard?8?$AA@ 0000000180001e48     libvcruntime:undname.obj
 0001:00000e68       ??_C@_0N@BDNMDMOL@operator?5?$CC?$CC?5?$AA@ 0000000180001e68     libvcruntime:undname.obj
 0001:00000e78       ??_C@_0BC@DAFEJGAK@?5Type?5Descriptor?8?$AA@ 0000000180001e78     libvcruntime:undname.obj
 0001:00000e90       ??_C@_0BM@LDKODKLH@?5Base?5Class?5Descriptor?5at?5?$CI?$AA@ 0000000180001e90     libvcruntime:undname.obj
 0001:00000eb0       ??_C@_0BD@LGICGFMM@?5Base?5Class?5Array?8?$AA@ 0000000180001eb0     libvcruntime:undname.obj
 0001:00000ec8       ??_C@_0BN@MECKDCOJ@?5Class?5Hierarchy?5Descriptor?8?$AA@ 0000000180001ec8     libvcruntime:undname.obj
 0001:00000ee8       ??_C@_0BK@CFCOFLF@?5Complete?5Object?5Locator?8?$AA@ 0000000180001ee8     libvcruntime:undname.obj
 0001:00000f10       __acrt_exception_action_table 0000000180001f10     libucrt:exception_filter.obj
 0001:00000fd0       __acrt_signal_action_table_count 0000000180001fd0     libucrt:exception_filter.obj
 0001:00000fd8       __acrt_signal_action_first_fpe_index 0000000180001fd8     libucrt:exception_filter.obj
 0001:00000fe0       __acrt_signal_action_fpe_count 0000000180001fe0     libucrt:exception_filter.obj
 0001:00000fe8       ??_C@_1BI@BGOHAHKC@?$AAm?$AAs?$AAc?$AAo?$AAr?$AAe?$AAe?$AA?4?$AAd?$AAl?$AAl?$AA?$AA@ 0000000180001fe8     libucrt:exit.obj
 0001:00001000       ??_C@_0P@MIGLKIOC@CorExitProcess?$AA@ 0000000180002000     libucrt:exit.obj
 0001:00001100       __lc_time_c                0000000180002100     libucrt:nlsdata.obj
 0001:000013c0       ??_C@_03KOEHGMDN@Sun?$AA@  00000001800023c0     libucrt:nlsdata.obj
 0001:000013c4       ??_C@_03PDAGKDH@Mon?$AA@   00000001800023c4     libucrt:nlsdata.obj
 0001:000013c8       ??_C@_03NAGEINEP@Tue?$AA@  00000001800023c8     libucrt:nlsdata.obj
 0001:000013cc       ??_C@_03MHOMLAJA@Wed?$AA@  00000001800023cc     libucrt:nlsdata.obj
 0001:000013d0       ??_C@_03IOFIKPDN@Thu?$AA@  00000001800023d0     libucrt:nlsdata.obj
 0001:000013d4       ??_C@_03IDIOELNC@Fri?$AA@  00000001800023d4     libucrt:nlsdata.obj
 0001:000013d8       ??_C@_03FEFJNEK@Sat?$AA@   00000001800023d8     libucrt:nlsdata.obj
 0001:000013dc       ??_C@_06OOPIFAJ@Sunday?$AA@ 00000001800023dc     libucrt:nlsdata.obj
 0001:000013e4       ??_C@_06JLEDEDGH@Monday?$AA@ 00000001800023e4     libucrt:nlsdata.obj
 0001:000013f0       ??_C@_07BAAGCFCM@Tuesday?$AA@ 00000001800023f0     libucrt:nlsdata.obj
 0001:000013f8       ??_C@_09DLIGFAKA@Wednesday?$AA@ 00000001800023f8     libucrt:nlsdata.obj
 0001:00001408       ??_C@_08HACCIKIA@Thursday?$AA@ 0000000180002408     libucrt:nlsdata.obj
 0001:00001414       ??_C@_06JECMNKMI@Friday?$AA@ 0000000180002414     libucrt:nlsdata.obj
 0001:00001420       ??_C@_08INBOOONO@Saturday?$AA@ 0000000180002420     libucrt:nlsdata.obj
 0001:0000142c       ??_C@_03JIHJHPIE@Jan?$AA@  000000018000242c     libucrt:nlsdata.obj
 0001:00001430       ??_C@_03HJBDCHOM@Feb?$AA@  0000000180002430     libucrt:nlsdata.obj
 0001:00001434       ??_C@_03ODNJBKGA@Mar?$AA@  0000000180002434     libucrt:nlsdata.obj
 0001:00001438       ??_C@_03LEOLGMJP@Apr?$AA@  0000000180002438     libucrt:nlsdata.obj
 0001:0000143c       ??_C@_03CNMDKL@May?$AA@    000000018000243c     libucrt:nlsdata.obj
 0001:00001440       ??_C@_03IDFGHECI@Jun?$AA@  0000000180002440     libucrt:nlsdata.obj
 0001:00001444       ??_C@_03LBGABGKK@Jul?$AA@  0000000180002444     libucrt:nlsdata.obj
 0001:00001448       ??_C@_03IFJFEIGA@Aug?$AA@  0000000180002448     libucrt:nlsdata.obj
 0001:0000144c       ??_C@_03GGCAPAJC@Sep?$AA@  000000018000244c     libucrt:nlsdata.obj
 0001:00001450       ??_C@_03BMAOKBAD@Oct?$AA@  0000000180002450     libucrt:nlsdata.obj
 0001:00001454       ??_C@_03JPJOFNIA@Nov?$AA@  0000000180002454     libucrt:nlsdata.obj
 0001:00001458       ??_C@_03MKABNOCG@Dec?$AA@  0000000180002458     libucrt:nlsdata.obj
 0001:00001460       ??_C@_07CGJPFGJA@January?$AA@ 0000000180002460     libucrt:nlsdata.obj
 0001:00001468       ??_C@_08GNJGEPFN@February?$AA@ 0000000180002468     libucrt:nlsdata.obj
 0001:00001474       ??_C@_05HPCKOFNC@March?$AA@ 0000000180002474     libucrt:nlsdata.obj
 0001:0000147c       ??_C@_05DMJDNLEJ@April?$AA@ 000000018000247c     libucrt:nlsdata.obj
 0001:00001484       ??_C@_04CNLMGBGM@June?$AA@ 0000000180002484     libucrt:nlsdata.obj
 0001:0000148c       ??_C@_04MIEPOIFP@July?$AA@ 000000018000248c     libucrt:nlsdata.obj
 0001:00001494       ??_C@_06LBBHFDDG@August?$AA@ 0000000180002494     libucrt:nlsdata.obj
 0001:000014a0       ??_C@_09BHHEALKD@September?$AA@ 00000001800024a0     libucrt:nlsdata.obj
 0001:000014b0       ??_C@_07JJNFCEND@October?$AA@ 00000001800024b0     libucrt:nlsdata.obj
 0001:000014b8       ??_C@_08HCHEGEOA@November?$AA@ 00000001800024b8     libucrt:nlsdata.obj
 0001:000014c8       ??_C@_08EDHMEBNP@December?$AA@ 00000001800024c8     libucrt:nlsdata.obj
 0001:000014d4       ??_C@_02DEDBPAFC@AM?$AA@   00000001800024d4     libucrt:nlsdata.obj
 0001:000014d8       ??_C@_02CJNFDJBF@PM?$AA@   00000001800024d8     libucrt:nlsdata.obj
 0001:000014e0       ??_C@_08BPBNCDIB@MM?1dd?1yy?$AA@ 00000001800024e0     libucrt:nlsdata.obj
 0001:000014f0       ??_C@_0BE@CKGJFCPC@dddd?0?5MMMM?5dd?0?5yyyy?$AA@ 00000001800024f0     libucrt:nlsdata.obj
 0001:00001508       ??_C@_08JCCMCCIL@HH?3mm?3ss?$AA@ 0000000180002508     libucrt:nlsdata.obj
 0001:00001518       ??_C@_17MBGCMIPB@?$AAS?$AAu?$AAn?$AA?$AA@ 0000000180002518     libucrt:nlsdata.obj
 0001:00001520       ??_C@_17KBOMKBF@?$AAM?$AAo?$AAn?$AA?$AA@ 0000000180002520     libucrt:nlsdata.obj
 0001:00001528       ??_C@_17BMKGEGOJ@?$AAT?$AAu?$AAe?$AA?$AA@ 0000000180002528     libucrt:nlsdata.obj
 0001:00001530       ??_C@_17CJEDCEPE@?$AAW?$AAe?$AAd?$AA?$AA@ 0000000180002530     libucrt:nlsdata.obj
 0001:00001538       ??_C@_17PDPHAADD@?$AAT?$AAh?$AAu?$AA?$AA@ 0000000180002538     libucrt:nlsdata.obj
 0001:00001540       ??_C@_17HFOLPPLP@?$AAF?$AAr?$AAi?$AA?$AA@ 0000000180002540     libucrt:nlsdata.obj
 0001:00001548       ??_C@_17GGIBDPIH@?$AAS?$AAa?$AAt?$AA?$AA@ 0000000180002548     libucrt:nlsdata.obj
 0001:00001550       ??_C@_1O@IHNHDHPB@?$AAS?$AAu?$AAn?$AAd?$AAa?$AAy?$AA?$AA@ 0000000180002550     libucrt:nlsdata.obj
 0001:00001560       ??_C@_1O@MMNBFLIA@?$AAM?$AAo?$AAn?$AAd?$AAa?$AAy?$AA?$AA@ 0000000180002560     libucrt:nlsdata.obj
 0001:00001570       ??_C@_1BA@ENFBFFEK@?$AAT?$AAu?$AAe?$AAs?$AAd?$AAa?$AAy?$AA?$AA@ 0000000180002570     libucrt:nlsdata.obj
 0001:00001580       ??_C@_1BE@EBOGMDOH@?$AAW?$AAe?$AAd?$AAn?$AAe?$AAs?$AAd?$AAa?$AAy?$AA?$AA@ 0000000180002580     libucrt:nlsdata.obj
 0001:00001598       ??_C@_1BC@HHMNLIHE@?$AAT?$AAh?$AAu?$AAr?$AAs?$AAd?$AAa?$AAy?$AA?$AA@ 0000000180002598     libucrt:nlsdata.obj
 0001:000015b0       ??_C@_1O@PDICJHAG@?$AAF?$AAr?$AAi?$AAd?$AAa?$AAy?$AA?$AA@ 00000001800025b0     libucrt:nlsdata.obj
 0001:000015c0       ??_C@_1BC@ENMNNPAJ@?$AAS?$AAa?$AAt?$AAu?$AAr?$AAd?$AAa?$AAy?$AA?$AA@ 00000001800025c0     libucrt:nlsdata.obj
 0001:000015d8       ??_C@_17DKNBKCHM@?$AAJ?$AAa?$AAn?$AA?$AA@ 00000001800025d8     libucrt:nlsdata.obj
 0001:000015e0       ??_C@_17LMDJEKJN@?$AAF?$AAe?$AAb?$AA?$AA@ 00000001800025e0     libucrt:nlsdata.obj
 0001:000015e8       ??_C@_17CKNLEDEC@?$AAM?$AAa?$AAr?$AA?$AA@ 00000001800025e8     libucrt:nlsdata.obj
 0001:000015f0       ??_C@_17LFPOIHDD@?$AAA?$AAp?$AAr?$AA?$AA@ 00000001800025f0     libucrt:nlsdata.obj
 0001:000015f8       ??_C@_17PNNKMEED@?$AAM?$AAa?$AAy?$AA?$AA@ 00000001800025f8     libucrt:nlsdata.obj
 0001:00001600       ??_C@_17KCJGOCPB@?$AAJ?$AAu?$AAn?$AA?$AA@ 0000000180002600     libucrt:nlsdata.obj
 0001:00001608       ??_C@_17IJPCKHK@?$AAJ?$AAu?$AAl?$AA?$AA@ 0000000180002608     libucrt:nlsdata.obj
 0001:00001610       ??_C@_17ICPELBCN@?$AAA?$AAu?$AAg?$AA?$AA@ 0000000180002610     libucrt:nlsdata.obj
 0001:00001618       ??_C@_17HCHCOKMG@?$AAS?$AAe?$AAp?$AA?$AA@ 0000000180002618     libucrt:nlsdata.obj
 0001:00001620       ??_C@_17FNLKOI@?$AAO?$AAc?$AAt?$AA?$AA@ 0000000180002620     libucrt:nlsdata.obj
 0001:00001628       ??_C@_17BBDMLCIG@?$AAN?$AAo?$AAv?$AA?$AA@ 0000000180002628     libucrt:nlsdata.obj
 0001:00001630       ??_C@_17EGKACKIF@?$AAD?$AAe?$AAc?$AA?$AA@ 0000000180002630     libucrt:nlsdata.obj
 0001:00001638       ??_C@_1BA@EFMEIEBA@?$AAJ?$AAa?$AAn?$AAu?$AAa?$AAr?$AAy?$AA?$AA@ 0000000180002638     libucrt:nlsdata.obj
 0001:00001648       ??_C@_1BC@JGDDFFAM@?$AAF?$AAe?$AAb?$AAr?$AAu?$AAa?$AAr?$AAy?$AA?$AA@ 0000000180002648     libucrt:nlsdata.obj
 0001:00001660       ??_C@_1M@IKEENEDF@?$AAM?$AAa?$AAr?$AAc?$AAh?$AA?$AA@ 0000000180002660     libucrt:nlsdata.obj
 0001:00001670       ??_C@_1M@GJNLMHFD@?$AAA?$AAp?$AAr?$AAi?$AAl?$AA?$AA@ 0000000180002670     libucrt:nlsdata.obj
 0001:00001680       ??_C@_19EPFLPGAP@?$AAJ?$AAu?$AAn?$AAe?$AA?$AA@ 0000000180002680     libucrt:nlsdata.obj
 0001:00001690       ??_C@_19BIFMLPCD@?$AAJ?$AAu?$AAl?$AAy?$AA?$AA@ 0000000180002690     libucrt:nlsdata.obj
 0001:000016a0       ??_C@_1O@PAHLKOAC@?$AAA?$AAu?$AAg?$AAu?$AAs?$AAt?$AA?$AA@ 00000001800026a0     libucrt:nlsdata.obj
 0001:000016b0       ??_C@_1BE@DKAAMBJL@?$AAS?$AAe?$AAp?$AAt?$AAe?$AAm?$AAb?$AAe?$AAr?$AA?$AA@ 00000001800026b0     libucrt:nlsdata.obj
 0001:000016c8       ??_C@_1BA@EPANDLNG@?$AAO?$AAc?$AAt?$AAo?$AAb?$AAe?$AAr?$AA?$AA@ 00000001800026c8     libucrt:nlsdata.obj
 0001:000016d8       ??_C@_1BC@BGLIFPF@?$AAN?$AAo?$AAv?$AAe?$AAm?$AAb?$AAe?$AAr?$AA?$AA@ 00000001800026d8     libucrt:nlsdata.obj
 0001:000016f0       ??_C@_1BC@FEMKIFH@?$AAD?$AAe?$AAc?$AAe?$AAm?$AAb?$AAe?$AAr?$AA?$AA@ 00000001800026f0     libucrt:nlsdata.obj
 0001:00001704       ??_C@_15ODEHAHHF@?$AAA?$AAM?$AA?$AA@ 0000000180002704     libucrt:nlsdata.obj
 0001:0000170c       ??_C@_15CLMNNGEL@?$AAP?$AAM?$AA?$AA@ 000000018000270c     libucrt:nlsdata.obj
 0001:00001718       ??_C@_1BC@IEBCMHCM@?$AAM?$AAM?$AA?1?$AAd?$AAd?$AA?1?$AAy?$AAy?$AA?$AA@ 0000000180002718     libucrt:nlsdata.obj
 0001:00001730       ??_C@_1CI@KNAKOEBC@?$AAd?$AAd?$AAd?$AAd?$AA?0?$AA?5?$AAM?$AAM?$AAM?$AAM?$AA?5?$AAd?$AAd?$AA?0?$AA?5?$AAy?$AAy?$AAy?$AAy?$AA?$AA@ 0000000180002730     libucrt:nlsdata.obj
 0001:00001758       ??_C@_1BC@GDGBMEMK@?$AAH?$AAH?$AA?3?$AAm?$AAm?$AA?3?$AAs?$AAs?$AA?$AA@ 0000000180002758     libucrt:nlsdata.obj
 0001:00001770       ??_C@_1M@BMHNFIME@?$AAe?$AAn?$AA?9?$AAU?$AAS?$AA?$AA@ 0000000180002770     libucrt:nlsdata.obj
 0001:00001820       ??_C@_1EG@CNNIPFIM@?$AAa?$AAp?$AAi?$AA?9?$AAm?$AAs?$AA?9?$AAw?$AAi?$AAn?$AA?9?$AAa?$AAp?$AAp?$AAm?$AAo?$AAd?$AAe?$AAl?$AA?9?$AAr?$AAu?$AAn?$AAt?$AAi?$AAm?$AAe?$AA?9?$AAl?$AA1?$AA?9?$AA1@ 0000000180002820     libucrt:winapi_thunks.obj
 0001:00001870       ??_C@_1EA@JGEFHKEI@?$AAa?$AAp?$AAi?$AA?9?$AAm?$AAs?$AA?9?$AAw?$AAi?$AAn?$AA?9?$AAc?$AAo?$AAr?$AAe?$AA?9?$AAd?$AAa?$AAt?$AAe?$AAt?$AAi?$AAm?$AAe?$AA?9?$AAl?$AA1?$AA?9?$AA1?$AA?9?$AA1?$AA?$AA@ 0000000180002870     libucrt:winapi_thunks.obj
 0001:000018b0       ??_C@_1DI@GCIAAENM@?$AAa?$AAp?$AAi?$AA?9?$AAm?$AAs?$AA?9?$AAw?$AAi?$AAn?$AA?9?$AAc?$AAo?$AAr?$AAe?$AA?9?$AAf?$AAi?$AAl?$AAe?$AA?9?$AAl?$AA2?$AA?9?$AA1?$AA?9?$AA1?$AA?$AA@ 00000001800028b0     libucrt:winapi_thunks.obj
 0001:000018f0       ??_C@_1EI@MPIAOHOC@?$AAa?$AAp?$AAi?$AA?9?$AAm?$AAs?$AA?9?$AAw?$AAi?$AAn?$AA?9?$AAc?$AAo?$AAr?$AAe?$AA?9?$AAl?$AAo?$AAc?$AAa?$AAl?$AAi?$AAz?$AAa?$AAt?$AAi?$AAo?$AAn?$AA?9?$AAl?$AA1?$AA?9@ 00000001800028f0     libucrt:winapi_thunks.obj
 0001:00001940       ??_C@_1FK@FPHCKFIE@?$AAa?$AAp?$AAi?$AA?9?$AAm?$AAs?$AA?9?$AAw?$AAi?$AAn?$AA?9?$AAc?$AAo?$AAr?$AAe?$AA?9?$AAl?$AAo?$AAc?$AAa?$AAl?$AAi?$AAz?$AAa?$AAt?$AAi?$AAo?$AAn?$AA?9?$AAo?$AAb?$AAs@ 0000000180002940     libucrt:winapi_thunks.obj
 0001:000019a0       ??_C@_1EM@DILCGIIO@?$AAa?$AAp?$AAi?$AA?9?$AAm?$AAs?$AA?9?$AAw?$AAi?$AAn?$AA?9?$AAc?$AAo?$AAr?$AAe?$AA?9?$AAp?$AAr?$AAo?$AAc?$AAe?$AAs?$AAs?$AAt?$AAh?$AAr?$AAe?$AAa?$AAd?$AAs?$AA?9?$AAl@ 00000001800029a0     libucrt:winapi_thunks.obj
 0001:000019f0       ??_C@_1DM@LNCGDDPN@?$AAa?$AAp?$AAi?$AA?9?$AAm?$AAs?$AA?9?$AAw?$AAi?$AAn?$AA?9?$AAc?$AAo?$AAr?$AAe?$AA?9?$AAs?$AAt?$AAr?$AAi?$AAn?$AAg?$AA?9?$AAl?$AA1?$AA?9?$AA1?$AA?9?$AA0?$AA?$AA@ 00000001800029f0     libucrt:winapi_thunks.obj
 0001:00001a30       ??_C@_1DO@FPAPJEMD@?$AAa?$AAp?$AAi?$AA?9?$AAm?$AAs?$AA?9?$AAw?$AAi?$AAn?$AA?9?$AAc?$AAo?$AAr?$AAe?$AA?9?$AAs?$AAy?$AAs?$AAi?$AAn?$AAf?$AAo?$AA?9?$AAl?$AA1?$AA?9?$AA2?$AA?9?$AA1?$AA?$AA@ 0000000180002a30     libucrt:winapi_thunks.obj
 0001:00001a70       ??_C@_1DK@NDHNAHIO@?$AAa?$AAp?$AAi?$AA?9?$AAm?$AAs?$AA?9?$AAw?$AAi?$AAn?$AA?9?$AAc?$AAo?$AAr?$AAe?$AA?9?$AAw?$AAi?$AAn?$AAr?$AAt?$AA?9?$AAl?$AA1?$AA?9?$AA1?$AA?9?$AA0?$AA?$AA@ 0000000180002a70     libucrt:winapi_thunks.obj
 0001:00001ab0       ??_C@_1DM@KGHDGBCM@?$AAa?$AAp?$AAi?$AA?9?$AAm?$AAs?$AA?9?$AAw?$AAi?$AAn?$AA?9?$AAc?$AAo?$AAr?$AAe?$AA?9?$AAx?$AAs?$AAt?$AAa?$AAt?$AAe?$AA?9?$AAl?$AA2?$AA?9?$AA1?$AA?9?$AA0?$AA?$AA@ 0000000180002ab0     libucrt:winapi_thunks.obj
 0001:00001af0       ??_C@_1EO@IJIOEFOH@?$AAa?$AAp?$AAi?$AA?9?$AAm?$AAs?$AA?9?$AAw?$AAi?$AAn?$AA?9?$AAr?$AAt?$AAc?$AAo?$AAr?$AAe?$AA?9?$AAn?$AAt?$AAu?$AAs?$AAe?$AAr?$AA?9?$AAw?$AAi?$AAn?$AAd?$AAo?$AAw?$AA?9@ 0000000180002af0     libucrt:winapi_thunks.obj
 0001:00001b40       ??_C@_1FG@HHGEKANL@?$AAa?$AAp?$AAi?$AA?9?$AAm?$AAs?$AA?9?$AAw?$AAi?$AAn?$AA?9?$AAs?$AAe?$AAc?$AAu?$AAr?$AAi?$AAt?$AAy?$AA?9?$AAs?$AAy?$AAs?$AAt?$AAe?$AAm?$AAf?$AAu?$AAn?$AAc?$AAt?$AAi@ 0000000180002b40     libucrt:winapi_thunks.obj
 0001:00001ba0       ??_C@_1FG@NCKKOLKO@?$AAe?$AAx?$AAt?$AA?9?$AAm?$AAs?$AA?9?$AAw?$AAi?$AAn?$AA?9?$AAk?$AAe?$AAr?$AAn?$AAe?$AAl?$AA3?$AA2?$AA?9?$AAp?$AAa?$AAc?$AAk?$AAa?$AAg?$AAe?$AA?9?$AAc?$AAu?$AAr?$AAr@ 0000000180002ba0     libucrt:winapi_thunks.obj
 0001:00001c00       ??_C@_1EG@DBIOJECG@?$AAe?$AAx?$AAt?$AA?9?$AAm?$AAs?$AA?9?$AAw?$AAi?$AAn?$AA?9?$AAn?$AAt?$AAu?$AAs?$AAe?$AAr?$AA?9?$AAd?$AAi?$AAa?$AAl?$AAo?$AAg?$AAb?$AAo?$AAx?$AA?9?$AAl?$AA1?$AA?9?$AA1@ 0000000180002c00     libucrt:winapi_thunks.obj
 0001:00001c50       ??_C@_1EO@FIHMJCLF@?$AAe?$AAx?$AAt?$AA?9?$AAm?$AAs?$AA?9?$AAw?$AAi?$AAn?$AA?9?$AAn?$AAt?$AAu?$AAs?$AAe?$AAr?$AA?9?$AAw?$AAi?$AAn?$AAd?$AAo?$AAw?$AAs?$AAt?$AAa?$AAt?$AAi?$AAo?$AAn?$AA?9@ 0000000180002c50     libucrt:winapi_thunks.obj
 0001:00001ca0       ??_C@_1O@BCCLBEOE@?$AAu?$AAs?$AAe?$AAr?$AA3?$AA2?$AA?$AA@ 0000000180002ca0     libucrt:winapi_thunks.obj
 0001:00001cd8       ??_C@_0BE@JOGNEJCI@GetCurrentPackageId?$AA@ 0000000180002cd8     libucrt:winapi_thunks.obj
 0001:00001d00       ??_C@_0O@KKBNKAPF@LCMapStringEx?$AA@ 0000000180002d00     libucrt:winapi_thunks.obj
 0001:00001d18       ??_C@_0BB@HBDEELFH@LocaleNameToLCID?$AA@ 0000000180002d18     libucrt:winapi_thunks.obj
 0001:00001eb8       ??_C@_1M@HPNHIDJI@?$AAj?$AAa?$AA?9?$AAJ?$AAP?$AA?$AA@ 0000000180002eb8     libucrt:mbctype.obj
 0001:00001ec8       ??_C@_1M@BIBDDEMK@?$AAz?$AAh?$AA?9?$AAC?$AAN?$AA?$AA@ 0000000180002ec8     libucrt:mbctype.obj
 0001:00001ed8       ??_C@_1M@JLOOOEGK@?$AAk?$AAo?$AA?9?$AAK?$AAR?$AA?$AA@ 0000000180002ed8     libucrt:mbctype.obj
 0001:00001ee8       ??_C@_1M@CLNBBOPM@?$AAz?$AAh?$AA?9?$AAT?$AAW?$AA?$AA@ 0000000180002ee8     libucrt:mbctype.obj
 0001:00001f00       __newctype                 0000000180002f00     libucrt:ctype.obj
 0001:00002200       __newclmap                 0000000180003200     libucrt:ctype.obj
 0001:00002380       __newcumap                 0000000180003380     libucrt:ctype.obj
 0001:00002500       _wctype                    0000000180003500     libucrt:ctype.obj
 0001:00002704       ??_C@_15PJPFLCCM@?$AAu?$AAk?$AA?$AA@ 0000000180003704     libucrt:get_qualified_locale.obj
 0001:00003550       ??_C@_15EMKDOKLE@?$AAa?$AAr?$AA?$AA@ 0000000180004550     libucrt:lcidtoname_downlevel.obj
 0001:00003558       ??_C@_15KNPADPLH@?$AAb?$AAg?$AA?$AA@ 0000000180004558     libucrt:lcidtoname_downlevel.obj
 0001:00003560       ??_C@_15EDMHLDMO@?$AAc?$AAa?$AA?$AA@ 0000000180004560     libucrt:lcidtoname_downlevel.obj
 0001:00003568       ??_C@_1O@BPEAJADD@?$AAz?$AAh?$AA?9?$AAC?$AAH?$AAS?$AA?$AA@ 0000000180004568     libucrt:lcidtoname_downlevel.obj
 0001:00003578       ??_C@_15LJNHCMNK@?$AAc?$AAs?$AA?$AA@ 0000000180004578     libucrt:lcidtoname_downlevel.obj
 0001:00003580       ??_C@_15FOMCIDHG@?$AAd?$AAa?$AA?$AA@ 0000000180004580     libucrt:lcidtoname_downlevel.obj
 0001:00003588       ??_C@_15NBKABECB@?$AAd?$AAe?$AA?$AA@ 0000000180004588     libucrt:lcidtoname_downlevel.obj
 0001:00003590       ??_C@_15GHPEIIAO@?$AAe?$AAl?$AA?$AA@ 0000000180004590     libucrt:lcidtoname_downlevel.obj
 0001:00003598       ??_C@_15MNPNEAIF@?$AAe?$AAn?$AA?$AA@ 0000000180004598     libucrt:lcidtoname_downlevel.obj
 0001:000035a0       ??_C@_15GPIOMPMH@?$AAe?$AAs?$AA?$AA@ 00000001800045a0     libucrt:lcidtoname_downlevel.obj
 0001:000035a8       ??_C@_15NGLOAKJC@?$AAf?$AAi?$AA?$AA@ 00000001800045a8     libucrt:lcidtoname_downlevel.obj
 0001:000035b0       ??_C@_15FBKGNKAM@?$AAf?$AAr?$AA?$AA@ 00000001800045b0     libucrt:lcidtoname_downlevel.obj
 0001:000035b8       ??_C@_15KGGCNEFK@?$AAh?$AAe?$AA?$AA@ 00000001800045b8     libucrt:lcidtoname_downlevel.obj
 0001:000035c0       ??_C@_15PGHLIDMF@?$AAh?$AAu?$AA?$AA@ 00000001800045c0     libucrt:lcidtoname_downlevel.obj
 0001:000035c8       ??_C@_15BIEMAPLM@?$AAi?$AAs?$AA?$AA@ 00000001800045c8     libucrt:lcidtoname_downlevel.obj
 0001:000035d0       ??_C@_15IFJLDHAF@?$AAi?$AAt?$AA?$AA@ 00000001800045d0     libucrt:lcidtoname_downlevel.obj
 0001:000035d8       ??_C@_15GEMIOCAG@?$AAj?$AAa?$AA?$AA@ 00000001800045d8     libucrt:lcidtoname_downlevel.obj
 0001:000035e0       ??_C@_15EPELEGJA@?$AAk?$AAo?$AA?$AA@ 00000001800045e0     libucrt:lcidtoname_downlevel.obj
 0001:000035e8       ??_C@_15NDDHIMN@?$AAn?$AAl?$AA?$AA@ 00000001800045e8     libucrt:lcidtoname_downlevel.obj
 0001:000035f0       ??_C@_15BPIGNHCD@?$AAn?$AAo?$AA?$AA@ 00000001800045f0     libucrt:lcidtoname_downlevel.obj
 0001:000035f8       ??_C@_15DEOPBLCG@?$AAp?$AAl?$AA?$AA@ 00000001800045f8     libucrt:lcidtoname_downlevel.obj
 0001:00003600       ??_C@_15KBECGEFG@?$AAp?$AAt?$AA?$AA@ 0000000180004600     libucrt:lcidtoname_downlevel.obj
 0001:00003608       ??_C@_15GLJCBFMD@?$AAr?$AAo?$AA?$AA@ 0000000180004608     libucrt:lcidtoname_downlevel.obj
 0001:00003610       ??_C@_15FEDGKCDI@?$AAr?$AAu?$AA?$AA@ 0000000180004610     libucrt:lcidtoname_downlevel.obj
 0001:00003618       ??_C@_15GLKMLLHM@?$AAh?$AAr?$AA?$AA@ 0000000180004618     libucrt:lcidtoname_downlevel.obj
 0001:00003620       ??_C@_15CPKMFBDB@?$AAs?$AAk?$AA?$AA@ 0000000180004620     libucrt:lcidtoname_downlevel.obj
 0001:00003628       ??_C@_15BAAIOGMK@?$AAs?$AAq?$AA?$AA@ 0000000180004628     libucrt:lcidtoname_downlevel.obj
 0001:00003630       ??_C@_15INNPNOHD@?$AAs?$AAv?$AA?$AA@ 0000000180004630     libucrt:lcidtoname_downlevel.obj
 0001:00003638       ??_C@_15CABMMOGH@?$AAt?$AAh?$AA?$AA@ 0000000180004638     libucrt:lcidtoname_downlevel.obj
 0001:00003640       ??_C@_15BPLIHJJM@?$AAt?$AAr?$AA?$AA@ 0000000180004640     libucrt:lcidtoname_downlevel.obj
 0001:00003648       ??_C@_15NEOEKKDJ@?$AAu?$AAr?$AA?$AA@ 0000000180004648     libucrt:lcidtoname_downlevel.obj
 0001:00003650       ??_C@_15NFICGAJK@?$AAi?$AAd?$AA?$AA@ 0000000180004650     libucrt:lcidtoname_downlevel.obj
 0001:00003658       ??_C@_15HPJPHDM@?$AAb?$AAe?$AA?$AA@ 0000000180004658     libucrt:lcidtoname_downlevel.obj
 0001:00003660       ??_C@_15LCHLGJII@?$AAs?$AAl?$AA?$AA@ 0000000180004660     libucrt:lcidtoname_downlevel.obj
 0001:00003668       ??_C@_15PCFJPHHO@?$AAe?$AAt?$AA?$AA@ 0000000180004668     libucrt:lcidtoname_downlevel.obj
 0001:00003670       ??_C@_15HPFPGODN@?$AAl?$AAv?$AA?$AA@ 0000000180004670     libucrt:lcidtoname_downlevel.obj
 0001:00003678       ??_C@_15NFFGKGLG@?$AAl?$AAt?$AA?$AA@ 0000000180004678     libucrt:lcidtoname_downlevel.obj
 0001:00003680       ??_C@_15BDAKCCHN@?$AAf?$AAa?$AA?$AA@ 0000000180004680     libucrt:lcidtoname_downlevel.obj
 0001:00003688       ??_C@_15NFGIAIAJ@?$AAv?$AAi?$AA?$AA@ 0000000180004688     libucrt:lcidtoname_downlevel.obj
 0001:00003690       ??_C@_15LMKNDMHN@?$AAh?$AAy?$AA?$AA@ 0000000180004690     libucrt:lcidtoname_downlevel.obj
 0001:00003698       ??_C@_15IJBHMCFL@?$AAa?$AAz?$AA?$AA@ 0000000180004698     libucrt:lcidtoname_downlevel.obj
 0001:000036a0       ??_C@_15EKOFJABL@?$AAe?$AAu?$AA?$AA@ 00000001800046a0     libucrt:lcidtoname_downlevel.obj
 0001:000036a8       ??_C@_15BGHADCNK@?$AAm?$AAk?$AA?$AA@ 00000001800046a8     libucrt:lcidtoname_downlevel.obj
 0001:000036b0       ??_C@_15JDNICKHM@?$AAa?$AAf?$AA?$AA@ 00000001800046b0     libucrt:lcidtoname_downlevel.obj
 0001:000036b8       ??_C@_15KPJEDBKD@?$AAk?$AAa?$AA?$AA@ 00000001800046b8     libucrt:lcidtoname_downlevel.obj
 0001:000036c0       ??_C@_15PDNFFFEO@?$AAf?$AAo?$AA?$AA@ 00000001800046c0     libucrt:lcidtoname_downlevel.obj
 0001:000036c8       ??_C@_15OMLEGLOC@?$AAh?$AAi?$AA?$AA@ 00000001800046c8     libucrt:lcidtoname_downlevel.obj
 0001:000036d0       ??_C@_15IDNNENKK@?$AAm?$AAs?$AA?$AA@ 00000001800046d0     libucrt:lcidtoname_downlevel.obj
 0001:000036d8       ??_C@_15MACJNBMH@?$AAk?$AAk?$AA?$AA@ 00000001800046d8     libucrt:lcidtoname_downlevel.obj
 0001:000036e0       ??_C@_15DKDJEOND@?$AAk?$AAy?$AA?$AA@ 00000001800046e0     libucrt:lcidtoname_downlevel.obj
 0001:000036e8       ??_C@_15DFGDLJBG@?$AAs?$AAw?$AA?$AA@ 00000001800046e8     libucrt:lcidtoname_downlevel.obj
 0001:000036f0       ??_C@_15BBFAICNG@?$AAu?$AAz?$AA?$AA@ 00000001800046f0     libucrt:lcidtoname_downlevel.obj
 0001:000036f8       ??_C@_15DKNDCGEA@?$AAt?$AAt?$AA?$AA@ 00000001800046f8     libucrt:lcidtoname_downlevel.obj
 0001:00003700       ??_C@_15MGIFMDPL@?$AAp?$AAa?$AA?$AA@ 0000000180004700     libucrt:lcidtoname_downlevel.obj
 0001:00003708       ??_C@_15HCNDBBA@?$AAg?$AAu?$AA?$AA@ 0000000180004708     libucrt:lcidtoname_downlevel.obj
 0001:00003710       ??_C@_15FNBEIBON@?$AAt?$AAa?$AA?$AA@ 0000000180004710     libucrt:lcidtoname_downlevel.obj
 0001:00003718       ??_C@_15NCHGBGLK@?$AAt?$AAe?$AA?$AA@ 0000000180004718     libucrt:lcidtoname_downlevel.obj
 0001:00003720       ??_C@_15PHPHCBPF@?$AAk?$AAn?$AA?$AA@ 0000000180004720     libucrt:lcidtoname_downlevel.obj
 0001:00003728       ??_C@_15DLGBCKMP@?$AAm?$AAr?$AA?$AA@ 0000000180004728     libucrt:lcidtoname_downlevel.obj
 0001:00003730       ??_C@_15EABBLBFF@?$AAs?$AAa?$AA?$AA@ 0000000180004730     libucrt:lcidtoname_downlevel.obj
 0001:00003738       ??_C@_15CBKOMCOI@?$AAm?$AAn?$AA?$AA@ 0000000180004738     libucrt:lcidtoname_downlevel.obj
 0001:00003740       ??_C@_15CKDMCJAF@?$AAg?$AAl?$AA?$AA@ 0000000180004740     libucrt:lcidtoname_downlevel.obj
 0001:00003748       ??_C@_17CNJFBPG@?$AAk?$AAo?$AAk?$AA?$AA@ 0000000180004748     libucrt:lcidtoname_downlevel.obj
 0001:00003750       ??_C@_17FFBJICPL@?$AAs?$AAy?$AAr?$AA?$AA@ 0000000180004750     libucrt:lcidtoname_downlevel.obj
 0001:00003758       ??_C@_17KPNDCPAF@?$AAd?$AAi?$AAv?$AA?$AA@ 0000000180004758     libucrt:lcidtoname_downlevel.obj
 0001:00003760       ??_C@_1M@OKAHONE@?$AAa?$AAr?$AA?9?$AAS?$AAA?$AA?$AA@ 0000000180004760     libucrt:lcidtoname_downlevel.obj
 0001:00003770       ??_C@_1M@FFFIGIGK@?$AAb?$AAg?$AA?9?$AAB?$AAG?$AA?$AA@ 0000000180004770     libucrt:lcidtoname_downlevel.obj
 0001:00003780       ??_C@_1M@BJNKEDC@?$AAc?$AAa?$AA?9?$AAE?$AAS?$AA?$AA@ 0000000180004780     libucrt:lcidtoname_downlevel.obj
 0001:00003790       ??_C@_1M@IJJHFJHA@?$AAc?$AAs?$AA?9?$AAC?$AAZ?$AA?$AA@ 0000000180004790     libucrt:lcidtoname_downlevel.obj
 0001:000037a0       ??_C@_1M@CLPEOBGI@?$AAd?$AAa?$AA?9?$AAD?$AAK?$AA?$AA@ 00000001800047a0     libucrt:lcidtoname_downlevel.obj
 0001:000037b0       ??_C@_1M@MCMADGCB@?$AAd?$AAe?$AA?9?$AAD?$AAE?$AA?$AA@ 00000001800047b0     libucrt:lcidtoname_downlevel.obj
 0001:000037c0       ??_C@_1M@OOCKEMAM@?$AAe?$AAl?$AA?9?$AAG?$AAR?$AA?$AA@ 00000001800047c0     libucrt:lcidtoname_downlevel.obj
 0001:000037d0       ??_C@_1M@DDNJFGID@?$AAf?$AAi?$AA?9?$AAF?$AAI?$AA?$AA@ 00000001800047d0     libucrt:lcidtoname_downlevel.obj
 0001:000037e0       ??_C@_1M@GLIPPMAC@?$AAf?$AAr?$AA?9?$AAF?$AAR?$AA?$AA@ 00000001800047e0     libucrt:lcidtoname_downlevel.obj
 0001:000037f0       ??_C@_1M@GFMCHPE@?$AAh?$AAe?$AA?9?$AAI?$AAL?$AA?$AA@ 00000001800047f0     libucrt:lcidtoname_downlevel.obj
 0001:00003800       ??_C@_1M@MHLPGNKM@?$AAh?$AAu?$AA?9?$AAH?$AAU?$AA?$AA@ 0000000180004800     libucrt:lcidtoname_downlevel.obj
 0001:00003810       ??_C@_1M@LPDDNNPN@?$AAi?$AAs?$AA?9?$AAI?$AAS?$AA?$AA@ 0000000180004810     libucrt:lcidtoname_downlevel.obj
 0001:00003820       ??_C@_1M@MADIPODN@?$AAi?$AAt?$AA?9?$AAI?$AAT?$AA?$AA@ 0000000180004820     libucrt:lcidtoname_downlevel.obj
 0001:00003830       ??_C@_1M@IHBJJGG@?$AAn?$AAl?$AA?9?$AAN?$AAL?$AA?$AA@ 0000000180004830     libucrt:lcidtoname_downlevel.obj
 0001:00003840       ??_C@_1M@EANAGDL@?$AAn?$AAb?$AA?9?$AAN?$AAO?$AA?$AA@ 0000000180004840     libucrt:lcidtoname_downlevel.obj
 0001:00003850       ??_C@_1M@NEIEMEGP@?$AAp?$AAl?$AA?9?$AAP?$AAL?$AA?$AA@ 0000000180004850     libucrt:lcidtoname_downlevel.obj
 0001:00003860       ??_C@_1M@BOCFIGEP@?$AAp?$AAt?$AA?9?$AAB?$AAR?$AA?$AA@ 0000000180004860     libucrt:lcidtoname_downlevel.obj
 0001:00003870       ??_C@_1M@IMPFOPBG@?$AAr?$AAo?$AA?9?$AAR?$AAO?$AA?$AA@ 0000000180004870     libucrt:lcidtoname_downlevel.obj
 0001:00003880       ??_C@_1M@IDNNEJMM@?$AAr?$AAu?$AA?9?$AAR?$AAU?$AA?$AA@ 0000000180004880     libucrt:lcidtoname_downlevel.obj
 0001:00003890       ??_C@_1M@LILEEOGM@?$AAh?$AAr?$AA?9?$AAH?$AAR?$AA?$AA@ 0000000180004890     libucrt:lcidtoname_downlevel.obj
 0001:000038a0       ??_C@_1M@FKIFEHPB@?$AAs?$AAk?$AA?9?$AAS?$AAK?$AA?$AA@ 00000001800048a0     libucrt:lcidtoname_downlevel.obj
 0001:000038b0       ??_C@_1M@LJMAMNPJ@?$AAs?$AAq?$AA?9?$AAA?$AAL?$AA?$AA@ 00000001800048b0     libucrt:lcidtoname_downlevel.obj
 0001:000038c0       ??_C@_1M@GIAKDKJK@?$AAs?$AAv?$AA?9?$AAS?$AAE?$AA?$AA@ 00000001800048c0     libucrt:lcidtoname_downlevel.obj
 0001:000038d0       ??_C@_1M@MKJKIKCL@?$AAt?$AAh?$AA?9?$AAT?$AAH?$AA?$AA@ 00000001800048d0     libucrt:lcidtoname_downlevel.obj
 0001:000038e0       ??_C@_1M@MFLCCMPB@?$AAt?$AAr?$AA?9?$AAT?$AAR?$AA?$AA@ 00000001800048e0     libucrt:lcidtoname_downlevel.obj
 0001:000038f0       ??_C@_1M@OIJHDKJN@?$AAu?$AAr?$AA?9?$AAP?$AAK?$AA?$AA@ 00000001800048f0     libucrt:lcidtoname_downlevel.obj
 0001:00003900       ??_C@_1M@LHIPCIEK@?$AAi?$AAd?$AA?9?$AAI?$AAD?$AA?$AA@ 0000000180004900     libucrt:lcidtoname_downlevel.obj
 0001:00003910       ??_C@_1M@MFMOBGI@?$AAu?$AAk?$AA?9?$AAU?$AAA?$AA?$AA@ 0000000180004910     libucrt:lcidtoname_downlevel.obj
 0001:00003920       ??_C@_1M@OBGLJIPL@?$AAb?$AAe?$AA?9?$AAB?$AAY?$AA?$AA@ 0000000180004920     libucrt:lcidtoname_downlevel.obj
 0001:00003930       ??_C@_1M@BCFAJEAD@?$AAs?$AAl?$AA?9?$AAS?$AAI?$AA?$AA@ 0000000180004930     libucrt:lcidtoname_downlevel.obj
 0001:00003940       ??_C@_1M@FKFFEDDN@?$AAe?$AAt?$AA?9?$AAE?$AAE?$AA?$AA@ 0000000180004940     libucrt:lcidtoname_downlevel.obj
 0001:00003950       ??_C@_1M@KGKKAACI@?$AAl?$AAv?$AA?9?$AAL?$AAV?$AA?$AA@ 0000000180004950     libucrt:lcidtoname_downlevel.obj
 0001:00003960       ??_C@_1M@IFGBIJO@?$AAl?$AAt?$AA?9?$AAL?$AAT?$AA?$AA@ 0000000180004960     libucrt:lcidtoname_downlevel.obj
 0001:00003970       ??_C@_1M@FGEAHEDM@?$AAf?$AAa?$AA?9?$AAI?$AAR?$AA?$AA@ 0000000180004970     libucrt:lcidtoname_downlevel.obj
 0001:00003980       ??_C@_1M@KBMAIBFN@?$AAv?$AAi?$AA?9?$AAV?$AAN?$AA?$AA@ 0000000180004980     libucrt:lcidtoname_downlevel.obj
 0001:00003990       ??_C@_1M@GPCBKDJK@?$AAh?$AAy?$AA?9?$AAA?$AAM?$AA?$AA@ 0000000180004990     libucrt:lcidtoname_downlevel.obj
 0001:000039a0       ??_C@_1BG@BECMDDJB@?$AAa?$AAz?$AA?9?$AAA?$AAZ?$AA?9?$AAL?$AAa?$AAt?$AAn?$AA?$AA@ 00000001800049a0     libucrt:lcidtoname_downlevel.obj
 0001:000039b8       ??_C@_1M@MAOFCAEA@?$AAe?$AAu?$AA?9?$AAE?$AAS?$AA?$AA@ 00000001800049b8     libucrt:lcidtoname_downlevel.obj
 0001:000039c8       ??_C@_1M@IGHABKPI@?$AAm?$AAk?$AA?9?$AAM?$AAK?$AA?$AA@ 00000001800049c8     libucrt:lcidtoname_downlevel.obj
 0001:000039d8       ??_C@_1M@IAIGNEJG@?$AAt?$AAn?$AA?9?$AAZ?$AAA?$AA?$AA@ 00000001800049d8     libucrt:lcidtoname_downlevel.obj
 0001:000039e8       ??_C@_1M@IIJCOJFA@?$AAx?$AAh?$AA?9?$AAZ?$AAA?$AA?$AA@ 00000001800049e8     libucrt:lcidtoname_downlevel.obj
 0001:000039f8       ??_C@_1M@LGPJHNJH@?$AAz?$AAu?$AA?9?$AAZ?$AAA?$AA?$AA@ 00000001800049f8     libucrt:lcidtoname_downlevel.obj
 0001:00003a08       ??_C@_1M@HOKAOIO@?$AAa?$AAf?$AA?9?$AAZ?$AAA?$AA?$AA@ 0000000180004a08     libucrt:lcidtoname_downlevel.obj
 0001:00003a18       ??_C@_1M@DPCLHLIE@?$AAk?$AAa?$AA?9?$AAG?$AAE?$AA?$AA@ 0000000180004a18     libucrt:lcidtoname_downlevel.obj
 0001:00003a28       ??_C@_1M@BLKMHJBI@?$AAf?$AAo?$AA?9?$AAF?$AAO?$AA?$AA@ 0000000180004a28     libucrt:lcidtoname_downlevel.obj
 0001:00003a38       ??_C@_1M@LGGJAPPB@?$AAh?$AAi?$AA?9?$AAI?$AAN?$AA?$AA@ 0000000180004a38     libucrt:lcidtoname_downlevel.obj
 0001:00003a48       ??_C@_1M@FIKPIHFE@?$AAm?$AAt?$AA?9?$AAM?$AAT?$AA?$AA@ 0000000180004a48     libucrt:lcidtoname_downlevel.obj
 0001:00003a58       ??_C@_1M@HEGGPBFA@?$AAs?$AAe?$AA?9?$AAN?$AAO?$AA?$AA@ 0000000180004a58     libucrt:lcidtoname_downlevel.obj
 0001:00003a68       ??_C@_1M@EIBJEEPA@?$AAm?$AAs?$AA?9?$AAM?$AAY?$AA?$AA@ 0000000180004a68     libucrt:lcidtoname_downlevel.obj
 0001:00003a78       ??_C@_1M@FHLBGMPP@?$AAk?$AAk?$AA?9?$AAK?$AAZ?$AA?$AA@ 0000000180004a78     libucrt:lcidtoname_downlevel.obj
 0001:00003a88       ??_C@_1M@NGJJLCGI@?$AAk?$AAy?$AA?9?$AAK?$AAG?$AA?$AA@ 0000000180004a88     libucrt:lcidtoname_downlevel.obj
 0001:00003a98       ??_C@_1M@GIENNBFC@?$AAs?$AAw?$AA?9?$AAK?$AAE?$AA?$AA@ 0000000180004a98     libucrt:lcidtoname_downlevel.obj
 0001:00003aa8       ??_C@_1BG@NDGMJIMJ@?$AAu?$AAz?$AA?9?$AAU?$AAZ?$AA?9?$AAL?$AAa?$AAt?$AAn?$AA?$AA@ 0000000180004aa8     libucrt:lcidtoname_downlevel.obj
 0001:00003ac0       ??_C@_1M@IDCCIHBC@?$AAt?$AAt?$AA?9?$AAR?$AAU?$AA?$AA@ 0000000180004ac0     libucrt:lcidtoname_downlevel.obj
 0001:00003ad0       ??_C@_1M@LOICPMOJ@?$AAb?$AAn?$AA?9?$AAI?$AAN?$AA?$AA@ 0000000180004ad0     libucrt:lcidtoname_downlevel.obj
 0001:00003ae0       ??_C@_1M@KPKKNEAH@?$AAp?$AAa?$AA?9?$AAI?$AAN?$AA?$AA@ 0000000180004ae0     libucrt:lcidtoname_downlevel.obj
 0001:00003af0       ??_C@_1M@PJGPPBOG@?$AAg?$AAu?$AA?9?$AAI?$AAN?$AA?$AA@ 0000000180004af0     libucrt:lcidtoname_downlevel.obj
 0001:00003b00       ??_C@_1M@KMKMOPHI@?$AAt?$AAa?$AA?9?$AAI?$AAN?$AA?$AA@ 0000000180004b00     libucrt:lcidtoname_downlevel.obj
 0001:00003b10       ??_C@_1M@KFEHEPAC@?$AAt?$AAe?$AA?9?$AAI?$AAN?$AA?$AA@ 0000000180004b10     libucrt:lcidtoname_downlevel.obj
 0001:00003b20       ??_C@_1M@CDCLMGHI@?$AAk?$AAn?$AA?9?$AAI?$AAN?$AA?$AA@ 0000000180004b20     libucrt:lcidtoname_downlevel.obj
 0001:00003b30       ??_C@_1M@MIODLDKF@?$AAm?$AAl?$AA?9?$AAI?$AAN?$AA?$AA@ 0000000180004b30     libucrt:lcidtoname_downlevel.obj
 0001:00003b40       ??_C@_1M@PBIEACPO@?$AAm?$AAr?$AA?9?$AAI?$AAN?$AA?$AA@ 0000000180004b40     libucrt:lcidtoname_downlevel.obj
 0001:00003b50       ??_C@_1M@NIDEAGPH@?$AAs?$AAa?$AA?9?$AAI?$AAN?$AA?$AA@ 0000000180004b50     libucrt:lcidtoname_downlevel.obj
 0001:00003b60       ??_C@_1M@FHIHCBIO@?$AAm?$AAn?$AA?9?$AAM?$AAN?$AA?$AA@ 0000000180004b60     libucrt:lcidtoname_downlevel.obj
 0001:00003b70       ??_C@_1M@JAIJPENP@?$AAc?$AAy?$AA?9?$AAG?$AAB?$AA?$AA@ 0000000180004b70     libucrt:lcidtoname_downlevel.obj
 0001:00003b80       ??_C@_1M@PHGFBEPN@?$AAg?$AAl?$AA?9?$AAE?$AAS?$AA?$AA@ 0000000180004b80     libucrt:lcidtoname_downlevel.obj
 0001:00003b90       ??_C@_1O@KPIPDNCP@?$AAk?$AAo?$AAk?$AA?9?$AAI?$AAN?$AA?$AA@ 0000000180004b90     libucrt:lcidtoname_downlevel.obj
 0001:00003ba0       ??_C@_1O@KNHJLDJA@?$AAs?$AAy?$AAr?$AA?9?$AAS?$AAY?$AA?$AA@ 0000000180004ba0     libucrt:lcidtoname_downlevel.obj
 0001:00003bb0       ??_C@_1O@MKEKBLAH@?$AAd?$AAi?$AAv?$AA?9?$AAM?$AAV?$AA?$AA@ 0000000180004bb0     libucrt:lcidtoname_downlevel.obj
 0001:00003bc0       ??_C@_1O@OHDCKDDF@?$AAq?$AAu?$AAz?$AA?9?$AAB?$AAO?$AA?$AA@ 0000000180004bc0     libucrt:lcidtoname_downlevel.obj
 0001:00003bd0       ??_C@_1M@LEPJNLFD@?$AAn?$AAs?$AA?9?$AAZ?$AAA?$AA?$AA@ 0000000180004bd0     libucrt:lcidtoname_downlevel.obj
 0001:00003be0       ??_C@_1M@OMLEIIJB@?$AAm?$AAi?$AA?9?$AAN?$AAZ?$AA?$AA@ 0000000180004be0     libucrt:lcidtoname_downlevel.obj
 0001:00003bf0       ??_C@_1M@PMPEAILG@?$AAa?$AAr?$AA?9?$AAI?$AAQ?$AA?$AA@ 0000000180004bf0     libucrt:lcidtoname_downlevel.obj
 0001:00003c00       ??_C@_1M@CNKPNOEE@?$AAd?$AAe?$AA?9?$AAC?$AAH?$AA?$AA@ 0000000180004c00     libucrt:lcidtoname_downlevel.obj
 0001:00003c10       ??_C@_1M@LKMGMLKO@?$AAe?$AAn?$AA?9?$AAG?$AAB?$AA?$AA@ 0000000180004c10     libucrt:lcidtoname_downlevel.obj
 0001:00003c20       ??_C@_1M@PGKJFFGL@?$AAe?$AAs?$AA?9?$AAM?$AAX?$AA?$AA@ 0000000180004c20     libucrt:lcidtoname_downlevel.obj
 0001:00003c30       ??_C@_1M@DNNANBDC@?$AAf?$AAr?$AA?9?$AAB?$AAE?$AA?$AA@ 0000000180004c30     libucrt:lcidtoname_downlevel.obj
 0001:00003c40       ??_C@_1M@HLGMDFHM@?$AAi?$AAt?$AA?9?$AAC?$AAH?$AA?$AA@ 0000000180004c40     libucrt:lcidtoname_downlevel.obj
 0001:00003c50       ??_C@_1M@CLLBGJH@?$AAn?$AAl?$AA?9?$AAB?$AAE?$AA?$AA@ 0000000180004c50     libucrt:lcidtoname_downlevel.obj
 0001:00003c60       ??_C@_1M@BODBOGLF@?$AAn?$AAn?$AA?9?$AAN?$AAO?$AA?$AA@ 0000000180004c60     libucrt:lcidtoname_downlevel.obj
 0001:00003c70       ??_C@_1M@HFFAHKAD@?$AAp?$AAt?$AA?9?$AAP?$AAT?$AA?$AA@ 0000000180004c70     libucrt:lcidtoname_downlevel.obj
 0001:00003c80       ??_C@_1BG@LNOAKHIE@?$AAs?$AAr?$AA?9?$AAS?$AAP?$AA?9?$AAL?$AAa?$AAt?$AAn?$AA?$AA@ 0000000180004c80     libucrt:lcidtoname_downlevel.obj
 0001:00003c98       ??_C@_1M@HBMHBGAK@?$AAs?$AAv?$AA?9?$AAF?$AAI?$AA?$AA@ 0000000180004c98     libucrt:lcidtoname_downlevel.obj
 0001:00003ca8       ??_C@_1BG@DGCJGJBE@?$AAa?$AAz?$AA?9?$AAA?$AAZ?$AA?9?$AAC?$AAy?$AAr?$AAl?$AA?$AA@ 0000000180004ca8     libucrt:lcidtoname_downlevel.obj
 0001:00003cc0       ??_C@_1M@KEJDAAHB@?$AAs?$AAe?$AA?9?$AAS?$AAE?$AA?$AA@ 0000000180004cc0     libucrt:lcidtoname_downlevel.obj
 0001:00003cd0       ??_C@_1M@HEIBJJAD@?$AAm?$AAs?$AA?9?$AAB?$AAN?$AA?$AA@ 0000000180004cd0     libucrt:lcidtoname_downlevel.obj
 0001:00003ce0       ??_C@_1BG@PBGJMCEM@?$AAu?$AAz?$AA?9?$AAU?$AAZ?$AA?9?$AAC?$AAy?$AAr?$AAl?$AA?$AA@ 0000000180004ce0     libucrt:lcidtoname_downlevel.obj
 0001:00003cf8       ??_C@_1O@LAOBCMDF@?$AAq?$AAu?$AAz?$AA?9?$AAE?$AAC?$AA?$AA@ 0000000180004cf8     libucrt:lcidtoname_downlevel.obj
 0001:00003d08       ??_C@_1M@POEEMAIO@?$AAa?$AAr?$AA?9?$AAE?$AAG?$AA?$AA@ 0000000180004d08     libucrt:lcidtoname_downlevel.obj
 0001:00003d18       ??_C@_1M@EFAKDEDL@?$AAz?$AAh?$AA?9?$AAH?$AAK?$AA?$AA@ 0000000180004d18     libucrt:lcidtoname_downlevel.obj
 0001:00003d28       ??_C@_1M@HKKIJHGI@?$AAd?$AAe?$AA?9?$AAA?$AAT?$AA?$AA@ 0000000180004d28     libucrt:lcidtoname_downlevel.obj
 0001:00003d38       ??_C@_1M@KBFBEHJF@?$AAe?$AAn?$AA?9?$AAA?$AAU?$AA?$AA@ 0000000180004d38     libucrt:lcidtoname_downlevel.obj
 0001:00003d48       ??_C@_1M@MNPLFAAH@?$AAe?$AAs?$AA?9?$AAE?$AAS?$AA?$AA@ 0000000180004d48     libucrt:lcidtoname_downlevel.obj
 0001:00003d58       ??_C@_1M@HJOOJFMA@?$AAf?$AAr?$AA?9?$AAC?$AAA?$AA?$AA@ 0000000180004d58     libucrt:lcidtoname_downlevel.obj
 0001:00003d68       ??_C@_1BG@JPOFPNAB@?$AAs?$AAr?$AA?9?$AAS?$AAP?$AA?9?$AAC?$AAy?$AAr?$AAl?$AA?$AA@ 0000000180004d68     libucrt:lcidtoname_downlevel.obj
 0001:00003d80       ??_C@_1M@LNFOCMOB@?$AAs?$AAe?$AA?9?$AAF?$AAI?$AA?$AA@ 0000000180004d80     libucrt:lcidtoname_downlevel.obj
 0001:00003d90       ??_C@_1O@MGJBOAMB@?$AAq?$AAu?$AAz?$AA?9?$AAP?$AAE?$AA?$AA@ 0000000180004d90     libucrt:lcidtoname_downlevel.obj
 0001:00003da0       ??_C@_1M@GJINLBOK@?$AAa?$AAr?$AA?9?$AAL?$AAY?$AA?$AA@ 0000000180004da0     libucrt:lcidtoname_downlevel.obj
 0001:00003db0       ??_C@_1M@GGMNHJNL@?$AAz?$AAh?$AA?9?$AAS?$AAG?$AA?$AA@ 0000000180004db0     libucrt:lcidtoname_downlevel.obj
 0001:00003dc0       ??_C@_1M@HOIKODND@?$AAd?$AAe?$AA?9?$AAL?$AAU?$AA?$AA@ 0000000180004dc0     libucrt:lcidtoname_downlevel.obj
 0001:00003dd0       ??_C@_1M@DDOCCGFG@?$AAe?$AAn?$AA?9?$AAC?$AAA?$AA?$AA@ 0000000180004dd0     libucrt:lcidtoname_downlevel.obj
 0001:00003de0       ??_C@_1M@BNOEMJLF@?$AAe?$AAs?$AA?9?$AAG?$AAT?$AA?$AA@ 0000000180004de0     libucrt:lcidtoname_downlevel.obj
 0001:00003df0       ??_C@_1M@EOGNKEK@?$AAf?$AAr?$AA?9?$AAC?$AAH?$AA?$AA@ 0000000180004df0     libucrt:lcidtoname_downlevel.obj
 0001:00003e00       ??_C@_1M@FLIDJFHL@?$AAh?$AAr?$AA?9?$AAB?$AAA?$AA?$AA@ 0000000180004e00     libucrt:lcidtoname_downlevel.obj
 0001:00003e10       ??_C@_1O@FMCELNAJ@?$AAs?$AAm?$AAj?$AA?9?$AAN?$AAO?$AA?$AA@ 0000000180004e10     libucrt:lcidtoname_downlevel.obj
 0001:00003e20       ??_C@_1M@JHGLJMGJ@?$AAa?$AAr?$AA?9?$AAD?$AAZ?$AA?$AA@ 0000000180004e20     libucrt:lcidtoname_downlevel.obj
 0001:00003e30       ??_C@_1M@JKKFDCNP@?$AAz?$AAh?$AA?9?$AAM?$AAO?$AA?$AA@ 0000000180004e30     libucrt:lcidtoname_downlevel.obj
 0001:00003e40       ??_C@_1M@GEEFALPE@?$AAd?$AAe?$AA?9?$AAL?$AAI?$AA?$AA@ 0000000180004e40     libucrt:lcidtoname_downlevel.obj
 0001:00003e50       ??_C@_1M@IGEOFBG@?$AAe?$AAn?$AA?9?$AAN?$AAZ?$AA?$AA@ 0000000180004e50     libucrt:lcidtoname_downlevel.obj
 0001:00003e60       ??_C@_1M@KDBONEHP@?$AAe?$AAs?$AA?9?$AAC?$AAR?$AA?$AA@ 0000000180004e60     libucrt:lcidtoname_downlevel.obj
 0001:00003e70       ??_C@_1M@FHMDOHNN@?$AAf?$AAr?$AA?9?$AAL?$AAU?$AA?$AA@ 0000000180004e70     libucrt:lcidtoname_downlevel.obj
 0001:00003e80       ??_C@_1BG@NFKKMAFG@?$AAb?$AAs?$AA?9?$AAB?$AAA?$AA?9?$AAL?$AAa?$AAt?$AAn?$AA?$AA@ 0000000180004e80     libucrt:lcidtoname_downlevel.obj
 0001:00003e98       ??_C@_1O@IMNBEMCI@?$AAs?$AAm?$AAj?$AA?9?$AAS?$AAE?$AA?$AA@ 0000000180004e98     libucrt:lcidtoname_downlevel.obj
 0001:00003ea8       ??_C@_1M@DHHMBNDP@?$AAa?$AAr?$AA?9?$AAM?$AAA?$AA?$AA@ 0000000180004ea8     libucrt:lcidtoname_downlevel.obj
 0001:00003eb8       ??_C@_1M@BNBLJCGH@?$AAe?$AAn?$AA?9?$AAI?$AAE?$AA?$AA@ 0000000180004eb8     libucrt:lcidtoname_downlevel.obj
 0001:00003ec8       ??_C@_1M@GEPAFMDL@?$AAe?$AAs?$AA?9?$AAP?$AAA?$AA?$AA@ 0000000180004ec8     libucrt:lcidtoname_downlevel.obj
 0001:00003ed8       ??_C@_1M@OJONDMDL@?$AAf?$AAr?$AA?9?$AAM?$AAC?$AA?$AA@ 0000000180004ed8     libucrt:lcidtoname_downlevel.obj
 0001:00003ee8       ??_C@_1BG@OBCNFJB@?$AAs?$AAr?$AA?9?$AAB?$AAA?$AA?9?$AAL?$AAa?$AAt?$AAn?$AA?$AA@ 0000000180004ee8     libucrt:lcidtoname_downlevel.obj
 0001:00003f00       ??_C@_1O@KEMEEGPO@?$AAs?$AAm?$AAa?$AA?9?$AAN?$AAO?$AA?$AA@ 0000000180004f00     libucrt:lcidtoname_downlevel.obj
 0001:00003f10       ??_C@_1M@ELMGFODK@?$AAa?$AAr?$AA?9?$AAT?$AAN?$AA?$AA@ 0000000180004f10     libucrt:lcidtoname_downlevel.obj
 0001:00003f20       ??_C@_1M@BHDLHFAF@?$AAe?$AAn?$AA?9?$AAZ?$AAA?$AA?$AA@ 0000000180004f20     libucrt:lcidtoname_downlevel.obj
 0001:00003f30       ??_C@_1M@BMGIGLIF@?$AAe?$AAs?$AA?9?$AAD?$AAO?$AA?$AA@ 0000000180004f30     libucrt:lcidtoname_downlevel.obj
 0001:00003f40       ??_C@_1BG@CMBHIPBE@?$AAs?$AAr?$AA?9?$AAB?$AAA?$AA?9?$AAC?$AAy?$AAr?$AAl?$AA?$AA@ 0000000180004f40     libucrt:lcidtoname_downlevel.obj
 0001:00003f58       ??_C@_1O@HEDBLHNP@?$AAs?$AAm?$AAa?$AA?9?$AAS?$AAE?$AA?$AA@ 0000000180004f58     libucrt:lcidtoname_downlevel.obj
 0001:00003f68       ??_C@_1M@DAGCADIM@?$AAa?$AAr?$AA?9?$AAO?$AAM?$AA?$AA@ 0000000180004f68     libucrt:lcidtoname_downlevel.obj
 0001:00003f78       ??_C@_1M@FODLMICG@?$AAe?$AAn?$AA?9?$AAJ?$AAM?$AA?$AA@ 0000000180004f78     libucrt:lcidtoname_downlevel.obj
 0001:00003f88       ??_C@_1M@DNMLCIHB@?$AAe?$AAs?$AA?9?$AAV?$AAE?$AA?$AA@ 0000000180004f88     libucrt:lcidtoname_downlevel.obj
 0001:00003f98       ??_C@_1O@EOKHMKJK@?$AAs?$AAm?$AAs?$AA?9?$AAF?$AAI?$AA?$AA@ 0000000180004f98     libucrt:lcidtoname_downlevel.obj
 0001:00003fa8       ??_C@_1M@CAFJMKOF@?$AAa?$AAr?$AA?9?$AAY?$AAE?$AA?$AA@ 0000000180004fa8     libucrt:lcidtoname_downlevel.obj
 0001:00003fb8       ??_C@_1M@CBFHIJLI@?$AAe?$AAn?$AA?9?$AAC?$AAB?$AA?$AA@ 0000000180004fb8     libucrt:lcidtoname_downlevel.obj
 0001:00003fc8       ??_C@_1M@BGNFLDN@?$AAe?$AAs?$AA?9?$AAC?$AAO?$AA?$AA@ 0000000180004fc8     libucrt:lcidtoname_downlevel.obj
 0001:00003fd8       ??_C@_1O@JMPHMAMC@?$AAs?$AAm?$AAn?$AA?9?$AAF?$AAI?$AA?$AA@ 0000000180004fd8     libucrt:lcidtoname_downlevel.obj
 0001:00003fe8       ??_C@_1M@JLANABKE@?$AAa?$AAr?$AA?9?$AAS?$AAY?$AA?$AA@ 0000000180004fe8     libucrt:lcidtoname_downlevel.obj
 0001:00003ff8       ??_C@_1M@HPKGCFGN@?$AAe?$AAn?$AA?9?$AAB?$AAZ?$AA?$AA@ 0000000180004ff8     libucrt:lcidtoname_downlevel.obj
 0001:00004008       ??_C@_1M@OLJCMLGM@?$AAe?$AAs?$AA?9?$AAP?$AAE?$AA?$AA@ 0000000180005008     libucrt:lcidtoname_downlevel.obj
 0001:00004018       ??_C@_1M@MKKGFKLE@?$AAa?$AAr?$AA?9?$AAJ?$AAO?$AA?$AA@ 0000000180005018     libucrt:lcidtoname_downlevel.obj
 0001:00004028       ??_C@_1M@EKPGLDNI@?$AAe?$AAn?$AA?9?$AAT?$AAT?$AA?$AA@ 0000000180005028     libucrt:lcidtoname_downlevel.obj
 0001:00004038       ??_C@_1M@OONGHFHE@?$AAe?$AAs?$AA?9?$AAA?$AAR?$AA?$AA@ 0000000180005038     libucrt:lcidtoname_downlevel.obj
 0001:00004048       ??_C@_1M@OOJFGBHE@?$AAa?$AAr?$AA?9?$AAL?$AAB?$AA?$AA@ 0000000180005048     libucrt:lcidtoname_downlevel.obj
 0001:00004058       ??_C@_1M@GCEJHNEG@?$AAe?$AAn?$AA?9?$AAZ?$AAW?$AA?$AA@ 0000000180005058     libucrt:lcidtoname_downlevel.obj
 0001:00004068       ??_C@_1M@JNOCAHJI@?$AAe?$AAs?$AA?9?$AAE?$AAC?$AA?$AA@ 0000000180005068     libucrt:lcidtoname_downlevel.obj
 0001:00004078       ??_C@_1M@JEFHPGGB@?$AAa?$AAr?$AA?9?$AAK?$AAW?$AA?$AA@ 0000000180005078     libucrt:lcidtoname_downlevel.obj
 0001:00004088       ??_C@_1M@MLKIBJOJ@?$AAe?$AAn?$AA?9?$AAP?$AAH?$AA?$AA@ 0000000180005088     libucrt:lcidtoname_downlevel.obj
 0001:00004098       ??_C@_1M@BDNIPEND@?$AAe?$AAs?$AA?9?$AAC?$AAL?$AA?$AA@ 0000000180005098     libucrt:lcidtoname_downlevel.obj
 0001:000040a8       ??_C@_1M@MPNMEKBD@?$AAa?$AAr?$AA?9?$AAA?$AAE?$AA?$AA@ 00000001800050a8     libucrt:lcidtoname_downlevel.obj
 0001:000040b8       ??_C@_1M@KBJALCPI@?$AAe?$AAs?$AA?9?$AAU?$AAY?$AA?$AA@ 00000001800050b8     libucrt:lcidtoname_downlevel.obj
 0001:000040c8       ??_C@_1M@LLCCOAGA@?$AAa?$AAr?$AA?9?$AAB?$AAH?$AA?$AA@ 00000001800050c8     libucrt:lcidtoname_downlevel.obj
 0001:000040d8       ??_C@_1M@PBFNCDEL@?$AAe?$AAs?$AA?9?$AAP?$AAY?$AA?$AA@ 00000001800050d8     libucrt:lcidtoname_downlevel.obj
 0001:000040e8       ??_C@_1M@EDGINPNP@?$AAa?$AAr?$AA?9?$AAQ?$AAA?$AA?$AA@ 00000001800050e8     libucrt:lcidtoname_downlevel.obj
 0001:000040f8       ??_C@_1M@MKDBIIJI@?$AAe?$AAs?$AA?9?$AAB?$AAO?$AA?$AA@ 00000001800050f8     libucrt:lcidtoname_downlevel.obj
 0001:00004108       ??_C@_1M@CPKKEBLD@?$AAe?$AAs?$AA?9?$AAS?$AAV?$AA?$AA@ 0000000180005108     libucrt:lcidtoname_downlevel.obj
 0001:00004118       ??_C@_1M@NDBGMMJL@?$AAe?$AAs?$AA?9?$AAH?$AAN?$AA?$AA@ 0000000180005118     libucrt:lcidtoname_downlevel.obj
 0001:00004128       ??_C@_1M@JIJIBHDP@?$AAe?$AAs?$AA?9?$AAN?$AAI?$AA?$AA@ 0000000180005128     libucrt:lcidtoname_downlevel.obj
 0001:00004138       ??_C@_1M@CGFMKEEK@?$AAe?$AAs?$AA?9?$AAP?$AAR?$AA?$AA@ 0000000180005138     libucrt:lcidtoname_downlevel.obj
 0001:00004148       ??_C@_1O@ICJHKIIK@?$AAz?$AAh?$AA?9?$AAC?$AAH?$AAT?$AA?$AA@ 0000000180005148     libucrt:lcidtoname_downlevel.obj
 0001:00004158       ??_C@_15CLNEJCE@?$AAs?$AAr?$AA?$AA@ 0000000180005158     libucrt:lcidtoname_downlevel.obj
 0001:00004fa0       ??_C@_1M@KAHEKEIG@?$AAa?$AAf?$AA?9?$AAz?$AAa?$AA?$AA@ 0000000180005fa0     libucrt:lcidtoname_downlevel.obj
 0001:00004fb0       ??_C@_1M@GIECOABL@?$AAa?$AAr?$AA?9?$AAa?$AAe?$AA?$AA@ 0000000180005fb0     libucrt:lcidtoname_downlevel.obj
 0001:00004fc0       ??_C@_1M@BMLMEKGI@?$AAa?$AAr?$AA?9?$AAb?$AAh?$AA?$AA@ 0000000180005fc0     libucrt:lcidtoname_downlevel.obj
 0001:00004fd0       ??_C@_1M@DAPFDGGB@?$AAa?$AAr?$AA?9?$AAd?$AAz?$AA?$AA@ 0000000180005fd0     libucrt:lcidtoname_downlevel.obj
 0001:00004fe0       ??_C@_1M@FJNKGKIG@?$AAa?$AAr?$AA?9?$AAe?$AAg?$AA?$AA@ 0000000180005fe0     libucrt:lcidtoname_downlevel.obj
 0001:00004ff0       ??_C@_1M@FLGKKCLO@?$AAa?$AAr?$AA?9?$AAi?$AAq?$AA?$AA@ 0000000180005ff0     libucrt:lcidtoname_downlevel.obj
 0001:00005000       ??_C@_1M@GNDIPALM@?$AAa?$AAr?$AA?9?$AAj?$AAo?$AA?$AA@ 0000000180006000     libucrt:lcidtoname_downlevel.obj
 0001:00005010       ??_C@_1M@DDMJFMGJ@?$AAa?$AAr?$AA?9?$AAk?$AAw?$AA?$AA@ 0000000180006010     libucrt:lcidtoname_downlevel.obj
 0001:00005020       ??_C@_1M@EJALMLHM@?$AAa?$AAr?$AA?9?$AAl?$AAb?$AA?$AA@ 0000000180006020     libucrt:lcidtoname_downlevel.obj
 0001:00005030       ??_C@_1M@MOBDBLOC@?$AAa?$AAr?$AA?9?$AAl?$AAy?$AA?$AA@ 0000000180006030     libucrt:lcidtoname_downlevel.obj
 0001:00005040       ??_C@_1M@JAOCLHDH@?$AAa?$AAr?$AA?9?$AAm?$AAa?$AA?$AA@ 0000000180006040     libucrt:lcidtoname_downlevel.obj
 0001:00005050       ??_C@_1M@JHPMKJIE@?$AAa?$AAr?$AA?9?$AAo?$AAm?$AA?$AA@ 0000000180006050     libucrt:lcidtoname_downlevel.obj
 0001:00005060       ??_C@_1M@OEPGHFNH@?$AAa?$AAr?$AA?9?$AAq?$AAa?$AA?$AA@ 0000000180006060     libucrt:lcidtoname_downlevel.obj
 0001:00005070       ??_C@_1M@KJDONENM@?$AAa?$AAr?$AA?9?$AAs?$AAa?$AA?$AA@ 0000000180006070     libucrt:lcidtoname_downlevel.obj
 0001:00005080       ??_C@_1M@DMJDKLKM@?$AAa?$AAr?$AA?9?$AAs?$AAy?$AA?$AA@ 0000000180006080     libucrt:lcidtoname_downlevel.obj
 0001:00005090       ??_C@_1M@OMFIPEDC@?$AAa?$AAr?$AA?9?$AAt?$AAn?$AA?$AA@ 0000000180006090     libucrt:lcidtoname_downlevel.obj
 0001:000050a0       ??_C@_1M@IHMHGAON@?$AAa?$AAr?$AA?9?$AAy?$AAe?$AA?$AA@ 00000001800060a0     libucrt:lcidtoname_downlevel.obj
 0001:000050b0       ??_C@_1BG@KDCPGJGB@?$AAa?$AAz?$AA?9?$AAa?$AAz?$AA?9?$AAc?$AAy?$AAr?$AAl?$AA?$AA@ 00000001800060b0     libucrt:lcidtoname_downlevel.obj
 0001:000050c8       ??_C@_1BG@IBCKDDOE@?$AAa?$AAz?$AA?9?$AAa?$AAz?$AA?9?$AAl?$AAa?$AAt?$AAn?$AA?$AA@ 00000001800060c8     libucrt:lcidtoname_downlevel.obj
 0001:000050e0       ??_C@_1M@EGPFDCPD@?$AAb?$AAe?$AA?9?$AAb?$AAy?$AA?$AA@ 00000001800060e0     libucrt:lcidtoname_downlevel.obj
 0001:000050f0       ??_C@_1M@PCMGMCGC@?$AAb?$AAg?$AA?9?$AAb?$AAg?$AA?$AA@ 00000001800060f0     libucrt:lcidtoname_downlevel.obj
 0001:00005100       ??_C@_1M@BJBMFGOB@?$AAb?$AAn?$AA?9?$AAi?$AAn?$AA?$AA@ 0000000180006100     libucrt:lcidtoname_downlevel.obj
 0001:00005110       ??_C@_1BG@EAKMMACD@?$AAb?$AAs?$AA?9?$AAb?$AAa?$AA?9?$AAl?$AAa?$AAt?$AAn?$AA?$AA@ 0000000180006110     libucrt:lcidtoname_downlevel.obj
 0001:00005128       ??_C@_1M@KGADAODK@?$AAc?$AAa?$AA?9?$AAe?$AAs?$AA?$AA@ 0000000180006128     libucrt:lcidtoname_downlevel.obj
 0001:00005138       ??_C@_1M@COAJPDHI@?$AAc?$AAs?$AA?9?$AAc?$AAz?$AA?$AA@ 0000000180006138     libucrt:lcidtoname_downlevel.obj
 0001:00005148       ??_C@_1M@DHBHFONH@?$AAc?$AAy?$AA?9?$AAg?$AAb?$AA?$AA@ 0000000180006148     libucrt:lcidtoname_downlevel.obj
 0001:00005158       ??_C@_1M@IMGKELGA@?$AAd?$AAa?$AA?9?$AAd?$AAk?$AA?$AA@ 0000000180006158     libucrt:lcidtoname_downlevel.obj
 0001:00005168       ??_C@_1M@NNDGDNGA@?$AAd?$AAe?$AA?9?$AAa?$AAt?$AA?$AA@ 0000000180006168     libucrt:lcidtoname_downlevel.obj
 0001:00005178       ??_C@_1M@IKDBHEEM@?$AAd?$AAe?$AA?9?$AAc?$AAh?$AA?$AA@ 0000000180006178     libucrt:lcidtoname_downlevel.obj
 0001:00005188       ??_C@_1M@GFFOJMCJ@?$AAd?$AAe?$AA?9?$AAd?$AAe?$AA?$AA@ 0000000180006188     libucrt:lcidtoname_downlevel.obj
 0001:00005198       ??_C@_1M@MDNLKBPM@?$AAd?$AAe?$AA?9?$AAl?$AAi?$AA?$AA@ 0000000180006198     libucrt:lcidtoname_downlevel.obj
 0001:000051a8       ??_C@_1M@NJBEEJNL@?$AAd?$AAe?$AA?9?$AAl?$AAu?$AA?$AA@ 00000001800061a8     libucrt:lcidtoname_downlevel.obj
 0001:000051b8       ??_C@_1O@GNNELBAP@?$AAd?$AAi?$AAv?$AA?9?$AAm?$AAv?$AA?$AA@ 00000001800061b8     libucrt:lcidtoname_downlevel.obj
 0001:000051c8       ??_C@_1M@EJLEOGAE@?$AAe?$AAl?$AA?9?$AAg?$AAr?$AA?$AA@ 00000001800061c8     libucrt:lcidtoname_downlevel.obj
 0001:000051d8       ??_C@_1M@GMPONJN@?$AAe?$AAn?$AA?9?$AAa?$AAu?$AA?$AA@ 00000001800061d8     libucrt:lcidtoname_downlevel.obj
 0001:000051e8       ??_C@_1M@NIDIIPGF@?$AAe?$AAn?$AA?9?$AAb?$AAz?$AA?$AA@ 00000001800061e8     libucrt:lcidtoname_downlevel.obj
 0001:000051f8       ??_C@_1M@JEHMIMFO@?$AAe?$AAn?$AA?9?$AAc?$AAa?$AA?$AA@ 00000001800061f8     libucrt:lcidtoname_downlevel.obj
 0001:00005208       ??_C@_1M@IGMJCDLA@?$AAe?$AAn?$AA?9?$AAc?$AAb?$AA?$AA@ 0000000180006208     libucrt:lcidtoname_downlevel.obj
 0001:00005218       ??_C@_1M@BNFIGBKG@?$AAe?$AAn?$AA?9?$AAg?$AAb?$AA?$AA@ 0000000180006218     libucrt:lcidtoname_downlevel.obj
 0001:00005228       ??_C@_1M@LKIFDIGP@?$AAe?$AAn?$AA?9?$AAi?$AAe?$AA?$AA@ 0000000180006228     libucrt:lcidtoname_downlevel.obj
 0001:00005238       ??_C@_1M@PJKFGCCO@?$AAe?$AAn?$AA?9?$AAj?$AAm?$AA?$AA@ 0000000180006238     libucrt:lcidtoname_downlevel.obj
 0001:00005248       ??_C@_1M@KPPKEPBO@?$AAe?$AAn?$AA?9?$AAn?$AAz?$AA?$AA@ 0000000180006248     libucrt:lcidtoname_downlevel.obj
 0001:00005258       ??_C@_1M@GMDGLDOB@?$AAe?$AAn?$AA?9?$AAp?$AAh?$AA?$AA@ 0000000180006258     libucrt:lcidtoname_downlevel.obj
 0001:00005268       ??_C@_1M@ONGIBJNA@?$AAe?$AAn?$AA?9?$AAt?$AAt?$AA?$AA@ 0000000180006268     libucrt:lcidtoname_downlevel.obj
 0001:00005278       ??_C@_1M@LLODPCMM@?$AAe?$AAn?$AA?9?$AAu?$AAs?$AA?$AA@ 0000000180006278     libucrt:lcidtoname_downlevel.obj
 0001:00005288       ??_C@_1M@LAKFNPAN@?$AAe?$AAn?$AA?9?$AAz?$AAa?$AA?$AA@ 0000000180006288     libucrt:lcidtoname_downlevel.obj
 0001:00005298       ??_C@_1M@MFNHNHEO@?$AAe?$AAn?$AA?9?$AAz?$AAw?$AA?$AA@ 0000000180006298     libucrt:lcidtoname_downlevel.obj
 0001:000052a8       ??_C@_1M@EJEINPHM@?$AAe?$AAs?$AA?9?$AAa?$AAr?$AA?$AA@ 00000001800062a8     libucrt:lcidtoname_downlevel.obj
 0001:000052b8       ??_C@_1M@GNKPCCJA@?$AAe?$AAs?$AA?9?$AAb?$AAo?$AA?$AA@ 00000001800062b8     libucrt:lcidtoname_downlevel.obj
 0001:000052c8       ??_C@_1M@LEEGFONL@?$AAe?$AAs?$AA?9?$AAc?$AAl?$AA?$AA@ 00000001800062c8     libucrt:lcidtoname_downlevel.obj
 0001:000052d8       ??_C@_1M@KGPDPBDF@?$AAe?$AAs?$AA?9?$AAc?$AAo?$AA?$AA@ 00000001800062d8     libucrt:lcidtoname_downlevel.obj
 0001:000052e8       ??_C@_1M@EIAHOHH@?$AAe?$AAs?$AA?9?$AAc?$AAr?$AA?$AA@ 00000001800062e8     libucrt:lcidtoname_downlevel.obj
 0001:000052f8       ??_C@_1M@LLPGMBIN@?$AAe?$AAs?$AA?9?$AAd?$AAo?$AA?$AA@ 00000001800062f8     libucrt:lcidtoname_downlevel.obj
 0001:00005308       ??_C@_1M@DKHMKNJA@?$AAe?$AAs?$AA?9?$AAe?$AAc?$AA?$AA@ 0000000180006308     libucrt:lcidtoname_downlevel.obj
 0001:00005318       ??_C@_1M@GKGFPKAP@?$AAe?$AAs?$AA?9?$AAe?$AAs?$AA?$AA@ 0000000180006318     libucrt:lcidtoname_downlevel.obj
 0001:00005328       ??_C@_1M@LKHKGDLN@?$AAe?$AAs?$AA?9?$AAg?$AAt?$AA?$AA@ 0000000180006328     libucrt:lcidtoname_downlevel.obj
 0001:00005338       ??_C@_1M@HEIIGGJD@?$AAe?$AAs?$AA?9?$AAh?$AAn?$AA?$AA@ 0000000180006338     libucrt:lcidtoname_downlevel.obj
 0001:00005348       ??_C@_1M@FBDHPPGD@?$AAe?$AAs?$AA?9?$AAm?$AAx?$AA?$AA@ 0000000180006348     libucrt:lcidtoname_downlevel.obj
 0001:00005358       ??_C@_1M@DPAGLNDH@?$AAe?$AAs?$AA?9?$AAn?$AAi?$AA?$AA@ 0000000180006358     libucrt:lcidtoname_downlevel.obj
 0001:00005368       ??_C@_1M@MDGOPGDD@?$AAe?$AAs?$AA?9?$AAp?$AAa?$AA?$AA@ 0000000180006368     libucrt:lcidtoname_downlevel.obj
 0001:00005378       ??_C@_1M@EMAMGBGE@?$AAe?$AAs?$AA?9?$AAp?$AAe?$AA?$AA@ 0000000180006378     libucrt:lcidtoname_downlevel.obj
 0001:00005388       ??_C@_1M@IBMCAOEC@?$AAe?$AAs?$AA?9?$AAp?$AAr?$AA?$AA@ 0000000180006388     libucrt:lcidtoname_downlevel.obj
 0001:00005398       ??_C@_1M@FGMDIJED@?$AAe?$AAs?$AA?9?$AAp?$AAy?$AA?$AA@ 0000000180006398     libucrt:lcidtoname_downlevel.obj
 0001:000053a8       ??_C@_1M@IIDEOLLL@?$AAe?$AAs?$AA?9?$AAs?$AAv?$AA?$AA@ 00000001800063a8     libucrt:lcidtoname_downlevel.obj
 0001:000053b8       ??_C@_1M@GAOBIPA@?$AAe?$AAs?$AA?9?$AAu?$AAy?$AA?$AA@ 00000001800063b8     libucrt:lcidtoname_downlevel.obj
 0001:000053c8       ??_C@_1M@JKFFICHJ@?$AAe?$AAs?$AA?9?$AAv?$AAe?$AA?$AA@ 00000001800063c8     libucrt:lcidtoname_downlevel.obj
 0001:000053d8       ??_C@_1M@PNMLOJDF@?$AAe?$AAt?$AA?9?$AAe?$AAe?$AA?$AA@ 00000001800063d8     libucrt:lcidtoname_downlevel.obj
 0001:000053e8       ??_C@_1M@GHHLIKEI@?$AAe?$AAu?$AA?9?$AAe?$AAs?$AA?$AA@ 00000001800063e8     libucrt:lcidtoname_downlevel.obj
 0001:000053f8       ??_C@_1M@PBNONODE@?$AAf?$AAa?$AA?9?$AAi?$AAr?$AA?$AA@ 00000001800063f8     libucrt:lcidtoname_downlevel.obj
 0001:00005408       ??_C@_1M@JEEHPMIL@?$AAf?$AAi?$AA?9?$AAf?$AAi?$AA?$AA@ 0000000180006408     libucrt:lcidtoname_downlevel.obj
 0001:00005418       ??_C@_1M@LMDCNDBA@?$AAf?$AAo?$AA?9?$AAf?$AAo?$AA?$AA@ 0000000180006418     libucrt:lcidtoname_downlevel.obj
 0001:00005428       ??_C@_1M@JKEOHLDK@?$AAf?$AAr?$AA?9?$AAb?$AAe?$AA?$AA@ 0000000180006428     libucrt:lcidtoname_downlevel.obj
 0001:00005438       ??_C@_1M@NOHADPMI@?$AAf?$AAr?$AA?9?$AAc?$AAa?$AA?$AA@ 0000000180006438     libucrt:lcidtoname_downlevel.obj
 0001:00005448       ??_C@_1M@KDHIHAEC@?$AAf?$AAr?$AA?9?$AAc?$AAh?$AA?$AA@ 0000000180006448     libucrt:lcidtoname_downlevel.obj
 0001:00005458       ??_C@_1M@MMBBFGAK@?$AAf?$AAr?$AA?9?$AAf?$AAr?$AA?$AA@ 0000000180006458     libucrt:lcidtoname_downlevel.obj
 0001:00005468       ??_C@_1M@PAFNENNF@?$AAf?$AAr?$AA?9?$AAl?$AAu?$AA?$AA@ 0000000180006468     libucrt:lcidtoname_downlevel.obj
 0001:00005478       ??_C@_1M@EOHDJGDD@?$AAf?$AAr?$AA?9?$AAm?$AAc?$AA?$AA@ 0000000180006478     libucrt:lcidtoname_downlevel.obj
 0001:00005488       ??_C@_1M@FAPLLOPF@?$AAg?$AAl?$AA?9?$AAe?$AAs?$AA?$AA@ 0000000180006488     libucrt:lcidtoname_downlevel.obj
 0001:00005498       ??_C@_1M@FOPBFLOO@?$AAg?$AAu?$AA?9?$AAi?$AAn?$AA?$AA@ 0000000180006498     libucrt:lcidtoname_downlevel.obj
 0001:000054a8       ??_C@_1M@KBMCINPM@?$AAh?$AAe?$AA?9?$AAi?$AAl?$AA?$AA@ 00000001800064a8     libucrt:lcidtoname_downlevel.obj
 0001:000054b8       ??_C@_1M@BBPHKFPJ@?$AAh?$AAi?$AA?9?$AAi?$AAn?$AA?$AA@ 00000001800064b8     libucrt:lcidtoname_downlevel.obj
 0001:000054c8       ??_C@_1M@PMBNDPHD@?$AAh?$AAr?$AA?9?$AAb?$AAa?$AA?$AA@ 00000001800064c8     libucrt:lcidtoname_downlevel.obj
 0001:000054d8       ??_C@_1M@BPCKOEGE@?$AAh?$AAr?$AA?9?$AAh?$AAr?$AA?$AA@ 00000001800064d8     libucrt:lcidtoname_downlevel.obj
 0001:000054e8       ??_C@_1M@GACBMHKE@?$AAh?$AAu?$AA?9?$AAh?$AAu?$AA?$AA@ 00000001800064e8     libucrt:lcidtoname_downlevel.obj
 0001:000054f8       ??_C@_1M@MILPAJJC@?$AAh?$AAy?$AA?9?$AAa?$AAm?$AA?$AA@ 00000001800064f8     libucrt:lcidtoname_downlevel.obj
 0001:00005508       ??_C@_1M@BABBICEC@?$AAi?$AAd?$AA?9?$AAi?$AAd?$AA?$AA@ 0000000180006508     libucrt:lcidtoname_downlevel.obj
 0001:00005518       ??_C@_1M@BIKNHHPF@?$AAi?$AAs?$AA?9?$AAi?$AAs?$AA?$AA@ 0000000180006518     libucrt:lcidtoname_downlevel.obj
 0001:00005528       ??_C@_1M@NMPCJPHE@?$AAi?$AAt?$AA?9?$AAc?$AAh?$AA?$AA@ 0000000180006528     libucrt:lcidtoname_downlevel.obj
 0001:00005538       ??_C@_1M@GHKGFEDF@?$AAi?$AAt?$AA?9?$AAi?$AAt?$AA?$AA@ 0000000180006538     libucrt:lcidtoname_downlevel.obj
 0001:00005548       ??_C@_1M@NIEJCJJA@?$AAj?$AAa?$AA?9?$AAj?$AAp?$AA?$AA@ 0000000180006548     libucrt:lcidtoname_downlevel.obj
 0001:00005558       ??_C@_1M@JILFNBIM@?$AAk?$AAa?$AA?9?$AAg?$AAe?$AA?$AA@ 0000000180006558     libucrt:lcidtoname_downlevel.obj
 0001:00005568       ??_C@_1M@PACPMGPH@?$AAk?$AAk?$AA?9?$AAk?$AAz?$AA?$AA@ 0000000180006568     libucrt:lcidtoname_downlevel.obj
 0001:00005578       ??_C@_1M@IELFGMHA@?$AAk?$AAn?$AA?9?$AAi?$AAn?$AA?$AA@ 0000000180006578     libucrt:lcidtoname_downlevel.obj
 0001:00005588       ??_C@_1O@IBBJHCH@?$AAk?$AAo?$AAk?$AA?9?$AAi?$AAn?$AA?$AA@ 0000000180006588     libucrt:lcidtoname_downlevel.obj
 0001:00005598       ??_C@_1M@DMHAEOGC@?$AAk?$AAo?$AA?9?$AAk?$AAr?$AA?$AA@ 0000000180006598     libucrt:lcidtoname_downlevel.obj
 0001:000055a8       ??_C@_1M@HBAHBIGA@?$AAk?$AAy?$AA?9?$AAk?$AAg?$AA?$AA@ 00000001800065a8     libucrt:lcidtoname_downlevel.obj
 0001:000055b8       ??_C@_1M@KPMILCJG@?$AAl?$AAt?$AA?9?$AAl?$AAt?$AA?$AA@ 00000001800065b8     libucrt:lcidtoname_downlevel.obj
 0001:000055c8       ??_C@_1M@BDEKKCA@?$AAl?$AAv?$AA?9?$AAl?$AAv?$AA?$AA@ 00000001800065c8     libucrt:lcidtoname_downlevel.obj
 0001:000055d8       ??_C@_1M@ELCKCCJJ@?$AAm?$AAi?$AA?9?$AAn?$AAz?$AA?$AA@ 00000001800065d8     libucrt:lcidtoname_downlevel.obj
 0001:000055e8       ??_C@_1M@CBOOLAPA@?$AAm?$AAk?$AA?9?$AAm?$AAk?$AA?$AA@ 00000001800065e8     libucrt:lcidtoname_downlevel.obj
 0001:000055f8       ??_C@_1M@GPHNBJKN@?$AAm?$AAl?$AA?9?$AAi?$AAn?$AA?$AA@ 00000001800065f8     libucrt:lcidtoname_downlevel.obj
 0001:00005608       ??_C@_1M@PABJILIG@?$AAm?$AAn?$AA?9?$AAm?$AAn?$AA?$AA@ 0000000180006608     libucrt:lcidtoname_downlevel.obj
 0001:00005618       ??_C@_1M@FGBKKIPG@?$AAm?$AAr?$AA?9?$AAi?$AAn?$AA?$AA@ 0000000180006618     libucrt:lcidtoname_downlevel.obj
 0001:00005628       ??_C@_1M@NDBPDDAL@?$AAm?$AAs?$AA?9?$AAb?$AAn?$AA?$AA@ 0000000180006628     libucrt:lcidtoname_downlevel.obj
 0001:00005638       ??_C@_1M@OPIHOOPI@?$AAm?$AAs?$AA?9?$AAm?$AAy?$AA?$AA@ 0000000180006638     libucrt:lcidtoname_downlevel.obj
 0001:00005648       ??_C@_1M@PPDBCNFM@?$AAm?$AAt?$AA?9?$AAm?$AAt?$AA?$AA@ 0000000180006648     libucrt:lcidtoname_downlevel.obj
 0001:00005658       ??_C@_1M@KDJDKMDD@?$AAn?$AAb?$AA?9?$AAn?$AAo?$AA?$AA@ 0000000180006658     libucrt:lcidtoname_downlevel.obj
 0001:00005668       ??_C@_1M@KFCFLMJP@?$AAn?$AAl?$AA?9?$AAb?$AAe?$AA?$AA@ 0000000180006668     libucrt:lcidtoname_downlevel.obj
 0001:00005678       ??_C@_1M@KPOPDDGO@?$AAn?$AAl?$AA?9?$AAn?$AAl?$AA?$AA@ 0000000180006678     libucrt:lcidtoname_downlevel.obj
 0001:00005688       ??_C@_1M@LJKPEMLN@?$AAn?$AAn?$AA?9?$AAn?$AAo?$AA?$AA@ 0000000180006688     libucrt:lcidtoname_downlevel.obj
 0001:00005698       ??_C@_1M@BDGHHBFL@?$AAn?$AAs?$AA?9?$AAz?$AAa?$AA?$AA@ 0000000180006698     libucrt:lcidtoname_downlevel.obj
 0001:000056a8       ??_C@_1M@IDEHOAP@?$AAp?$AAa?$AA?9?$AAi?$AAn?$AA?$AA@ 00000001800066a8     libucrt:lcidtoname_downlevel.obj
 0001:000056b8       ??_C@_1M@HDBKGOGH@?$AAp?$AAl?$AA?9?$AAp?$AAl?$AA?$AA@ 00000001800066b8     libucrt:lcidtoname_downlevel.obj
 0001:000056c8       ??_C@_1M@LJLLCMEH@?$AAp?$AAt?$AA?9?$AAb?$AAr?$AA?$AA@ 00000001800066c8     libucrt:lcidtoname_downlevel.obj
 0001:000056d8       ??_C@_1M@NCMONAAL@?$AAp?$AAt?$AA?9?$AAp?$AAt?$AA?$AA@ 00000001800066d8     libucrt:lcidtoname_downlevel.obj
 0001:000056e8       ??_C@_1O@EAKMAJDN@?$AAq?$AAu?$AAz?$AA?9?$AAb?$AAo?$AA?$AA@ 00000001800066e8     libucrt:lcidtoname_downlevel.obj
 0001:000056f8       ??_C@_1O@BHHPIGDN@?$AAq?$AAu?$AAz?$AA?9?$AAe?$AAc?$AA?$AA@ 00000001800066f8     libucrt:lcidtoname_downlevel.obj
 0001:00005708       ??_C@_1O@GBAPEKMJ@?$AAq?$AAu?$AAz?$AA?9?$AAp?$AAe?$AA?$AA@ 0000000180006708     libucrt:lcidtoname_downlevel.obj
 0001:00005718       ??_C@_1M@CLGLEFBO@?$AAr?$AAo?$AA?9?$AAr?$AAo?$AA?$AA@ 0000000180006718     libucrt:lcidtoname_downlevel.obj
 0001:00005728       ??_C@_1M@CEEDODME@?$AAr?$AAu?$AA?9?$AAr?$AAu?$AA?$AA@ 0000000180006728     libucrt:lcidtoname_downlevel.obj
 0001:00005738       ??_C@_1M@HPKKKMPP@?$AAs?$AAa?$AA?9?$AAi?$AAn?$AA?$AA@ 0000000180006738     libucrt:lcidtoname_downlevel.obj
 0001:00005748       ??_C@_1M@BKMAIGOJ@?$AAs?$AAe?$AA?9?$AAf?$AAi?$AA?$AA@ 0000000180006748     libucrt:lcidtoname_downlevel.obj
 0001:00005758       ??_C@_1M@NDPIFLFI@?$AAs?$AAe?$AA?9?$AAn?$AAo?$AA?$AA@ 0000000180006758     libucrt:lcidtoname_downlevel.obj
 0001:00005768       ??_C@_1M@DANKKHJ@?$AAs?$AAe?$AA?9?$AAs?$AAe?$AA?$AA@ 0000000180006768     libucrt:lcidtoname_downlevel.obj
 0001:00005778       ??_C@_1M@PNBLONPJ@?$AAs?$AAk?$AA?9?$AAs?$AAk?$AA?$AA@ 0000000180006778     libucrt:lcidtoname_downlevel.obj
 0001:00005788       ??_C@_1M@LFMODOAL@?$AAs?$AAl?$AA?9?$AAs?$AAi?$AA?$AA@ 0000000180006788     libucrt:lcidtoname_downlevel.obj
 0001:00005798       ??_C@_1O@DFKOMPG@?$AAs?$AAm?$AAa?$AA?9?$AAn?$AAo?$AA?$AA@ 0000000180006798     libucrt:lcidtoname_downlevel.obj
 0001:000057a8       ??_C@_1O@NDKPBNNH@?$AAs?$AAm?$AAa?$AA?9?$AAs?$AAe?$AA?$AA@ 00000001800067a8     libucrt:lcidtoname_downlevel.obj
 0001:000057b8       ??_C@_1O@PLLKBHAB@?$AAs?$AAm?$AAj?$AA?9?$AAn?$AAo?$AA?$AA@ 00000001800067b8     libucrt:lcidtoname_downlevel.obj
 0001:000057c8       ??_C@_1O@CLEPOGCA@?$AAs?$AAm?$AAj?$AA?9?$AAs?$AAe?$AA?$AA@ 00000001800067c8     libucrt:lcidtoname_downlevel.obj
 0001:000057d8       ??_C@_1O@DLGJGKMK@?$AAs?$AAm?$AAn?$AA?9?$AAf?$AAi?$AA?$AA@ 00000001800067d8     libucrt:lcidtoname_downlevel.obj
 0001:000057e8       ??_C@_1O@OJDJGAJC@?$AAs?$AAm?$AAs?$AA?9?$AAf?$AAi?$AA?$AA@ 00000001800067e8     libucrt:lcidtoname_downlevel.obj
 0001:000057f8       ??_C@_1M@BOFOGHPB@?$AAs?$AAq?$AA?9?$AAa?$AAl?$AA?$AA@ 00000001800067f8     libucrt:lcidtoname_downlevel.obj
 0001:00005808       ??_C@_1BG@LJBBIPGB@?$AAs?$AAr?$AA?9?$AAb?$AAa?$AA?9?$AAc?$AAy?$AAr?$AAl?$AA?$AA@ 0000000180006808     libucrt:lcidtoname_downlevel.obj
 0001:00005820       ??_C@_1BG@JLBENFOE@?$AAs?$AAr?$AA?9?$AAb?$AAa?$AA?9?$AAl?$AAa?$AAt?$AAn?$AA?$AA@ 0000000180006820     libucrt:lcidtoname_downlevel.obj
 0001:00005838       ??_C@_1BG@KODPNHE@?$AAs?$AAr?$AA?9?$AAs?$AAp?$AA?9?$AAc?$AAy?$AAr?$AAl?$AA?$AA@ 0000000180006838     libucrt:lcidtoname_downlevel.obj
 0001:00005850       ??_C@_1BG@CIOGKHPB@?$AAs?$AAr?$AA?9?$AAs?$AAp?$AA?9?$AAl?$AAa?$AAt?$AAn?$AA?$AA@ 0000000180006850     libucrt:lcidtoname_downlevel.obj
 0001:00005868       ??_C@_1M@NGFJLMAC@?$AAs?$AAv?$AA?9?$AAf?$AAi?$AA?$AA@ 0000000180006868     libucrt:lcidtoname_downlevel.obj
 0001:00005878       ??_C@_1M@MPJEJAJC@?$AAs?$AAv?$AA?9?$AAs?$AAe?$AA?$AA@ 0000000180006878     libucrt:lcidtoname_downlevel.obj
 0001:00005888       ??_C@_1M@MPNDHLFK@?$AAs?$AAw?$AA?9?$AAk?$AAe?$AA?$AA@ 0000000180006888     libucrt:lcidtoname_downlevel.obj
 0001:00005898       ??_C@_1O@KOHBJJI@?$AAs?$AAy?$AAr?$AA?9?$AAs?$AAy?$AA?$AA@ 0000000180006898     libucrt:lcidtoname_downlevel.obj
 0001:000058a8       ??_C@_1M@LDCEFHA@?$AAt?$AAa?$AA?9?$AAi?$AAn?$AA?$AA@ 00000001800068a8     libucrt:lcidtoname_downlevel.obj
 0001:000058b8       ??_C@_1M@CNJOFAK@?$AAt?$AAe?$AA?9?$AAi?$AAn?$AA?$AA@ 00000001800068b8     libucrt:lcidtoname_downlevel.obj
 0001:000058c8       ??_C@_1M@GNAECACD@?$AAt?$AAh?$AA?9?$AAt?$AAh?$AA?$AA@ 00000001800068c8     libucrt:lcidtoname_downlevel.obj
 0001:000058d8       ??_C@_1M@CHBIHOJO@?$AAt?$AAn?$AA?9?$AAz?$AAa?$AA?$AA@ 00000001800068d8     libucrt:lcidtoname_downlevel.obj
 0001:000058e8       ??_C@_1M@GCCMIGPJ@?$AAt?$AAr?$AA?9?$AAt?$AAr?$AA?$AA@ 00000001800068e8     libucrt:lcidtoname_downlevel.obj
 0001:000058f8       ??_C@_1M@CELMCNBK@?$AAt?$AAt?$AA?9?$AAr?$AAu?$AA?$AA@ 00000001800068f8     libucrt:lcidtoname_downlevel.obj
 0001:00005908       ??_C@_1M@KLMCELGA@?$AAu?$AAk?$AA?9?$AAu?$AAa?$AA?$AA@ 0000000180006908     libucrt:lcidtoname_downlevel.obj
 0001:00005918       ??_C@_1M@EPAJJAJF@?$AAu?$AAr?$AA?9?$AAp?$AAk?$AA?$AA@ 0000000180006918     libucrt:lcidtoname_downlevel.obj
 0001:00005928       ??_C@_1BG@GEGPMCDJ@?$AAu?$AAz?$AA?9?$AAu?$AAz?$AA?9?$AAc?$AAy?$AAr?$AAl?$AA?$AA@ 0000000180006928     libucrt:lcidtoname_downlevel.obj
 0001:00005940       ??_C@_1BG@EGGKJILM@?$AAu?$AAz?$AA?9?$AAu?$AAz?$AA?9?$AAl?$AAa?$AAt?$AAn?$AA?$AA@ 0000000180006940     libucrt:lcidtoname_downlevel.obj
 0001:00005958       ??_C@_1M@GFOCLFF@?$AAv?$AAi?$AA?9?$AAv?$AAn?$AA?$AA@ 0000000180006958     libucrt:lcidtoname_downlevel.obj
 0001:00005968       ??_C@_1M@CPAMEDFI@?$AAx?$AAh?$AA?9?$AAz?$AAa?$AA?$AA@ 0000000180006968     libucrt:lcidtoname_downlevel.obj
 0001:00005978       ??_C@_1O@EBKIFIGN@?$AAz?$AAh?$AA?9?$AAc?$AAh?$AAs?$AA?$AA@ 0000000180006978     libucrt:lcidtoname_downlevel.obj
 0001:00005988       ??_C@_1O@NMHPGANE@?$AAz?$AAh?$AA?9?$AAc?$AAh?$AAt?$AA?$AA@ 0000000180006988     libucrt:lcidtoname_downlevel.obj
 0001:00005998       ??_C@_1M@LPINJOMC@?$AAz?$AAh?$AA?9?$AAc?$AAn?$AA?$AA@ 0000000180006998     libucrt:lcidtoname_downlevel.obj
 0001:000059a8       ??_C@_1M@OCJEJODD@?$AAz?$AAh?$AA?9?$AAh?$AAk?$AA?$AA@ 00000001800069a8     libucrt:lcidtoname_downlevel.obj
 0001:000059b8       ??_C@_1M@DNDLJINH@?$AAz?$AAh?$AA?9?$AAm?$AAo?$AA?$AA@ 00000001800069b8     libucrt:lcidtoname_downlevel.obj
 0001:000059c8       ??_C@_1M@MBFDNDND@?$AAz?$AAh?$AA?9?$AAs?$AAg?$AA?$AA@ 00000001800069c8     libucrt:lcidtoname_downlevel.obj
 0001:000059d8       ??_C@_1M@IMEPLEPE@?$AAz?$AAh?$AA?9?$AAt?$AAw?$AA?$AA@ 00000001800069d8     libucrt:lcidtoname_downlevel.obj
 0001:000059e8       ??_C@_1M@BBGHNHJP@?$AAz?$AAu?$AA?9?$AAz?$AAa?$AA?$AA@ 00000001800069e8     libucrt:lcidtoname_downlevel.obj
 0001:00005c50       __log10_256_lead           0000000180006c50     libucrt:log10_256_lead_tail_table.obj
 0001:00006460       __log10_256_tail           0000000180007460     libucrt:log10_256_lead_tail_table.obj
 0001:00006c70       __log_F_inv_qword          0000000180007c70     libucrt:log_f_inv_qword_table.obj
 0001:00007480       ??_C@_05HGHHAHAP@log10?$AA@ 0000000180008480     libucrt:log_special.obj
 0001:00007488       ??_C@_1BA@BALFACEM@?$AAC?$AAO?$AAN?$AAO?$AAU?$AAT?$AA$?$AA?$AA@ 0000000180008488     libucrt:initcon.obj
 0001:000074e0       _load_config_used          00000001800084e0     LIBCMT:loadcfg.obj
 0001:00007578       ??_R4exception@std@@6B@    0000000180008578     LIBCMT:throw_bad_alloc.obj
 0001:000075a0       ??_R3exception@std@@8      00000001800085a0     LIBCMT:throw_bad_alloc.obj
 0001:000075b8       ??_R2exception@std@@8      00000001800085b8     LIBCMT:throw_bad_alloc.obj
 0001:000075c8       ??_R1A@?0A@EA@exception@std@@8 00000001800085c8     LIBCMT:throw_bad_alloc.obj
 0001:000075f0       ??_R4bad_alloc@std@@6B@    00000001800085f0     LIBCMT:throw_bad_alloc.obj
 0001:00007618       ??_R3bad_alloc@std@@8      0000000180008618     LIBCMT:throw_bad_alloc.obj
 0001:00007630       ??_R2bad_alloc@std@@8      0000000180008630     LIBCMT:throw_bad_alloc.obj
 0001:00007648       ??_R1A@?0A@EA@bad_alloc@std@@8 0000000180008648     LIBCMT:throw_bad_alloc.obj
 0001:00007670       ??_R4bad_array_new_length@std@@6B@ 0000000180008670     LIBCMT:throw_bad_alloc.obj
 0001:00007698       ??_R3bad_array_new_length@std@@8 0000000180008698     LIBCMT:throw_bad_alloc.obj
 0001:000076b0       ??_R2bad_array_new_length@std@@8 00000001800086b0     LIBCMT:throw_bad_alloc.obj
 0001:000076d0       ??_R1A@?0A@EA@bad_array_new_length@std@@8 00000001800086d0     LIBCMT:throw_bad_alloc.obj
 0001:000076f8       ??_R4type_info@@6B@        00000001800086f8     LIBCMT:std_type_info_static.obj
 0001:00007720       ??_R3type_info@@8          0000000180008720     LIBCMT:std_type_info_static.obj
 0001:00007738       ??_R2type_info@@8          0000000180008738     LIBCMT:std_type_info_static.obj
 0001:00007748       ??_R1A@?0A@EA@type_info@@8 0000000180008748     LIBCMT:std_type_info_static.obj
 0001:00007770       ?_TraceLoggingMetadata@?1??_TlgWrite@__vcrt_trace_logging_provider@@YAJPEBU_TlgProvider_t@2@PEFBXPEBU_GUID@@2IPEAU_EVENT_DATA_DESCRIPTOR@@@Z@4U_TraceLoggingMetadata_t@2@B 0000000180008770     libvcruntime:telemetry.obj
 0001:00007823       ?_TraceLoggingMetadataEnd@?1??_TlgWrite@__vcrt_trace_logging_provider@@YAJPEBU_TlgProvider_t@2@PEFBXPEBU_GUID@@2IPEAU_EVENT_DATA_DESCRIPTOR@@@Z@4EB 0000000180008823     libvcruntime:telemetry.obj
 0001:00007b70       __rtc_iaa                  0000000180008b70     LIBCMT:_initsect_.obj
 0001:00007b78       __rtc_izz                  0000000180008b78     LIBCMT:_initsect_.obj
 0001:00007b80       __rtc_taa                  0000000180008b80     LIBCMT:_initsect_.obj
 0001:00007b88       __rtc_tzz                  0000000180008b88     LIBCMT:_initsect_.obj
 0001:00007b90       ?TraceLoggingRegister@__vcrt_trace_logging_provider@@YAJPEBU_TlgProvider_t@1@PEBU_GUID@@P6AX1KE_K2PEAU_EVENT_FILTER_DESCRIPTOR@@PEAX@Z4@Z 0000000180008b90 f i libvcruntime:telemetry.obj
 0001:00007c0c       ?_TlgEnableCallback@__vcrt_trace_logging_provider@@YAXPEBU_GUID@@KE_K1PEAU_EVENT_FILTER_DESCRIPTOR@@PEAX@Z 0000000180008c0c f i libvcruntime:telemetry.obj
 0001:00007cd0       ?_TlgWrite@__vcrt_trace_logging_provider@@YAJPEBU_TlgProvider_t@1@PEFBXPEBU_GUID@@2IPEAU_EVENT_DATA_DESCRIPTOR@@@Z 0000000180008cd0 f i libvcruntime:telemetry.obj
 0001:00007d80       _alloca_probe              0000000180008d80 f   chkstk.obj
 0001:00007d80       __chkstk                   0000000180008d80 f   chkstk.obj
 0001:00007de0       ??0PluginIntEditFieldBinding@@QEAA@AEBUPluginStartupInfo@@PEAPEAXHPEAHH@Z 0000000180008de0 f i AutoWrap.obj
 0001:00007ea0       ??0PluginUIntEditFieldBinding@@QEAA@AEBUPluginStartupInfo@@PEAPEAXHPEAIH@Z 0000000180008ea0 f i AutoWrap.obj
 0001:00007f60       ??1?$DialogBuilderBase@UFarDialogItem@@@@MEAA@XZ 0000000180008f60 f i AutoWrap.obj
 0001:00007fe0       ??_G?$DialogBuilderBase@UFarDialogItem@@@@MEAAPEAXI@Z 0000000180008fe0 f i AutoWrap.obj
 0001:00007fe0       ??_E?$DialogBuilderBase@UFarDialogItem@@@@MEAAPEAXI@Z 0000000180008fe0 f i AutoWrap.obj
 0001:00008020       ??_E?$DialogItemBinding@UFarDialogItem@@@@UEAAPEAXI@Z 0000000180009020 f i AutoWrap.obj
 0001:00008020       ??_G?$DialogItemBinding@UFarDialogItem@@@@UEAAPEAXI@Z 0000000180009020 f i AutoWrap.obj
 0001:00008050       ??_GPluginEditFieldBinding@@UEAAPEAXI@Z 0000000180009050 f i AutoWrap.obj
 0001:00008050       ??_GPluginCheckBoxBinding@@UEAAPEAXI@Z 0000000180009050 f i AutoWrap.obj
 0001:00008050       ??_EPluginCheckBoxBinding@@UEAAPEAXI@Z 0000000180009050 f i AutoWrap.obj
 0001:00008050       ??_EPluginEditFieldBinding@@UEAAPEAXI@Z 0000000180009050 f i AutoWrap.obj
 0001:00008080       ??_GPluginDialogBuilder@@UEAAPEAXI@Z 0000000180009080 f i AutoWrap.obj
 0001:00008080       ??_EPluginDialogBuilder@@UEAAPEAXI@Z 0000000180009080 f i AutoWrap.obj
 0001:000080d0       ??_GPluginIntEditFieldBinding@@UEAAPEAXI@Z 00000001800090d0 f i AutoWrap.obj
 0001:000080d0       ??_EPluginUIntEditFieldBinding@@UEAAPEAXI@Z 00000001800090d0 f i AutoWrap.obj
 0001:000080d0       ??_EPluginIntEditFieldBinding@@UEAAPEAXI@Z 00000001800090d0 f i AutoWrap.obj
 0001:000080d0       ??_GPluginUIntEditFieldBinding@@UEAAPEAXI@Z 00000001800090d0 f i AutoWrap.obj
 0001:00008100       ??_EPluginRadioButtonBinding@@UEAAPEAXI@Z 0000000180009100 f i AutoWrap.obj
 0001:00008100       ??_GPluginRadioButtonBinding@@UEAAPEAXI@Z 0000000180009100 f i AutoWrap.obj
 0001:00008130       ?AddButtons@?$DialogBuilderBase@UFarDialogItem@@@@QEAAXHPEBHHH@Z 0000000180009130 f i AutoWrap.obj
 0001:00008290       ?AddDialogItem@?$DialogBuilderBase@UFarDialogItem@@@@IEAAPEAUFarDialogItem@@W4FARDIALOGITEMTYPES@@PEB_W@Z 0000000180009290 f i AutoWrap.obj
 0001:00008320       ?AddIntEditField@PluginDialogBuilder@@UEAAPEAUFarDialogItem@@PEAHH@Z 0000000180009320 f i AutoWrap.obj
 0001:00008430       ?AddTextAfter@?$DialogBuilderBase@UFarDialogItem@@@@QEAAPEAUFarDialogItem@@PEAU2@PEB_WH@Z 0000000180009430 f i AutoWrap.obj
 0001:00008500       ?GetLangString@?$DialogBuilderBase@UFarDialogItem@@@@MEAAPEB_WH@Z 0000000180009500 f i AutoWrap.obj
 0001:00008500       ?AddUIntEditField@?$DialogBuilderBase@UFarDialogItem@@@@UEAAPEAUFarDialogItem@@PEAIH@Z 0000000180009500 f i AutoWrap.obj
 0001:00008500       ?CreateRadioButtonBinding@?$DialogBuilderBase@UFarDialogItem@@@@MEAAPEAU?$DialogItemBinding@UFarDialogItem@@@@PEAH@Z 0000000180009500 f i AutoWrap.obj
 0001:00008500       ?CreateCheckBoxBinding@?$DialogBuilderBase@UFarDialogItem@@@@MEAAPEAU?$DialogItemBinding@UFarDialogItem@@@@PEAHH@Z 0000000180009500 f i AutoWrap.obj
 0001:00008500       ?AddIntEditField@?$DialogBuilderBase@UFarDialogItem@@@@UEAAPEAUFarDialogItem@@PEAHH@Z 0000000180009500 f i AutoWrap.obj
 0001:00008510       ?AddUIntEditField@PluginDialogBuilder@@UEAAPEAUFarDialogItem@@PEAIH@Z 0000000180009510 f i AutoWrap.obj
 0001:00008620       ?CreateCheckBoxBinding@PluginDialogBuilder@@MEAAPEAU?$DialogItemBinding@UFarDialogItem@@@@PEAHH@Z 0000000180009620 f i AutoWrap.obj
 0001:000086a0       ?CreateRadioButtonBinding@PluginDialogBuilder@@MEAAPEAU?$DialogItemBinding@UFarDialogItem@@@@PEAH@Z 00000001800096a0 f i AutoWrap.obj
 0001:00008710       ?DoShowDialog@?$DialogBuilderBase@UFarDialogItem@@@@MEAA_JXZ 0000000180009710 f i AutoWrap.obj
 0001:00008720       ?DoShowDialog@PluginDialogBuilder@@MEAA_JXZ 0000000180009720 f i AutoWrap.obj
 0001:000087d0       ?GetCommaWord@@YAPEB_WPEB_WPEA_W@Z 00000001800097d0 f   AutoWrap.obj
 0001:000088d0       ?GetLangString@PluginDialogBuilder@@MEAAPEB_WH@Z 00000001800098d0 f i AutoWrap.obj
 0001:000088e0       ?SaveValue@?$DialogItemBinding@UFarDialogItem@@@@UEAAXPEAUFarDialogItem@@H@Z 00000001800098e0 f i AutoWrap.obj
 0001:000088e0       _guard_check_icall_nop     00000001800098e0 f i LIBCMT:guard_support.obj
 0001:000088e0       ?InitDialogItem@?$DialogBuilderBase@UFarDialogItem@@@@MEAAXPEAUFarDialogItem@@PEB_W@Z 00000001800098e0 f i AutoWrap.obj
 0001:000088e0       __except_validate_context_record 00000001800098e0 f i libvcruntime:jbcxrval.obj
 0001:000088f0       ?InitDialogItem@PluginDialogBuilder@@MEAAXPEAUFarDialogItem@@PEB_W@Z 00000001800098f0 f i AutoWrap.obj
 0001:00008920       ?ItemWidth@?$DialogBuilderBase@UFarDialogItem@@@@IEAA_JAEBUFarDialogItem@@@Z 0000000180009920 f i AutoWrap.obj
 0001:000089c0       ?MaxTextWidth@?$DialogBuilderBase@UFarDialogItem@@@@IEAA_JXZ 00000001800099c0 f i AutoWrap.obj
 0001:00008af0       ?ReallocDialogItems@?$DialogBuilderBase@UFarDialogItem@@@@IEAAXXZ 0000000180009af0 f i AutoWrap.obj
 0001:00008c50       ?SaveValue@PluginCheckBoxBinding@@UEAAXPEAUFarDialogItem@@H@Z 0000000180009c50 f i AutoWrap.obj
 0001:00008cb0       ?SaveValue@PluginEditFieldBinding@@UEAAXPEAUFarDialogItem@@H@Z 0000000180009cb0 f i AutoWrap.obj
 0001:00008cf0       ?SaveValue@PluginIntEditFieldBinding@@UEAAXPEAUFarDialogItem@@H@Z 0000000180009cf0 f i AutoWrap.obj
 0001:00008d40       ?SaveValue@PluginRadioButtonBinding@@UEAAXPEAUFarDialogItem@@H@Z 0000000180009d40 f i AutoWrap.obj
 0001:00008d90       ?SaveValue@PluginUIntEditFieldBinding@@UEAAXPEAUFarDialogItem@@H@Z 0000000180009d90 f i AutoWrap.obj
 0001:00008de0       ?SaveValues@?$DialogBuilderBase@UFarDialogItem@@@@IEAAXXZ 0000000180009de0 f i AutoWrap.obj
 0001:00008e70       ?TextWidth@?$DialogBuilderBase@UFarDialogItem@@@@MEAAHAEBUFarDialogItem@@@Z 0000000180009e70 f i AutoWrap.obj
 0001:00008e80       ?TextWidth@PluginDialogBuilder@@MEAAHAEBUFarDialogItem@@@Z 0000000180009e80 f i AutoWrap.obj
 0001:00008e90       ?UpdateBorderSize@?$DialogBuilderBase@UFarDialogItem@@@@IEAAXXZ 0000000180009e90 f i AutoWrap.obj
 0001:00008f50       GetGlobalInfoW             0000000180009f50 f   AutoWrap.obj
 0001:00008fd0       GetPluginInfoW             0000000180009fd0 f   AutoWrap.obj
 0001:00009030       OpenW                      000000018000a030 f   AutoWrap.obj
 0001:00009920       ProcessEditorInputW        000000018000a920 f   AutoWrap.obj
 0001:00009e60       SetStartupInfoW            000000018000ae60 f   AutoWrap.obj
 0001:0000a0fc       ??2@YAPEAX_K@Z             000000018000b0fc f   LIBCMT:new_scalar.obj
 0001:0000a138       ??_V@YAXPEAX@Z             000000018000b138 f   LIBCMT:delete_array.obj
 0001:0000a138       ??3@YAXPEAX_K@Z            000000018000b138 f   LIBCMT:delete_scalar_size.obj
 0001:0000a140       ??_U@YAPEAX_K@Z            000000018000b140 f   LIBCMT:new_array.obj
 0001:0000a4b8       _DllMainCRTStartup         000000018000b4b8 f   LIBCMT:dll_dllmain.obj
 0001:0000a4f8       ??0bad_alloc@std@@QEAA@AEBV01@@Z 000000018000b4f8 f i LIBCMT:throw_bad_alloc.obj
 0001:0000a538       ??0bad_alloc@std@@QEAA@XZ  000000018000b538 f i LIBCMT:throw_bad_alloc.obj
 0001:0000a558       ??0bad_array_new_length@std@@QEAA@AEBV01@@Z 000000018000b558 f i LIBCMT:throw_bad_alloc.obj
 0001:0000a598       ??0bad_array_new_length@std@@QEAA@XZ 000000018000b598 f i LIBCMT:throw_bad_alloc.obj
 0001:0000a5b8       ??0exception@std@@QEAA@AEBV01@@Z 000000018000b5b8 f i LIBCMT:throw_bad_alloc.obj
 0001:0000a5f0       ??1bad_array_new_length@std@@UEAA@XZ 000000018000b5f0 f i LIBCMT:throw_bad_alloc.obj
 0001:0000a5f0       ??1bad_alloc@std@@UEAA@XZ  000000018000b5f0 f i LIBCMT:throw_bad_alloc.obj
 0001:0000a604       ??_Gbad_alloc@std@@UEAAPEAXI@Z 000000018000b604 f i LIBCMT:throw_bad_alloc.obj
 0001:0000a604       ??_Eexception@std@@UEAAPEAXI@Z 000000018000b604 f i LIBCMT:throw_bad_alloc.obj
 0001:0000a604       ??_Ebad_alloc@std@@UEAAPEAXI@Z 000000018000b604 f i LIBCMT:throw_bad_alloc.obj
 0001:0000a604       ??_Gbad_array_new_length@std@@UEAAPEAXI@Z 000000018000b604 f i LIBCMT:throw_bad_alloc.obj
 0001:0000a604       ??_Gexception@std@@UEAAPEAXI@Z 000000018000b604 f i LIBCMT:throw_bad_alloc.obj
 0001:0000a604       ??_Ebad_array_new_length@std@@UEAAPEAXI@Z 000000018000b604 f i LIBCMT:throw_bad_alloc.obj
 0001:0000a648       ?__scrt_throw_std_bad_alloc@@YAXXZ 000000018000b648 f   LIBCMT:throw_bad_alloc.obj
 0001:0000a668       ?__scrt_throw_std_bad_array_new_length@@YAXXZ 000000018000b668 f   LIBCMT:throw_bad_alloc.obj
 0001:0000a688       ?what@exception@std@@UEBAPEBDXZ 000000018000b688 f i LIBCMT:throw_bad_alloc.obj
 0001:0000a69c       ??3@YAXPEAX@Z              000000018000b69c f   LIBCMT:delete_scalar.obj
 0001:0000a6a4       __scrt_acquire_startup_lock 000000018000b6a4 f   LIBCMT:utility.obj
 0001:0000a6e0       __scrt_dllmain_after_initialize_c 000000018000b6e0 f   LIBCMT:utility.obj
 0001:0000a714       __scrt_dllmain_before_initialize_c 000000018000b714 f   LIBCMT:utility.obj
 0001:0000a72c       __scrt_dllmain_crt_thread_attach 000000018000b72c f   LIBCMT:utility.obj
 0001:0000a754       __scrt_dllmain_crt_thread_detach 000000018000b754 f   LIBCMT:utility.obj
 0001:0000a76c       __scrt_dllmain_exception_filter 000000018000b76c f   LIBCMT:utility.obj
 0001:0000a7d0       __scrt_dllmain_uninitialize_c 000000018000b7d0 f   LIBCMT:utility.obj
 0001:0000a800       __scrt_dllmain_uninitialize_critical 000000018000b800 f   LIBCMT:utility.obj
 0001:0000a814       __scrt_initialize_crt      000000018000b814 f   LIBCMT:utility.obj
 0001:0000a860       __scrt_initialize_onexit_tables 000000018000b860 f   LIBCMT:utility.obj
 0001:0000a92c       __scrt_is_nonwritable_in_current_image 000000018000b92c f   LIBCMT:utility.obj
 0001:0000a9c8       __scrt_release_startup_lock 000000018000b9c8 f   LIBCMT:utility.obj
 0001:0000a9ec       __scrt_uninitialize_crt    000000018000b9ec f   LIBCMT:utility.obj
 0001:0000aa18       _onexit                    000000018000ba18 f   LIBCMT:utility.obj
 0001:0000aa68       atexit                     000000018000ba68 f   LIBCMT:utility.obj
 0001:0000aa80       __security_init_cookie     000000018000ba80 f   LIBCMT:gs_support.obj
 0001:0000ab2c       ?__scrt_initialize_type_info@@YAXXZ 000000018000bb2c f   LIBCMT:tncleanup.obj
 0001:0000ab3c       ?__scrt_uninitialize_type_info@@YAXXZ 000000018000bb3c f   LIBCMT:tncleanup.obj
 0001:0000ab48       __local_stdio_printf_options 000000018000bb48 f i LIBCMT:default_local_stdio_options.obj
 0001:0000ab50       __local_stdio_scanf_options 000000018000bb50 f i LIBCMT:default_local_stdio_options.obj
 0001:0000ab58       __scrt_initialize_default_local_stdio_options 000000018000bb58 f   LIBCMT:default_local_stdio_options.obj
 0001:0000ab74       __scrt_get_dyn_tls_init_callback 000000018000bb74 f   LIBCMT:dyn_tls_init.obj
 0001:0000ab7c       __crt_debugger_hook        000000018000bb7c f   LIBCMT:utility_desktop.obj
 0001:0000ab84       __scrt_fastfail            000000018000bb84 f   LIBCMT:utility_desktop.obj
 0001:0000accc       _RTC_Initialize            000000018000bccc f   LIBCMT:_initsect_.obj
 0001:0000ad18       _RTC_Terminate             000000018000bd18 f   LIBCMT:_initsect_.obj
 0001:0000ad64       _guard_check_icall         000000018000bd64 f i LIBCMT:checkcfg.obj
 0001:0000ad6c       ??_Etype_info@@UEAAPEAXI@Z 000000018000bd6c f i LIBCMT:std_type_info_static.obj
 0001:0000ad6c       ??_Gtype_info@@UEAAPEAXI@Z 000000018000bd6c f i LIBCMT:std_type_info_static.obj
 0001:0000ad98       __isa_available_init       000000018000bd98 f   LIBCMT:_cpu_disp_.obj
 0001:0000af5c       _get_startup_argv_mode     000000018000bf5c f   LIBCMT:argv_mode.obj
 0001:0000af5c       DllMain                    000000018000bf5c f   LIBCMT:dll_dllmain_stub.obj
 0001:0000af64       __scrt_is_ucrt_dll_in_use  000000018000bf64 f   LIBCMT:ucrt_detection.obj
 0001:0000af70       wcschr                     000000018000bf70 f   libvcruntime:wcschr.obj
 0001:0000b010       memset                     000000018000c010 f   libvcruntime:memset.obj
 0001:0000b1b4       __telemetry_main_invoke_trigger 000000018000c1b4 f   libvcruntime:telemetry.obj
 0001:0000b2cc       __telemetry_main_return_trigger 000000018000c2cc f   libvcruntime:telemetry.obj
 0001:0000b3e4       __vcrt_initialize_telemetry_provider 000000018000c3e4 f   libvcruntime:telemetry.obj
 0001:0000b3f8       __vcrt_uninitialize_telemetry_provider 000000018000c3f8 f   libvcruntime:telemetry.obj
 0001:0000b418       __C_specific_handler       000000018000c418 f   libvcruntime:_chandler_.obj
 0001:0000b614       __std_exception_copy       000000018000c614 f   libvcruntime:std_exception.obj
 0001:0000b6a4       __std_exception_destroy    000000018000c6a4 f   libvcruntime:std_exception.obj
 0001:0000b6cc       _CxxThrowException         000000018000c6cc f   libvcruntime:throw.obj
 0001:0000b7a4       __vcrt_initialize          000000018000c7a4 f   libvcruntime:initialization.obj
 0001:0000b7dc       __vcrt_thread_attach       000000018000c7dc f   libvcruntime:initialization.obj
 0001:0000b7f0       __vcrt_thread_detach       000000018000c7f0 f   libvcruntime:initialization.obj
 0001:0000b804       __vcrt_uninitialize        000000018000c804 f   libvcruntime:initialization.obj
 0001:0000b830       __vcrt_uninitialize_critical 000000018000c830 f   libvcruntime:initialization.obj
 0001:0000b840       __std_type_info_destroy_list 000000018000c840 f   libvcruntime:std_type_info.obj
 0001:0000ba34       __vcrt_EventRegister       000000018000ca34 f   libvcruntime:winapi_downlevel.obj
 0001:0000bab8       __vcrt_EventSetInformation 000000018000cab8 f   libvcruntime:winapi_downlevel.obj
 0001:0000bb3c       __vcrt_EventUnregister     000000018000cb3c f   libvcruntime:winapi_downlevel.obj
 0001:0000bb90       __vcrt_EventWriteTransfer  000000018000cb90 f   libvcruntime:winapi_downlevel.obj
 0001:0000bc28       __vcrt_FlsAlloc            000000018000cc28 f   libvcruntime:winapi_downlevel.obj
 0001:0000bc7c       __vcrt_FlsFree             000000018000cc7c f   libvcruntime:winapi_downlevel.obj
 0001:0000bcd0       __vcrt_FlsGetValue         000000018000ccd0 f   libvcruntime:winapi_downlevel.obj
 0001:0000bd24       __vcrt_FlsSetValue         000000018000cd24 f   libvcruntime:winapi_downlevel.obj
 0001:0000bd8c       __vcrt_InitializeCriticalSectionEx 000000018000cd8c f   libvcruntime:winapi_downlevel.obj
 0001:0000be04       __vcrt_initialize_winapi_thunks 000000018000ce04 f   libvcruntime:winapi_downlevel.obj
 0001:0000be3c       __vcrt_uninitialize_winapi_thunks 000000018000ce3c f   libvcruntime:winapi_downlevel.obj
 0001:0000be90       _local_unwind              000000018000ce90 f   libvcruntime:_jmpuwind_.obj
 0001:0000bec0       _NLG_Notify                000000018000cec0 f   libvcruntime:_jmpuwind_.obj
 0001:0000bee0       __NLG_Dispatch2            000000018000cee0 f   libvcruntime:_jmpuwind_.obj
 0001:0000bef0       __NLG_Return2              000000018000cef0 f   libvcruntime:_jmpuwind_.obj
 0001:0000bef4       __vcrt_freefls             000000018000cef4 f   libvcruntime:per_thread_data.obj
 0001:0000bf14       __vcrt_freeptd             000000018000cf14 f   libvcruntime:per_thread_data.obj
 0001:0000bf64       __vcrt_getptd_noexit       000000018000cf64 f   libvcruntime:per_thread_data.obj
 0001:0000c01c       __vcrt_initialize_ptd      000000018000d01c f   libvcruntime:per_thread_data.obj
 0001:0000c05c       __vcrt_uninitialize_ptd    000000018000d05c f   libvcruntime:per_thread_data.obj
 0001:0000c080       __vcrt_initialize_locks    000000018000d080 f   libvcruntime:locks.obj
 0001:0000c0c8       __vcrt_uninitialize_locks  000000018000d0c8 f   libvcruntime:locks.obj
 0001:0000c100       __vcrt_initialize_pure_virtual_call_handler 000000018000d100 f   libvcruntime:purevirt_data.obj
 0001:0000c124       ??0_LocaleUpdate@@QEAA@QEAU__crt_locale_pointers@@@Z 000000018000d124 f i libucrt:_wctype.obj
 0001:0000c1b4       _isleadbyte_l              000000018000d1b4 f i libucrt:_wctype.obj
 0001:0000c1f4       iswspace                   000000018000d1f4 f i libucrt:_wctype.obj
 0001:0000c200       __acrt_initialize_new_handler 000000018000d200 f   libucrt:new_handler.obj
 0001:0000c208       _callnewh                  000000018000d208 f   libucrt:new_handler.obj
 0001:0000c248       _query_new_handler         000000018000d248 f   libucrt:new_handler.obj
 0001:0000c27c       malloc                     000000018000d27c f   libucrt:malloc.obj
 0001:0000c284       _initterm                  000000018000d284 f   libucrt:initterm.obj
 0001:0000c2fc       _initterm_e                000000018000d2fc f   libucrt:initterm.obj
 0001:0000c348       free                       000000018000d348 f   libucrt:free.obj
 0001:0000c350       _seh_filter_dll            000000018000d350 f   libucrt:exception_filter.obj
 0001:0000c364       _seh_filter_exe            000000018000d364 f   libucrt:exception_filter.obj
 0001:0000c724       __acrt_initialize_thread_local_exit_callback 000000018000d724 f   libucrt:exit.obj
 0001:0000c72c       _cexit                     000000018000d72c f   libucrt:exit.obj
 0001:0000c73c       _exit                      000000018000d73c f   libucrt:exit.obj
 0001:0000c748       _is_c_termination_complete 000000018000d748 f   libucrt:exit.obj
 0001:0000c90c       __acrt_allocate_buffer_for_argv 000000018000d90c f   libucrt:argv_parsing.obj
 0001:0000c970       _configure_narrow_argv     000000018000d970 f   libucrt:argv_parsing.obj
 0001:0000cccc       __dcrt_uninitialize_environments_nolock 000000018000dccc f   libucrt:environment_initialization.obj
 0001:0000cd04       _initialize_narrow_environment 000000018000dd04 f   libucrt:environment_initialization.obj
 0001:0000cd0c       ??$?RV<lambda_b8c45f8f788dd370798f47cfe8ac3a86>@@AEAV<lambda_4e60a939b0d047cfe11ddc22648dfba9>@@V<lambda_332c3edc96d0294ec56c57d38c1cdfd5>@@@?$__crt_seh_guarded_call@H@@QEAAH$$QEAV<lambda_b8c45f8f788dd370798f47cfe8ac3a86>@@AEAV<lambda_4e60a939b0d047cfe11ddc22648dfba9>@@$$QEAV<lambda_332c3edc96d0294ec56c57d38c1cdfd5>@@@Z 000000018000dd0c f i libucrt:onexit.obj
 0001:0000cd48       ??$?RV<lambda_e24bbb7b643b32fcea6fa61b31d4c984>@@AEAV<lambda_275893d493268fdec8709772e3fcec0e>@@V<lambda_9d71df4d7cf3f480f8d633942495c3b0>@@@?$__crt_seh_guarded_call@H@@QEAAH$$QEAV<lambda_e24bbb7b643b32fcea6fa61b31d4c984>@@AEAV<lambda_275893d493268fdec8709772e3fcec0e>@@$$QEAV<lambda_9d71df4d7cf3f480f8d633942495c3b0>@@@Z 000000018000dd48 f i libucrt:onexit.obj
 0001:0000d0c4       _crt_atexit                000000018000e0c4 f   libucrt:onexit.obj
 0001:0000d0d4       _execute_onexit_table      000000018000e0d4 f   libucrt:onexit.obj
 0001:0000d110       _initialize_onexit_table   000000018000e110 f   libucrt:onexit.obj
 0001:0000d150       _register_onexit_function  000000018000e150 f   libucrt:onexit.obj
 0001:0000d1d0       __acrt_uninitialize_command_line 000000018000e1d0 f   libucrt:argv_data.obj
 0001:0000d2d0       __acrt_initialize          000000018000e2d0 f   libucrt:initialization.obj
 0001:0000d2e4       __acrt_thread_attach       000000018000e2e4 f   libucrt:initialization.obj
 0001:0000d2f8       __acrt_thread_detach       000000018000e2f8 f   libucrt:initialization.obj
 0001:0000d308       __acrt_uninitialize        000000018000e308 f   libucrt:initialization.obj
 0001:0000d31c       __acrt_uninitialize_critical 000000018000e31c f   libucrt:initialization.obj
 0001:0000d32c       terminate                  000000018000e32c f   libucrt:terminate.obj
 0001:0000d354       strcpy_s                   000000018000e354 f   libucrt:strcpy_s.obj
 0001:0000d3b4       _free_base                 000000018000e3b4 f   libucrt:free_base.obj
 0001:0000d3f4       _malloc_base               000000018000e3f4 f   libucrt:malloc_base.obj
 0001:0000d454       abort                      000000018000e454 f   libucrt:abort.obj
 0001:0000d4ac       _calloc_base               000000018000e4ac f   libucrt:calloc_base.obj
 0001:0000d524       iswctype                   000000018000e524 f   libucrt:iswctype.obj
 0001:0000d594       ??$?RV<lambda_46352004c1216016012b18bd6f87e700>@@AEAV<lambda_3bd07e1a1191394380780325891bf33f>@@V<lambda_334532d3f185bcaa59b5be82d7d22bff>@@@?$__crt_seh_guarded_call@X@@QEAAX$$QEAV<lambda_46352004c1216016012b18bd6f87e700>@@AEAV<lambda_3bd07e1a1191394380780325891bf33f>@@$$QEAV<lambda_334532d3f185bcaa59b5be82d7d22bff>@@@Z 000000018000e594 f i libucrt:per_thread_data.obj
 0001:0000d5f4       ??$?RV<lambda_5e887d1dcbef67a5eb4283622ba103bf>@@AEAV<lambda_4466841279450cc726390878d4a41900>@@V<lambda_341c25c0346d94847f1f3c463c57e077>@@@?$__crt_seh_guarded_call@X@@QEAAX$$QEAV<lambda_5e887d1dcbef67a5eb4283622ba103bf>@@AEAV<lambda_4466841279450cc726390878d4a41900>@@$$QEAV<lambda_341c25c0346d94847f1f3c463c57e077>@@@Z 000000018000e5f4 f i libucrt:per_thread_data.obj
 0001:0000d63c       ??$?RV<lambda_72d1df2b273a38828b1ce30cbf4cdab5>@@AEAV<lambda_876a65b173b8412d3a47c70a915b0cf4>@@V<lambda_41932305e351933ebe8f8be3ed8bb5dc>@@@?$__crt_seh_guarded_call@X@@QEAAX$$QEAV<lambda_72d1df2b273a38828b1ce30cbf4cdab5>@@AEAV<lambda_876a65b173b8412d3a47c70a915b0cf4>@@$$QEAV<lambda_41932305e351933ebe8f8be3ed8bb5dc>@@@Z 000000018000e63c f i libucrt:per_thread_data.obj
 0001:0000d67c       ??$?RV<lambda_fb3a7dec4e47f37f22dae91bb15c9095>@@AEAV<lambda_698284760c8add0bfb0756c19673e34b>@@V<lambda_dfb8eca1e75fef3034a8fb18dd509707>@@@?$__crt_seh_guarded_call@X@@QEAAX$$QEAV<lambda_fb3a7dec4e47f37f22dae91bb15c9095>@@AEAV<lambda_698284760c8add0bfb0756c19673e34b>@@$$QEAV<lambda_dfb8eca1e75fef3034a8fb18dd509707>@@@Z 000000018000e67c f i libucrt:per_thread_data.obj
 0001:0000d90c       __acrt_freeptd             000000018000e90c f   libucrt:per_thread_data.obj
 0001:0000d950       __acrt_getptd              000000018000e950 f   libucrt:per_thread_data.obj
 0001:0000d9e4       __acrt_getptd_noexit       000000018000e9e4 f   libucrt:per_thread_data.obj
 0001:0000da84       __acrt_initialize_ptd      000000018000ea84 f   libucrt:per_thread_data.obj
 0001:0000dac0       __acrt_uninitialize_ptd    000000018000eac0 f   libucrt:per_thread_data.obj
 0001:0000dae4       __acrt_update_locale_info  000000018000eae4 f   libucrt:locale_update.obj
 0001:0000db18       __acrt_update_multibyte_info 000000018000eb18 f   libucrt:locale_update.obj
 0001:0000db4c       __acrt_set_locale_changed  000000018000eb4c f   libucrt:wsetlocale.obj
 0001:0000db58       __acrt_uninitialize_locale 000000018000eb58 f   libucrt:wsetlocale.obj
 0001:0000dba0       __acrt_initialize_locks    000000018000eba0 f   libucrt:locks.obj
 0001:0000dbe8       __acrt_lock                000000018000ebe8 f   libucrt:locks.obj
 0001:0000dc04       __acrt_uninitialize_locks  000000018000ec04 f   libucrt:locks.obj
 0001:0000dc3c       __acrt_unlock              000000018000ec3c f   libucrt:locks.obj
 0001:0000ddf8       __acrt_FlsAlloc            000000018000edf8 f   libucrt:winapi_thunks.obj
 0001:0000de50       __acrt_FlsFree             000000018000ee50 f   libucrt:winapi_thunks.obj
 0001:0000dea8       __acrt_FlsGetValue         000000018000eea8 f   libucrt:winapi_thunks.obj
 0001:0000df00       __acrt_FlsSetValue         000000018000ef00 f   libucrt:winapi_thunks.obj
 0001:0000df68       __acrt_InitializeCriticalSectionEx 000000018000ef68 f   libucrt:winapi_thunks.obj
 0001:0000dfe0       __acrt_LCMapStringEx       000000018000efe0 f   libucrt:winapi_thunks.obj
 0001:0000e0d0       __acrt_LocaleNameToLCID    000000018000f0d0 f   libucrt:winapi_thunks.obj
 0001:0000e138       __acrt_initialize_winapi_thunks 000000018000f138 f   libucrt:winapi_thunks.obj
 0001:0000e170       __acrt_is_packaged_app     000000018000f170 f   libucrt:winapi_thunks.obj
 0001:0000e1f8       __acrt_uninitialize_winapi_thunks 000000018000f1f8 f   libucrt:winapi_thunks.obj
 0001:0000e23c       __acrt_call_reportfault    000000018000f23c f   libucrt:invalid_parameter.obj
 0001:0000e398       __acrt_initialize_invalid_parameter_handler 000000018000f398 f   libucrt:invalid_parameter.obj
 0001:0000e3a0       _invalid_parameter         000000018000f3a0 f   libucrt:invalid_parameter.obj
 0001:0000e448       _invalid_parameter_noinfo  000000018000f448 f   libucrt:invalid_parameter.obj
 0001:0000e468       _invoke_watson             000000018000f468 f   libucrt:invalid_parameter.obj
 0001:0000e4b0       __acrt_errno_from_os_error 000000018000f4b0 f   libucrt:errno.obj
 0001:0000e4f8       __acrt_errno_map_os_error  000000018000f4f8 f   libucrt:errno.obj
 0001:0000e548       __doserrno                 000000018000f548 f   libucrt:errno.obj
 0001:0000e568       _errno                     000000018000f568 f   libucrt:errno.obj
 0001:0000ea64       ?expand_if_necessary@?$argument_list@D@?A0xca0879c4@@AEAAHXZ 000000018000fa64 f i libucrt:argv_wildcards.obj
 0001:0000eb2c       __acrt_expand_narrow_argv_wildcards 000000018000fb2c f   libucrt:argv_wildcards.obj
 0001:0000eb34       ??$?RV<lambda_99476a1ad63dd22509b5d3e65b0ffc95>@@AEAV<lambda_ad1ced32f4ac17aa236e5ef05d6b3b7c>@@V<lambda_f7424dd8d45958661754dc4f2697e9c3>@@@?$__crt_seh_guarded_call@X@@QEAAX$$QEAV<lambda_99476a1ad63dd22509b5d3e65b0ffc95>@@AEAV<lambda_ad1ced32f4ac17aa236e5ef05d6b3b7c>@@$$QEAV<lambda_f7424dd8d45958661754dc4f2697e9c3>@@@Z 000000018000fb34 f i libucrt:mbctype.obj
 0001:0000f230       __acrt_initialize_multibyte 0000000180010230 f   libucrt:mbctype.obj
 0001:0000f258       __acrt_update_thread_multibyte_data 0000000180010258 f   libucrt:mbctype.obj
 0001:0000f318       _setmbcp_nolock            0000000180010318 f   libucrt:mbctype.obj
 0001:0000f638       _ismbblead                 0000000180010638 f   libucrt:ismbbyte.obj
 0001:0000f64c       __acrt_initialize_command_line 000000018001064c f   libucrt:argv_data.obj
 0001:0000f674       __dcrt_get_narrow_environment_from_os 0000000180010674 f   libucrt:get_environment_from_os.obj
 0001:0000f778       _recalloc                  0000000180010778 f   libucrt:recalloc.obj
 0001:0000f780       _recalloc_base             0000000180010780 f   libucrt:recalloc.obj
 0001:0000f818       __acrt_initialize_heap     0000000180010818 f   libucrt:heap_handle.obj
 0001:0000f834       __acrt_uninitialize_heap   0000000180010834 f   libucrt:heap_handle.obj
 0001:0000fa28       __acrt_initialize_lowio    0000000180010a28 f   libucrt:ioinit.obj
 0001:0000fa64       __acrt_uninitialize_lowio  0000000180010a64 f   libucrt:ioinit.obj
 0001:0000faa4       __acrt_execute_initializers 0000000180010aa4 f   libucrt:shared_initialization.obj
 0001:0000fb38       __acrt_execute_uninitializers 0000000180010b38 f   libucrt:shared_initialization.obj
 0001:0000fb88       ??$?RV<lambda_c36588078e9f5dfd39652860aa6b3aaf>@@AEAV<lambda_ec61778202f4f5fc7e7711acc23c3bca>@@V<lambda_dc9d2797ccde5d239b4a0efae8ebd7db>@@@?$__crt_seh_guarded_call@P6AXH@Z@@QEAAP6AXH@Z$$QEAV<lambda_c36588078e9f5dfd39652860aa6b3aaf>@@AEAV<lambda_ec61778202f4f5fc7e7711acc23c3bca>@@$$QEAV<lambda_dc9d2797ccde5d239b4a0efae8ebd7db>@@@Z 0000000180010b88 f i libucrt:signal.obj
 0001:0000fbd0       __acrt_get_sigabrt_handler 0000000180010bd0 f   libucrt:signal.obj
 0001:0000fc00       __acrt_initialize_signal_handlers 0000000180010c00 f   libucrt:signal.obj
 0001:0000fc20       raise                      0000000180010c20 f   libucrt:signal.obj
 0001:0000febc       __acrt_has_user_matherr    0000000180010ebc f   libucrt:matherr.obj
 0001:0000fedc       __acrt_initialize_user_matherr 0000000180010edc f   libucrt:matherr.obj
 0001:0000fee4       __acrt_invoke_user_matherr 0000000180010ee4 f   libucrt:matherr.obj
 0001:0000ff2c       _query_new_mode            0000000180010f2c f   libucrt:new_mode.obj
 0001:0000ff34       _mbtowc_l                  0000000180010f34 f   libucrt:mbtowc.obj
 0001:0001007c       mbtowc                     000000018001107c f   libucrt:mbtowc.obj
 0001:00010084       _fileno                    0000000180011084 f   libucrt:fileno.obj
 0001:000100ac       __acrt_initialize_stdio    00000001800110ac f   libucrt:_file.obj
 0001:000101cc       __acrt_uninitialize_stdio  00000001800111cc f   libucrt:_file.obj
 0001:00010228       _lock_file                 0000000180011228 f   libucrt:_file.obj
 0001:00010234       _unlock_file               0000000180011234 f   libucrt:_file.obj
 0001:00010240       __pctype_func              0000000180011240 f   libucrt:ctype.obj
 0001:00010270       __acrt_add_locale_ref      0000000180011270 f   libucrt:locale_refcounting.obj
 0001:000102fc       __acrt_free_locale         00000001800112fc f   libucrt:locale_refcounting.obj
 0001:00010474       __acrt_locale_add_lc_time_reference 0000000180011474 f   libucrt:locale_refcounting.obj
 0001:0001049c       __acrt_locale_free_lc_time_if_unreferenced 000000018001149c f   libucrt:locale_refcounting.obj
 0001:000104d4       __acrt_locale_release_lc_time_reference 00000001800114d4 f   libucrt:locale_refcounting.obj
 0001:000104fc       __acrt_release_locale_ref  00000001800114fc f   libucrt:locale_refcounting.obj
 0001:000105a4       __acrt_update_thread_locale_data 00000001800115a4 f   libucrt:locale_refcounting.obj
 0001:00010614       _updatetlocinfoEx_nolock   0000000180011614 f   libucrt:locale_refcounting.obj
 0001:0001067c       __acrt_locale_free_monetary 000000018001167c f   libucrt:initmon.obj
 0001:00010788       __acrt_locale_free_numeric 0000000180011788 f   libucrt:initnum.obj
 0001:0001084c       __acrt_locale_free_time    000000018001184c f   libucrt:inittime.obj
 0001:00010954       __acrt_GetStringTypeA      0000000180011954 f   libucrt:getstringtypea.obj
 0001:00010bd0       __acrt_DownlevelLocaleNameToLCID 0000000180011bd0 f   libucrt:lcidtoname_downlevel.obj
 0001:00010ce0       qsort                      0000000180011ce0 f   libucrt:qsort.obj
 0001:00011014       strncpy_s                  0000000180012014 f   libucrt:strncpy_s.obj
 0001:000110e8       strpbrk                    00000001800120e8 f   libucrt:strpbrk.obj
 0001:00011188       _mbsdec                    0000000180012188 f   libucrt:mbsdec.obj
 0001:00011190       _mbsdec_l                  0000000180012190 f   libucrt:mbsdec.obj
 0001:0001159c       __acrt_LCMapStringA        000000018001259c f   libucrt:lcmapstringa.obj
 0001:00011634       _msize                     0000000180012634 f   libucrt:msize.obj
 0001:00011670       _realloc_base              0000000180012670 f   libucrt:realloc_base.obj
 0001:000116f4       __acrt_lowio_create_handle_array 00000001800126f4 f   libucrt:osfinfo.obj
 0001:0001178c       __acrt_lowio_destroy_handle_array 000000018001278c f   libucrt:osfinfo.obj
 0001:000117dc       __acrt_lowio_ensure_fh_exists 00000001800127dc f   libucrt:osfinfo.obj
 0001:00011894       __acrt_lowio_lock_fh       0000000180012894 f   libucrt:osfinfo.obj
 0001:000118b8       __acrt_lowio_unlock_fh     00000001800128b8 f   libucrt:osfinfo.obj
 0001:000118dc       _free_osfhnd               00000001800128dc f   libucrt:osfinfo.obj
 0001:00011998       _get_osfhandle             0000000180012998 f   libucrt:osfinfo.obj
 0001:00011a10       _isatty                    0000000180012a10 f   libucrt:isatty.obj
 0001:00011a70       __acrt_stdio_flush_nolock  0000000180012a70 f   libucrt:fflush.obj
 0001:00011ae8       _fflush_nolock             0000000180012ae8 f   libucrt:fflush.obj
 0001:00011b34       _flushall                  0000000180012b34 f   libucrt:fflush.obj
 0001:00011c24       _fcloseall                 0000000180012c24 f   libucrt:closeall.obj
 0001:00011cd8       __acrt_stdio_free_buffer_nolock 0000000180012cd8 f   libucrt:_freebuf.obj
 0001:00011d18       __strncnt                  0000000180012d18 f   libucrt:strncnt.obj
 0001:00011d30       _query_app_type            0000000180012d30 f   libucrt:report_runtime_error.obj
 0001:00011d38       ??$?RV<lambda_b521505b218e5242e90febf6bfebc422>@@AEAV<lambda_6978c1fb23f02e42e1d9e99668cc68aa>@@V<lambda_314360699dd331753a4119843814e9a7>@@@?$__crt_seh_guarded_call@H@@QEAAH$$QEAV<lambda_b521505b218e5242e90febf6bfebc422>@@AEAV<lambda_6978c1fb23f02e42e1d9e99668cc68aa>@@$$QEAV<lambda_314360699dd331753a4119843814e9a7>@@@Z 0000000180012d38 f i libucrt:commit.obj
 0001:00011dc4       _commit                    0000000180012dc4 f   libucrt:commit.obj
 0001:000123f8       _write                     00000001800133f8 f   libucrt:write.obj
 0001:000124e4       _write_nolock              00000001800134e4 f   libucrt:write.obj
 0001:000127d0       log10                      00000001800137d0 f   libucrt:log10.obj
 0001:00012e18       _lseeki64_nolock           0000000180013e18 f   libucrt:lseek.obj
 0001:00012e20       _fclose_nolock             0000000180013e20 f   libucrt:fclose.obj
 0001:00012ea4       fclose                     0000000180013ea4 f   libucrt:fclose.obj
 0001:00012f10       _putwch_nolock             0000000180013f10 f   libucrt:putwch.obj
 0001:00013090       _handle_error              0000000180014090 f   libucrt:libm_error.obj
 0001:000131c0       __acrt_initialize_fma3     00000001800141c0 f   libucrt:fma3_available.obj
 0001:00013230       _log10_special             0000000180014230 f   libucrt:log_special.obj
 0001:000132e8       ??$?RV<lambda_bfedae4ebbf01fab1bb6dcc6a9e276e0>@@AEAV<lambda_2fe9b910cf3cbf4a0ab98a02ba45b3ec>@@V<lambda_237c231691f317818eb88cc1d5d642d6>@@@?$__crt_seh_guarded_call@H@@QEAAH$$QEAV<lambda_bfedae4ebbf01fab1bb6dcc6a9e276e0>@@AEAV<lambda_2fe9b910cf3cbf4a0ab98a02ba45b3ec>@@$$QEAV<lambda_237c231691f317818eb88cc1d5d642d6>@@@Z 00000001800142e8 f i libucrt:close.obj
 0001:0001335c       _close                     000000018001435c f   libucrt:close.obj
 0001:00013400       _close_nolock              0000000180014400 f   libucrt:close.obj
 0001:000134bc       ?__acrt_stdio_free_stream@@YAXV__crt_stdio_stream@@@Z 00000001800144bc f   libucrt:stream.obj
 0001:00013500       __dcrt_lowio_initialize_console_output 0000000180014500 f   libucrt:initcon.obj
 0001:0001353c       __dcrt_terminate_console_output 000000018001453c f   libucrt:initcon.obj
 0001:00013570       _get_fpsr                  0000000180014570 f   libucrt:fpsr.obj
 0001:00013580       _set_fpsr                  0000000180014580 f   libucrt:fpsr.obj
 0001:0001358a       _fclrf                     000000018001458a f   libucrt:fpsr.obj
 0001:0001359e       _frnd                      000000018001459e f   libucrt:fpsr.obj
 0001:000135c0       _raise_exc                 00000001800145c0 f   libucrt:fpexcept.obj
 0001:000135e8       _raise_exc_ex              00000001800145e8 f   libucrt:fpexcept.obj
 0001:000138f0       _set_errno_from_matherr    00000001800148f0 f   libucrt:fpexcept.obj
 0001:00013920       _clrfp                     0000000180014920 f   libucrt:fpctrl.obj
 0001:00013940       _ctrlfp                    0000000180014940 f   libucrt:fpctrl.obj
 0001:000139bc       _set_statfp                00000001800149bc f   libucrt:fpctrl.obj
 0001:000139dc       _statfp                    00000001800149dc f   libucrt:fpctrl.obj
 0001:000139ee       IsProcessorFeaturePresent  00000001800149ee f   kernel32:KERNEL32.dll
 0001:000139f4       RtlUnwindEx                00000001800149f4 f   kernel32:KERNEL32.dll
 0001:000139fa       SystemFunction036          00000001800149fa f   advapi32:ADVAPI32.dll
 0001:00013a00       __GSHandlerCheck           0000000180014a00 f   LIBCMT:_gshandler_.obj
 0001:00013a20       __GSHandlerCheckCommon     0000000180014a20 f   LIBCMT:_gshandler_.obj
 0001:00013a90       __security_check_cookie    0000000180014a90 f   LIBCMT:_amdsecgs_.obj
 0001:00013ac0       _FindPESection             0000000180014ac0 f   LIBCMT:pesect.obj
 0001:00013b10       _IsNonwritableInCurrentImage 0000000180014b10 f   LIBCMT:pesect.obj
 0001:00013b60       _ValidateImageBase         0000000180014b60 f   LIBCMT:pesect.obj
 0001:00013b90       __raise_securityfailure    0000000180014b90 f   LIBCMT:gs_report.obj
 0001:00013bc4       __report_gsfailure         0000000180014bc4 f   LIBCMT:gs_report.obj
 0001:00013c98       __report_rangecheckfailure 0000000180014c98 f   LIBCMT:gs_report.obj
 0001:00013cac       __report_securityfailure   0000000180014cac f   LIBCMT:gs_report.obj
 0001:00013e40       memcpy                     0000000180014e40 f   libvcruntime:memcpy.obj
 0001:00013e40       memmove                    0000000180014e40 f   libvcruntime:memcpy.obj
 0001:00014290       memcmp                     0000000180015290 f   libvcruntime:memcmp.obj
 0001:00014370       _guard_dispatch_icall_nop  0000000180015370 f   LIBCMT:_guard_dispatch_.obj
 0001:00015218       _TI2?AVbad_alloc@std@@     0000000180016218     LIBCMT:throw_bad_alloc.obj
 0001:00015238       _CTA2?AVbad_alloc@std@@    0000000180016238     LIBCMT:throw_bad_alloc.obj
 0001:00015250       _CT??_R0?AVbad_alloc@std@@@8??0bad_alloc@std@@QEAA@AEBV01@@Z24 0000000180016250     LIBCMT:throw_bad_alloc.obj
 0001:00015278       _CT??_R0?AVexception@std@@@8??0exception@std@@QEAA@AEBV01@@Z24 0000000180016278     LIBCMT:throw_bad_alloc.obj
 0001:000152a0       _TI3?AVbad_array_new_length@std@@ 00000001800162a0     LIBCMT:throw_bad_alloc.obj
 0001:000152c0       _CTA3?AVbad_array_new_length@std@@ 00000001800162c0     LIBCMT:throw_bad_alloc.obj
 0001:000152e0       _CT??_R0?AVbad_array_new_length@std@@@8??0bad_array_new_length@std@@QEAA@AEBV01@@Z24 00000001800162e0     LIBCMT:throw_bad_alloc.obj
 0002:00000000       __scrt_native_dllmain_reason 0000000180017000     LIBCMT:utility.obj
 0002:00000008       __isa_available            0000000180017008     LIBCMT:_cpu_disp_.obj
 0002:0000000c       __isa_enabled              000000018001700c     LIBCMT:_cpu_disp_.obj
 0002:00000010       __memcpy_nt_iters          0000000180017010     LIBCMT:_cpu_disp_.obj
 0002:00000018       __security_cookie          0000000180017018     LIBCMT:gs_cookie.obj
 0002:00000020       __security_cookie_complement 0000000180017020     LIBCMT:gs_cookie.obj
 0002:00000084       __abort_behavior           0000000180017084     libucrt:abort.obj
 0002:00000090       __acrt_initial_locale_data 0000000180017090     libucrt:nlsdata.obj
 0002:000001e8       __acrt_initial_locale_pointers 00000001800171e8     libucrt:nlsdata.obj
 0002:000001f8       __acrt_wide_c_locale_string 00000001800171f8     libucrt:nlsdata.obj
 0002:00000210       __acrt_initial_multibyte_data 0000000180017210     libucrt:mbctype.obj
 0002:00000438       __acrt_current_multibyte_data 0000000180017438     libucrt:mbctype.obj
 0002:00000540       _mbctype                   0000000180017540     libucrt:mbctype.obj
 0002:00000650       _mbcasemap                 0000000180017650     libucrt:mbctype.obj
 0002:00000750       _iob                       0000000180017750     libucrt:_file.obj
 0002:00000858       _pwctype                   0000000180017858     libucrt:ctype.obj
 0002:00000860       __globallocalestatus       0000000180017860     libucrt:glstatus.obj
 0002:00000870       __acrt_lconv_c             0000000180017870     libucrt:localeconv.obj
 0002:00000908       __acrt_lconv_static_decimal 0000000180017908     libucrt:localeconv.obj
 0002:0000090c       __acrt_lconv_static_W_decimal 000000018001790c     libucrt:localeconv.obj
 0002:00000910       __dcrt_lowio_console_output_handle 0000000180017910     libucrt:initcon.obj
 0002:00000930       _fltused                   0000000180017930     LIBCMT:fltused.obj
 0002:00000940       ??_R0?AVbad_alloc@std@@@8  0000000180017940     LIBCMT:throw_bad_alloc.obj
 0002:00000968       ??_R0?AVexception@std@@@8  0000000180017968     LIBCMT:throw_bad_alloc.obj
 0002:00000990       ??_R0?AVbad_array_new_length@std@@@8 0000000180017990     LIBCMT:throw_bad_alloc.obj
 0002:000009c0       ??_R0?AVtype_info@@@8      00000001800179c0     LIBCMT:std_type_info_static.obj
 0002:000009e0       ?Opt@@3UOptions@@A         00000001800179e0     AutoWrap.obj
 0002:00001490       __scrt_current_native_startup_state 0000000180018490     LIBCMT:utility.obj
 0002:00001498       __scrt_native_startup_lock 0000000180018498     LIBCMT:utility.obj
 0002:000014e0       ?__type_info_root_node@@3U__type_info_node@@A 00000001800184e0     LIBCMT:tncleanup.obj
 0002:000014f0       ?_OptionsStorage@?1??__local_stdio_printf_options@@9@4_KA 00000001800184f0     LIBCMT:default_local_stdio_options.obj
 0002:000014f8       ?_OptionsStorage@?1??__local_stdio_scanf_options@@9@4_KA 00000001800184f8     LIBCMT:default_local_stdio_options.obj
 0002:00001500       __scrt_debugger_hook_flag  0000000180018500     LIBCMT:utility_desktop.obj
 0002:00001504       __favor                    0000000180018504     LIBCMT:_cpu_disp_.obj
 0002:00001628       __pPurecall                0000000180018628     libvcruntime:purevirt_data.obj
 0002:00001630       ?pArgList@UnDecorator@@0PEAVReplicator@@EA 0000000180018630     libvcruntime:undname.obj
 0002:00001638       ?pZNameList@UnDecorator@@0PEAVReplicator@@EA 0000000180018638     libvcruntime:undname.obj
 0002:00001640       ?pTemplateArgList@UnDecorator@@0PEAVReplicator@@EA 0000000180018640     libvcruntime:undname.obj
 0002:00001648       ?gName@UnDecorator@@0PEBDEB 0000000180018648     libvcruntime:undname.obj
 0002:00001650       ?name@UnDecorator@@0PEBDEB 0000000180018650     libvcruntime:undname.obj
 0002:00001658       ?outputString@UnDecorator@@0PEADEA 0000000180018658     libvcruntime:undname.obj
 0002:00001660       ?maxStringLength@UnDecorator@@0HA 0000000180018660     libvcruntime:undname.obj
 0002:00001664       ?disableFlags@UnDecorator@@0KA 0000000180018664     libvcruntime:undname.obj
 0002:00001668       ?fExplicitTemplateParams@UnDecorator@@0_NA 0000000180018668     libvcruntime:undname.obj
 0002:00001669       ?fGetTemplateArgumentList@UnDecorator@@0_NA 0000000180018669     libvcruntime:undname.obj
 0002:00001670       ?m_pGetParameter@UnDecorator@@0P6APEADJ@ZEA 0000000180018670     libvcruntime:undname.obj
 0002:000017c8       _environ_table             00000001800187c8     libucrt:environment_initialization.obj
 0002:000017d0       _wenviron_table            00000001800187d0     libucrt:environment_initialization.obj
 0002:000017d8       __dcrt_initial_wide_environment 00000001800187d8     libucrt:environment_initialization.obj
 0002:000017e0       __dcrt_initial_narrow_environment 00000001800187e0     libucrt:environment_initialization.obj
 0002:000017e8       __acrt_atexit_table        00000001800187e8     libucrt:onexit.obj
 0002:00001800       __acrt_at_quick_exit_table 0000000180018800     libucrt:onexit.obj
 0002:00001818       __acrt_locale_changed_data 0000000180018818     libucrt:wsetlocale.obj
 0002:00001820       __acrt_current_locale_data 0000000180018820     libucrt:nlsdata.obj
 0002:00001bf0       __mbcodepage               0000000180018bf0     libucrt:mbctype.obj
 0002:00001bf4       __ismbcodepage             0000000180018bf4     libucrt:mbctype.obj
 0002:00001bf8       __mbulinfo                 0000000180018bf8     libucrt:mbctype.obj
 0002:00001c08       __mblocalename             0000000180018c08     libucrt:mbctype.obj
 0002:00001c14       __argc                     0000000180018c14     libucrt:argv_data.obj
 0002:00001c18       __argv                     0000000180018c18     libucrt:argv_data.obj
 0002:00001c20       __wargv                    0000000180018c20     libucrt:argv_data.obj
 0002:00001c28       _acmdln                    0000000180018c28     libucrt:argv_data.obj
 0002:00001c30       _wcmdln                    0000000180018c30     libucrt:argv_data.obj
 0002:00001c38       _pgmptr                    0000000180018c38     libucrt:argv_data.obj
 0002:00001c40       __acrt_heap                0000000180018c40     libucrt:heap_handle.obj
 0002:00001c50       __pioinfo                  0000000180018c50     libucrt:ioinit.obj
 0002:00002050       _nhandle                   0000000180019050     libucrt:ioinit.obj
 0002:00002080       __acrt_stdout_buffer       0000000180019080     libucrt:_sftbuf.obj
 0002:00002088       __acrt_stderr_buffer       0000000180019088     libucrt:_sftbuf.obj
 0002:00002098       _nstream                   0000000180019098     libucrt:_file.obj
 0002:000020a0       __piob                     00000001800190a0     libucrt:_file.obj
 0002:000020a8       __acrt_lconv_static_null   00000001800190a8     libucrt:localeconv.obj
 0002:000020ac       __acrt_lconv_static_W_null 00000001800190ac     libucrt:localeconv.obj
 0002:000020b4       __fma3_is_available        00000001800190b4     libucrt:fma3_available.obj
 0002:000020b8       __use_fma3_lib             00000001800190b8     libucrt:fma3_available.obj
 0002:00002630       __scrt_ucrt_dll_is_in_use  0000000180019630     <common>
 0002:00002638       __dyn_tls_init_callback    0000000180019638     <common>
 0002:00002640       _pDestructExceptionObject  0000000180019640     <common>
 0004:00000000       __imp_SystemFunction036    000000018001b000     advapi32:ADVAPI32.dll
 0004:00000008       \177ADVAPI32_NULL_THUNK_DATA 000000018001b008     advapi32:ADVAPI32.dll
 0004:00000010       __imp_QueryPerformanceCounter 000000018001b010     kernel32:KERNEL32.dll
 0004:00000018       __imp_GetCurrentProcessId  000000018001b018     kernel32:KERNEL32.dll
 0004:00000020       __imp_GetCurrentThreadId   000000018001b020     kernel32:KERNEL32.dll
 0004:00000028       __imp_GetSystemTimeAsFileTime 000000018001b028     kernel32:KERNEL32.dll
 0004:00000030       __imp_InitializeSListHead  000000018001b030     kernel32:KERNEL32.dll
 0004:00000038       __imp_RtlCaptureContext    000000018001b038     kernel32:KERNEL32.dll
 0004:00000040       __imp_RtlLookupFunctionEntry 000000018001b040     kernel32:KERNEL32.dll
 0004:00000048       __imp_RtlVirtualUnwind     000000018001b048     kernel32:KERNEL32.dll
 0004:00000050       __imp_IsDebuggerPresent    000000018001b050     kernel32:KERNEL32.dll
 0004:00000058       __imp_UnhandledExceptionFilter 000000018001b058     kernel32:KERNEL32.dll
 0004:00000060       __imp_SetUnhandledExceptionFilter 000000018001b060     kernel32:KERNEL32.dll
 0004:00000068       __imp_GetStartupInfoW      000000018001b068     kernel32:KERNEL32.dll
 0004:00000070       __imp_IsProcessorFeaturePresent 000000018001b070     kernel32:KERNEL32.dll
 0004:00000078       __imp_GetModuleHandleW     000000018001b078     kernel32:KERNEL32.dll
 0004:00000080       __imp_GetLastError         000000018001b080     kernel32:KERNEL32.dll
 0004:00000088       __imp_GetModuleFileNameW   000000018001b088     kernel32:KERNEL32.dll
 0004:00000090       __imp_RtlUnwindEx          000000018001b090     kernel32:KERNEL32.dll
 0004:00000098       __imp_RtlPcToFileHeader    000000018001b098     kernel32:KERNEL32.dll
 0004:000000a0       __imp_RaiseException       000000018001b0a0     kernel32:KERNEL32.dll
 0004:000000a8       __imp_InterlockedFlushSList 000000018001b0a8     kernel32:KERNEL32.dll
 0004:000000b0       __imp_InitializeCriticalSectionAndSpinCount 000000018001b0b0     kernel32:KERNEL32.dll
 0004:000000b8       __imp_TlsAlloc             000000018001b0b8     kernel32:KERNEL32.dll
 0004:000000c0       __imp_TlsGetValue          000000018001b0c0     kernel32:KERNEL32.dll
 0004:000000c8       __imp_TlsSetValue          000000018001b0c8     kernel32:KERNEL32.dll
 0004:000000d0       __imp_TlsFree              000000018001b0d0     kernel32:KERNEL32.dll
 0004:000000d8       __imp_FreeLibrary          000000018001b0d8     kernel32:KERNEL32.dll
 0004:000000e0       __imp_GetProcAddress       000000018001b0e0     kernel32:KERNEL32.dll
 0004:000000e8       __imp_LoadLibraryExW       000000018001b0e8     kernel32:KERNEL32.dll
 0004:000000f0       __imp_SetLastError         000000018001b0f0     kernel32:KERNEL32.dll
 0004:000000f8       __imp_EnterCriticalSection 000000018001b0f8     kernel32:KERNEL32.dll
 0004:00000100       __imp_LeaveCriticalSection 000000018001b100     kernel32:KERNEL32.dll
 0004:00000108       __imp_DeleteCriticalSection 000000018001b108     kernel32:KERNEL32.dll
 0004:00000110       __imp_GetCurrentProcess    000000018001b110     kernel32:KERNEL32.dll
 0004:00000118       __imp_ExitProcess          000000018001b118     kernel32:KERNEL32.dll
 0004:00000120       __imp_TerminateProcess     000000018001b120     kernel32:KERNEL32.dll
 0004:00000128       __imp_GetModuleHandleExW   000000018001b128     kernel32:KERNEL32.dll
 0004:00000130       __imp_GetModuleFileNameA   000000018001b130     kernel32:KERNEL32.dll
 0004:00000138       __imp_MultiByteToWideChar  000000018001b138     kernel32:KERNEL32.dll
 0004:00000140       __imp_WideCharToMultiByte  000000018001b140     kernel32:KERNEL32.dll
 0004:00000148       __imp_HeapFree             000000018001b148     kernel32:KERNEL32.dll
 0004:00000150       __imp_HeapAlloc            000000018001b150     kernel32:KERNEL32.dll
 0004:00000158       __imp_lstrlenW             000000018001b158     kernel32:KERNEL32.dll
 0004:00000160       __imp_GetACP               000000018001b160     kernel32:KERNEL32.dll
 0004:00000168       __imp_LCMapStringW         000000018001b168     kernel32:KERNEL32.dll
 0004:00000170       __imp_FindClose            000000018001b170     kernel32:KERNEL32.dll
 0004:00000178       __imp_FindFirstFileExA     000000018001b178     kernel32:KERNEL32.dll
 0004:00000180       __imp_FindNextFileA        000000018001b180     kernel32:KERNEL32.dll
 0004:00000188       __imp_IsValidCodePage      000000018001b188     kernel32:KERNEL32.dll
 0004:00000190       __imp_GetOEMCP             000000018001b190     kernel32:KERNEL32.dll
 0004:00000198       __imp_GetCPInfo            000000018001b198     kernel32:KERNEL32.dll
 0004:000001a0       __imp_GetCommandLineA      000000018001b1a0     kernel32:KERNEL32.dll
 0004:000001a8       __imp_GetCommandLineW      000000018001b1a8     kernel32:KERNEL32.dll
 0004:000001b0       __imp_GetEnvironmentStringsW 000000018001b1b0     kernel32:KERNEL32.dll
 0004:000001b8       __imp_FreeEnvironmentStringsW 000000018001b1b8     kernel32:KERNEL32.dll
 0004:000001c0       __imp_GetProcessHeap       000000018001b1c0     kernel32:KERNEL32.dll
 0004:000001c8       __imp_GetStdHandle         000000018001b1c8     kernel32:KERNEL32.dll
 0004:000001d0       __imp_GetFileType          000000018001b1d0     kernel32:KERNEL32.dll
 0004:000001d8       __imp_HeapSize             000000018001b1d8     kernel32:KERNEL32.dll
 0004:000001e0       __imp_HeapReAlloc          000000018001b1e0     kernel32:KERNEL32.dll
 0004:000001e8       __imp_SetStdHandle         000000018001b1e8     kernel32:KERNEL32.dll
 0004:000001f0       __imp_WriteFile            000000018001b1f0     kernel32:KERNEL32.dll
 0004:000001f8       __imp_FlushFileBuffers     000000018001b1f8     kernel32:KERNEL32.dll
 0004:00000200       __imp_GetConsoleCP         000000018001b200     kernel32:KERNEL32.dll
 0004:00000208       __imp_GetConsoleMode       000000018001b208     kernel32:KERNEL32.dll
 0004:00000210       __imp_SetFilePointerEx     000000018001b210     kernel32:KERNEL32.dll
 0004:00000218       __imp_CloseHandle          000000018001b218     kernel32:KERNEL32.dll
 0004:00000220       __imp_WriteConsoleW        000000018001b220     kernel32:KERNEL32.dll
 0004:00000228       __imp_CreateFileW          000000018001b228     kernel32:KERNEL32.dll
 0004:00000230       __imp_GetStringTypeW       000000018001b230     kernel32:KERNEL32.dll
 0004:00000238       __imp_lstrcpynW            000000018001b238     kernel32:KERNEL32.dll
 0004:00000240       \177KERNEL32_NULL_THUNK_DATA 000000018001b240     kernel32:KERNEL32.dll
 0004:00000248       __IMPORT_DESCRIPTOR_KERNEL32 000000018001b248     kernel32:KERNEL32.dll
 0004:0000025c       __IMPORT_DESCRIPTOR_ADVAPI32 000000018001b25c     advapi32:ADVAPI32.dll
 0004:00000270       __NULL_IMPORT_DESCRIPTOR   000000018001b270     kernel32:KERNEL32.dll

 entry point at        0001:0000a4b8

 Static symbols

 0001:000003a0       ?ExceptionTemplate@?1??_CxxThrowException@@9@4UEHExceptionRecord@@B 00000001800013a0     libvcruntime:throw.obj
 0001:000003e0       ?module_names@?A0x49c8dc86@@3QBQEB_WB 00000001800013e0     libvcruntime:winapi_downlevel.obj
 0001:000004ac       ?candidate_modules@?1??try_get_EventRegister@@YAP6AKPEBU_GUID@@P6AX0KE_K1PEAU_EVENT_FILTER_DESCRIPTOR@@PEAX@Z3PEA_K@ZXZ@4QBW4module_id@?A0x49c8dc86@@B 00000001800014ac     libvcruntime:winapi_downlevel.obj
 0001:000004c0       ?candidate_modules@?1??try_get_EventSetInformation@@YAP6AK_KW4_EVENT_INFO_CLASS@@PEAXK@ZXZ@4QBW4module_id@?A0x49c8dc86@@B 00000001800014c0     libvcruntime:winapi_downlevel.obj
 0001:000004dc       ?candidate_modules@?1??try_get_EventUnregister@@YAP6AK_K@ZXZ@4QBW4module_id@?A0x49c8dc86@@B 00000001800014dc     libvcruntime:winapi_downlevel.obj
 0001:000004f0       ?candidate_modules@?1??try_get_EventWriteTransfer@@YAP6AK_KPEBU_EVENT_DESCRIPTOR@@PEBU_GUID@@2KPEAU_EVENT_DATA_DESCRIPTOR@@@ZXZ@4QBW4module_id@?A0x49c8dc86@@B 00000001800014f0     libvcruntime:winapi_downlevel.obj
 0001:00000510       ?candidate_modules@?1??try_get_FlsAlloc@@YAP6AKP6AXPEAX@Z@ZXZ@4QBW4module_id@?A0x49c8dc86@@B 0000000180001510     libvcruntime:winapi_downlevel.obj
 0001:00000528       ?candidate_modules@?1??try_get_FlsFree@@YAP6AHK@ZXZ@4QBW4module_id@?A0x49c8dc86@@B 0000000180001528     libvcruntime:winapi_downlevel.obj
 0001:00000538       ?candidate_modules@?1??try_get_FlsGetValue@@YAP6APEAXK@ZXZ@4QBW4module_id@?A0x49c8dc86@@B 0000000180001538     libvcruntime:winapi_downlevel.obj
 0001:00000550       ?candidate_modules@?1??try_get_FlsSetValue@@YAP6AHKPEAX@ZXZ@4QBW4module_id@?A0x49c8dc86@@B 0000000180001550     libvcruntime:winapi_downlevel.obj
 0001:00000568       ?candidate_modules@?1??try_get_InitializeCriticalSectionEx@@YAP6AHPEAU_RTL_CRITICAL_SECTION@@KK@ZXZ@4QBW4module_id@?A0x49c8dc86@@B 0000000180001568     libvcruntime:winapi_downlevel.obj
 0001:00000590       ?tokenTable@@3QBQEBDB      0000000180001590     libvcruntime:undname.obj
 0001:00000600       ?nameTable@@3QBQEBDB       0000000180001600     libvcruntime:undname.obj
 0001:00000888       ?rttiTable@@3QBQEBDB       0000000180001888     libvcruntime:undname.obj
 0001:00001010       __acrt_initializers        0000000180002010     libucrt:initialization.obj
 0001:00001780       module_names               0000000180002780     libucrt:winapi_thunks.obj
 0001:00001cb0       ?candidate_modules@?1??try_get_FlsAlloc@@YAP6AKP6AXPEAX@Z@ZXZ@4QBW4module_id@?A0x63058377@@B 0000000180002cb0     libucrt:winapi_thunks.obj
 0001:00001cb8       ?candidate_modules@?1??try_get_FlsFree@@YAP6AHK@ZXZ@4QBW4module_id@?A0x63058377@@B 0000000180002cb8     libucrt:winapi_thunks.obj
 0001:00001cc0       ?candidate_modules@?1??try_get_FlsGetValue@@YAP6APEAXK@ZXZ@4QBW4module_id@?A0x63058377@@B 0000000180002cc0     libucrt:winapi_thunks.obj
 0001:00001cc8       ?candidate_modules@?1??try_get_FlsSetValue@@YAP6AHKPEAX@ZXZ@4QBW4module_id@?A0x63058377@@B 0000000180002cc8     libucrt:winapi_thunks.obj
 0001:00001cd0       ?candidate_modules@?1??try_get_GetCurrentPackageId@@YAP6AJPEAIPEAE@ZXZ@4QBW4module_id@?A0x63058377@@B 0000000180002cd0     libucrt:winapi_thunks.obj
 0001:00001cf0       ?candidate_modules@?1??try_get_InitializeCriticalSectionEx@@YAP6AHPEAU_RTL_CRITICAL_SECTION@@KK@ZXZ@4QBW4module_id@?A0x63058377@@B 0000000180002cf0     libucrt:winapi_thunks.obj
 0001:00001cf8       ?candidate_modules@?1??try_get_LCMapStringEx@@YAP6AHPEB_WK0HPEA_WHPEAU_nlsversioninfo@@PEAX_J@ZXZ@4QBW4module_id@?A0x63058377@@B 0000000180002cf8     libucrt:winapi_thunks.obj
 0001:00001d10       ?candidate_modules@?1??try_get_LocaleNameToLCID@@YAP6AKPEB_WK@ZXZ@4QBW4module_id@?A0x63058377@@B 0000000180002d10     libucrt:winapi_thunks.obj
 0001:00001d30       errtable                   0000000180002d30     libucrt:errno.obj
 0001:00001e98       _mb_locale_names           0000000180002e98     libucrt:mbctype.obj
 0001:00002710       LcidToLocaleNameTable      0000000180003710     libucrt:lcidtoname_downlevel.obj
 0001:00004160       LocaleNameToIndexTable     0000000180005160     libucrt:lcidtoname_downlevel.obj
 0001:00005a00       __real_ninf                0000000180006a00     libucrt:log10.obj
 0001:00005a10       __real_inf                 0000000180006a10     libucrt:log10.obj
 0001:00005a20       __real_neg_qnan            0000000180006a20     libucrt:log10.obj
 0001:00005a30       __real_qnanbit             0000000180006a30     libucrt:log10.obj
 0001:00005a40       __int_1023                 0000000180006a40     libucrt:log10.obj
 0001:00005a50       __mask_001                 0000000180006a50     libucrt:log10.obj
 0001:00005a60       __mask_mant                0000000180006a60     libucrt:log10.obj
 0001:00005a70       __mask_mant_top8           0000000180006a70     libucrt:log10.obj
 0001:00005a80       __mask_mant9               0000000180006a80     libucrt:log10.obj
 0001:00005a90       __real_log10_e             0000000180006a90     libucrt:log10.obj
 0001:00005aa0       __real_log10_e_lead        0000000180006aa0     libucrt:log10.obj
 0001:00005ab0       __real_log10_e_tail        0000000180006ab0     libucrt:log10.obj
 0001:00005ac0       __real_log10_2_lead        0000000180006ac0     libucrt:log10.obj
 0001:00005ad0       __real_log10_2_tail        0000000180006ad0     libucrt:log10.obj
 0001:00005ae0       __real_two                 0000000180006ae0     libucrt:log10.obj
 0001:00005af0       __real_one                 0000000180006af0     libucrt:log10.obj
 0001:00005b00       __real_half                0000000180006b00     libucrt:log10.obj
 0001:00005b10       __mask_100                 0000000180006b10     libucrt:log10.obj
 0001:00005b20       __real_1_over_512          0000000180006b20     libucrt:log10.obj
 0001:00005b30       __real_1_over_2            0000000180006b30     libucrt:log10.obj
 0001:00005b40       __real_1_over_3            0000000180006b40     libucrt:log10.obj
 0001:00005b50       __real_1_over_4            0000000180006b50     libucrt:log10.obj
 0001:00005b60       __real_1_over_5            0000000180006b60     libucrt:log10.obj
 0001:00005b70       __real_1_over_6            0000000180006b70     libucrt:log10.obj
 0001:00005b80       __real_neg_1023            0000000180006b80     libucrt:log10.obj
 0001:00005b90       __mask_2045                0000000180006b90     libucrt:log10.obj
 0001:00005ba0       __real_threshold           0000000180006ba0     libucrt:log10.obj
 0001:00005bb0       __real_near_one_lt         0000000180006bb0     libucrt:log10.obj
 0001:00005bc0       __real_near_one_gt         0000000180006bc0     libucrt:log10.obj
 0001:00005bd0       __real_min_norm            0000000180006bd0     libucrt:log10.obj
 0001:00005be0       __real_notsign             0000000180006be0     libucrt:log10.obj
 0001:00005bf0       __real_ca1                 0000000180006bf0     libucrt:log10.obj
 0001:00005c00       __real_ca2                 0000000180006c00     libucrt:log10.obj
 0001:00005c10       __real_ca3                 0000000180006c10     libucrt:log10.obj
 0001:00005c20       __real_ca4                 0000000180006c20     libucrt:log10.obj
 0001:00005c30       __mask_lower               0000000180006c30     libucrt:log10.obj
 0001:00005c40       __flag_x_zero              0000000180006c40     libucrt:log10.obj
 0001:00005c44       __flag_x_neg               0000000180006c44     libucrt:log10.obj
 0001:00005c48       __flag_x_nan               0000000180006c48     libucrt:log10.obj
 0001:000074a0       __real@433fffffffffffff    00000001800084a0     libucrt:fpsr.obj
 0001:000074a8       __real@c33fffffffffffff    00000001800084a8     libucrt:fpsr.obj
 0001:000074b0       GS_ExceptionPointers       00000001800084b0     LIBCMT:gs_report.obj
 0001:00007780       ?_TlgEvent@?3??__telemetry_main_invoke_trigger@@9@4U<unnamed-type-_TlgEvent>@?3??1@YAXQEAUHINSTANCE__@@@Z@B 0000000180008780     libvcruntime:telemetry.obj
 0001:000077bc       ?_TlgEvent@?3??__telemetry_main_return_trigger@@9@4U<unnamed-type-_TlgEvent>@?3??1@YAXQEAUHINSTANCE__@@@Z@B 00000001800087bc     libvcruntime:telemetry.obj
 0001:000077f7       ?_Tlg_Microsoft_CRTProviderProv_Meta@@3U<unnamed-type-_Tlg_Microsoft_CRTProviderProv_Meta>@@B 00000001800087f7     libvcruntime:telemetry.obj
 0001:00007d70       $$000000                   0000000180008d70     chkstk.obj
 0001:00008984       $LN10                      0000000180009984     AutoWrap.obj
 0001:00008ab8       $LN22                      0000000180009ab8     AutoWrap.obj
 0001:000098f0       $LN167                     000000018000a8f0     AutoWrap.obj
 0001:0000a148       ?dllmain_crt_dispatch@@YAHQEAUHINSTANCE__@@KQEAX@Z 000000018000b148 f   LIBCMT:dll_dllmain.obj
 0001:0000a198       ?dllmain_crt_process_attach@@YAHQEAUHINSTANCE__@@QEAX@Z 000000018000b198 f   LIBCMT:dll_dllmain.obj
 0001:0000a2c4       ?dllmain_crt_process_detach@@YAH_N@Z 000000018000b2c4 f   LIBCMT:dll_dllmain.obj
 0001:0000a348       ?dllmain_dispatch@@YAHQEAUHINSTANCE__@@KQEAX@Z 000000018000b348 f   LIBCMT:dll_dllmain.obj
 0001:0000a464       ?dllmain_raw@@YAHQEAUHINSTANCE__@@KQEAX@Z 000000018000b464 f   LIBCMT:dll_dllmain.obj
 0001:0000b000       $$000000                   000000018000c000     libvcruntime:memset.obj
 0001:0000b0ec       MsetTab                    000000018000c0ec     libvcruntime:memset.obj
 0001:0000b1b0       _TlgDefineProvider_annotation__Tlg_Microsoft_CRTProviderProv 000000018000c1b0 f   libvcruntime:telemetry.obj
 0001:0000b86c       ?try_get_function@@YAPEAXW4function_id@?A0x49c8dc86@@QEBDQEBW4module_id@2@2@Z 000000018000c86c f   libvcruntime:winapi_downlevel.obj
 0001:0000be80       $$000000                   000000018000ce80     libvcruntime:_jmpuwind_.obj
 0001:0000c4f4       ?atexit_exception_filter@@YAHK@Z 000000018000d4f4 f   libucrt:exit.obj
 0001:0000c500       ?common_exit@@YAXHW4_crt_exit_cleanup_mode@@W4_crt_exit_return_mode@@@Z 000000018000d500 f   libucrt:exit.obj
 0001:0000c66c       ?exit_or_terminate_process@@YAXI@Z 000000018000d66c f   libucrt:exit.obj
 0001:0000c6b8       ?try_cor_exit_process@@YAXI@Z 000000018000d6b8 f   libucrt:exit.obj
 0001:0000c750       ??$parse_command_line@D@@YAXPEADPEAPEAD0PEA_K2@Z 000000018000d750 f   libucrt:argv_parsing.obj
 0001:0000cae8       ??$common_initialize_environment_nolock@D@@YAHXZ 000000018000dae8 f   libucrt:environment_initialization.obj
 0001:0000cb54       ??$create_environment@D@@YAQEAPEADQEAD@Z 000000018000db54 f   libucrt:environment_initialization.obj
 0001:0000cc50       ??$free_environment@_W@@YAXQEAPEA_W@Z 000000018000dc50 f   libucrt:environment_initialization.obj
 0001:0000cc50       ??$free_environment@D@@YAXQEAPEAD@Z 000000018000dc50 f   libucrt:environment_initialization.obj
 0001:0000cc94       ??$uninitialize_environment_internal@D@@YAXAEAPEAPEAD@Z 000000018000dc94 f   libucrt:environment_initialization.obj
 0001:0000ccb0       ??$uninitialize_environment_internal@_W@@YAXAEAPEAPEA_W@Z 000000018000dcb0 f   libucrt:environment_initialization.obj
 0001:0000cee8       ??R<lambda_4e60a939b0d047cfe11ddc22648dfba9>@@QEBAHXZ 000000018000dee8 f   libucrt:onexit.obj
 0001:0000d198       initialize_global_variables 000000018000e198 f   libucrt:initialization.obj
 0001:0000d1ac       initialize_c               000000018000e1ac f   libucrt:initialization.obj
 0001:0000d1d0       report_memory_leaks        000000018000e1d0 f   libucrt:initialization.obj
 0001:0000d1d0       initialize_environment     000000018000e1d0 f   libucrt:initialization.obj
 0001:0000d1d0       initialize_global_state_isolation 000000018000e1d0 f   libucrt:initialization.obj
 0001:0000d1d0       uninitialize_global_state_isolation 000000018000e1d0 f   libucrt:initialization.obj
 0001:0000d1d0       uninitialize_c             000000018000e1d0 f   libucrt:initialization.obj
 0001:0000d1d4       uninitialize_environment   000000018000e1d4 f   libucrt:initialization.obj
 0001:0000d1e4       initialize_pointers        000000018000e1e4 f   libucrt:initialization.obj
 0001:0000d238       uninitialize_vcruntime     000000018000e238 f   libucrt:initialization.obj
 0001:0000d240       uninitialize_allocated_memory 000000018000e240 f   libucrt:initialization.obj
 0001:0000d6bc       ?construct_ptd_array@@YAXQEAU__acrt_ptd@@@Z 000000018000e6bc f   libucrt:per_thread_data.obj
 0001:0000d78c       ?destroy_fls@@YAXPEAX@Z    000000018000e78c f   libucrt:per_thread_data.obj
 0001:0000d7ac       ?destroy_ptd_array@@YAXQEAU__acrt_ptd@@@Z 000000018000e7ac f   libucrt:per_thread_data.obj
 0001:0000d8a4       ?replace_current_thread_locale_nolock@@YAXQEAU__acrt_ptd@@QEAU__crt_locale_data@@@Z 000000018000e8a4 f   libucrt:per_thread_data.obj
 0001:0000dc58       ?try_get_function@@YAPEAXW4function_id@?A0x63058377@@QEBDQEBW4module_id@2@2@Z 000000018000ec58 f   libucrt:winapi_thunks.obj
 0001:0000e588       ?<helper_func_cdecl>@<lambda_2feae5270eb4d0d5532525f423405775>@@CAHPEBX0@Z 000000018000f588 f   libucrt:argv_wildcards.obj
 0001:0000e59c       ??$common_expand_argv_wildcards@D@@YAHQEAPEADQEAPEAPEAD@Z 000000018000f59c f   libucrt:argv_wildcards.obj
 0001:0000e7a8       ??$copy_and_add_argument_to_buffer@D@@YAHQEBD0_KAEAV?$argument_list@D@?A0xca0879c4@@@Z 000000018000f7a8 f   libucrt:argv_wildcards.obj
 0001:0000e8b8       ??$expand_argument_wildcards@D@@YAHQEAD0AEAV?$argument_list@D@?A0xca0879c4@@@Z 000000018000f8b8 f   libucrt:argv_wildcards.obj
 0001:0000eb6c       ??R<lambda_ad1ced32f4ac17aa236e5ef05d6b3b7c>@@QEBAXXZ 000000018000fb6c f   libucrt:mbctype.obj
 0001:0000ed84       ?getSystemCP@@YAHH@Z       000000018000fd84 f   libucrt:mbctype.obj
 0001:0000ee04       ?setSBCS@@YAXPEAU__crt_multibyte_data@@@Z 000000018000fe04 f   libucrt:mbctype.obj
 0001:0000ee94       ?setSBUpLow@@YAXPEAU__crt_multibyte_data@@@Z 000000018000fe94 f   libucrt:mbctype.obj
 0001:0000f078       ?setmbcp_internal@@YAHH_N@Z 0000000180010078 f   libucrt:mbctype.obj
 0001:0000f5c0       ?x_ismbbtype_l@@YAHPEAU__crt_locale_pointers@@IHH@Z 00000001800105c0 f   libucrt:ismbbyte.obj
 0001:0000f840       ?initialize_inherited_file_handles_nolock@@YAXXZ 0000000180010840 f   libucrt:ioinit.obj
 0001:0000f92c       ?initialize_stdio_handles_nolock@@YAXXZ 000000018001092c f   libucrt:ioinit.obj
 0001:000107f4       ?free_crt_array_internal@@YAXQEAPEBX_K@Z 00000001800117f4 f   libucrt:inittime.obj
 0001:00010b08       ?GetTableIndexFromLocaleName@@YAHPEB_W@Z 0000000180011b08 f   libucrt:lcidtoname_downlevel.obj
 0001:00010c10       ?shortsort@@YAXPEAD0_KP6AHPEBX2@Z@Z 0000000180011c10 f   libucrt:qsort.obj
 0001:00011228       ?initialize_multibyte@@YAHXZ 0000000180012228 f   libucrt:multibyte_initializer.obj
 0001:00011240       ?__acrt_LCMapStringA_stat@@YAHPEAU__crt_locale_pointers@@PEB_WKPEBDHPEADHHH@Z 0000000180012240 f   libucrt:lcmapstringa.obj
 0001:00011b40       common_flush_all           0000000180012b40 f   libucrt:fflush.obj
 0001:00011e58       ?write_double_translated_ansi_nolock@@YA?AUwrite_result@?A0x9c548279@@HQEBDI@Z 0000000180012e58 f   libucrt:write.obj
 0001:00012060       ?write_text_ansi_nolock@@YA?AUwrite_result@?A0x9c548279@@HQEBDI@Z 0000000180013060 f   libucrt:write.obj
 0001:00012168       ?write_text_utf16le_nolock@@YA?AUwrite_result@?A0x9c548279@@HQEBDI@Z 0000000180013168 f   libucrt:write.obj
 0001:00012284       ?write_text_utf8_nolock@@YA?AUwrite_result@?A0x9c548279@@HQEBDI@Z 0000000180013284 f   libucrt:write.obj
 0001:000127d0       $$000000                   00000001800137d0     libucrt:log10.obj
 0001:00012d7c       ??$common_lseek_nolock@_J@@YA_JH_JH@Z 0000000180013d7c f   libucrt:lseek.obj
 0001:00012f6c       _call_matherr              0000000180013f6c f   libucrt:libm_error.obj
 0001:00012fd4       _exception_enabled         0000000180013fd4 f   libucrt:libm_error.obj
 0001:00013250       _log_special_common        0000000180014250 f   libucrt:log_special.obj
 0001:00013560       $$000000                   0000000180014560     libucrt:fpsr.obj
 0001:00013a80       $$000000                   0000000180014a80     LIBCMT:_amdsecgs_.obj
 0001:00013d48       capture_current_context    0000000180014d48 f   LIBCMT:gs_report.obj
 0001:00013db8       capture_previous_context   0000000180014db8 f   LIBCMT:gs_report.obj
 0001:00013e30       $$000000                   0000000180014e30     libvcruntime:memcpy.obj
 0001:00013ed7       MoveSmall                  0000000180014ed7     libvcruntime:memcpy.obj
 0001:00014280       $$000000                   0000000180015280     libvcruntime:memcmp.obj
 0001:00014360       $$000000                   0000000180015360     LIBCMT:_guard_dispatch_.obj
 0001:00014380       ?fin$0@?0??dllmain_crt_process_attach@@YAHQEAUHINSTANCE__@@QEAX@Z@4HA 0000000180015380 f   LIBCMT:dll_dllmain.obj
 0001:00014397       ?fin$0@?0??dllmain_crt_process_detach@@YAH_N@Z@4HA 0000000180015397 f   LIBCMT:dll_dllmain.obj
 0001:000143b3       ?filt$0@?0??dllmain_dispatch@@YAHQEAUHINSTANCE__@@KQEAX@Z@4HA 00000001800153b3 f   LIBCMT:dll_dllmain.obj
 0001:000143e9       __scrt_is_nonwritable_in_current_image$filt$0 00000001800153e9 f   LIBCMT:utility.obj
 0001:00014401       _query_new_handler$fin$0   0000000180015401 f   libucrt:new_handler.obj
 0001:00014417       ?filt$0@?0??common_exit@@YAXHW4_crt_exit_cleanup_mode@@W4_crt_exit_return_mode@@@Z@4HA 0000000180015417 f   libucrt:exit.obj
 0001:00014432       ?fin$1@?0??common_exit@@YAXHW4_crt_exit_cleanup_mode@@W4_crt_exit_return_mode@@@Z@4HA 0000000180015432 f   libucrt:exit.obj
 0001:0001444b       ?fin$0@?0???$?RV<lambda_e24bbb7b643b32fcea6fa61b31d4c984>@@AEAV<lambda_275893d493268fdec8709772e3fcec0e>@@V<lambda_9d71df4d7cf3f480f8d633942495c3b0>@@@?$__crt_seh_guarded_call@H@@QEAAH$$QEAV<lambda_e24bbb7b643b32fcea6fa61b31d4c984>@@AEAV<lambda_275893d493268fdec8709772e3fcec0e>@@$$QEAV<lambda_9d71df4d7cf3f480f8d633942495c3b0>@@@Z@4HA 000000018001544b f   libucrt:onexit.obj
 0001:00014468       __acrt_update_thread_locale_data$fin$0 0000000180015468 f   libucrt:locale_refcounting.obj
 0001:00014468       __acrt_uninitialize_locale$fin$0 0000000180015468 f   libucrt:wsetlocale.obj
 0001:00014481       __acrt_update_thread_multibyte_data$fin$0 0000000180015481 f   libucrt:mbctype.obj
 0001:0001449a       ?fin$0@?0???$?RV<lambda_fb3a7dec4e47f37f22dae91bb15c9095>@@AEAV<lambda_698284760c8add0bfb0756c19673e34b>@@V<lambda_dfb8eca1e75fef3034a8fb18dd509707>@@@?$__crt_seh_guarded_call@X@@QEAAX$$QEAV<lambda_fb3a7dec4e47f37f22dae91bb15c9095>@@AEAV<lambda_698284760c8add0bfb0756c19673e34b>@@$$QEAV<lambda_dfb8eca1e75fef3034a8fb18dd509707>@@@Z@4HA 000000018001549a f   libucrt:per_thread_data.obj
 0001:0001449a       ?fin$0@?0???$?RV<lambda_99476a1ad63dd22509b5d3e65b0ffc95>@@AEAV<lambda_ad1ced32f4ac17aa236e5ef05d6b3b7c>@@V<lambda_f7424dd8d45958661754dc4f2697e9c3>@@@?$__crt_seh_guarded_call@X@@QEAAX$$QEAV<lambda_99476a1ad63dd22509b5d3e65b0ffc95>@@AEAV<lambda_ad1ced32f4ac17aa236e5ef05d6b3b7c>@@$$QEAV<lambda_f7424dd8d45958661754dc4f2697e9c3>@@@Z@4HA 000000018001549a f   libucrt:mbctype.obj
 0001:0001449a       ?fin$0@?0???$?RV<lambda_5e887d1dcbef67a5eb4283622ba103bf>@@AEAV<lambda_4466841279450cc726390878d4a41900>@@V<lambda_341c25c0346d94847f1f3c463c57e077>@@@?$__crt_seh_guarded_call@X@@QEAAX$$QEAV<lambda_5e887d1dcbef67a5eb4283622ba103bf>@@AEAV<lambda_4466841279450cc726390878d4a41900>@@$$QEAV<lambda_341c25c0346d94847f1f3c463c57e077>@@@Z@4HA 000000018001549a f   libucrt:per_thread_data.obj
 0001:0001449a       ?fin$0@?0???$?RV<lambda_46352004c1216016012b18bd6f87e700>@@AEAV<lambda_3bd07e1a1191394380780325891bf33f>@@V<lambda_334532d3f185bcaa59b5be82d7d22bff>@@@?$__crt_seh_guarded_call@X@@QEAAX$$QEAV<lambda_46352004c1216016012b18bd6f87e700>@@AEAV<lambda_3bd07e1a1191394380780325891bf33f>@@$$QEAV<lambda_334532d3f185bcaa59b5be82d7d22bff>@@@Z@4HA 000000018001549a f   libucrt:per_thread_data.obj
 0001:0001449a       ?fin$0@?0???$?RV<lambda_b8c45f8f788dd370798f47cfe8ac3a86>@@AEAV<lambda_4e60a939b0d047cfe11ddc22648dfba9>@@V<lambda_332c3edc96d0294ec56c57d38c1cdfd5>@@@?$__crt_seh_guarded_call@H@@QEAAH$$QEAV<lambda_b8c45f8f788dd370798f47cfe8ac3a86>@@AEAV<lambda_4e60a939b0d047cfe11ddc22648dfba9>@@$$QEAV<lambda_332c3edc96d0294ec56c57d38c1cdfd5>@@@Z@4HA 000000018001549a f   libucrt:onexit.obj
 0001:0001449a       ?fin$0@?0???$?RV<lambda_72d1df2b273a38828b1ce30cbf4cdab5>@@AEAV<lambda_876a65b173b8412d3a47c70a915b0cf4>@@V<lambda_41932305e351933ebe8f8be3ed8bb5dc>@@@?$__crt_seh_guarded_call@X@@QEAAX$$QEAV<lambda_72d1df2b273a38828b1ce30cbf4cdab5>@@AEAV<lambda_876a65b173b8412d3a47c70a915b0cf4>@@$$QEAV<lambda_41932305e351933ebe8f8be3ed8bb5dc>@@@Z@4HA 000000018001549a f   libucrt:per_thread_data.obj
 0001:0001449a       ?fin$0@?0???$?RV<lambda_c36588078e9f5dfd39652860aa6b3aaf>@@AEAV<lambda_ec61778202f4f5fc7e7711acc23c3bca>@@V<lambda_dc9d2797ccde5d239b4a0efae8ebd7db>@@@?$__crt_seh_guarded_call@P6AXH@Z@@QEAAP6AXH@Z$$QEAV<lambda_c36588078e9f5dfd39652860aa6b3aaf>@@AEAV<lambda_ec61778202f4f5fc7e7711acc23c3bca>@@$$QEAV<lambda_dc9d2797ccde5d239b4a0efae8ebd7db>@@@Z@4HA 000000018001549a f   libucrt:signal.obj
 0001:000144b4       raise$fin$0                00000001800154b4 f   libucrt:signal.obj
 0001:000144d8       __acrt_initialize_lowio$fin$0 00000001800154d8 f   libucrt:ioinit.obj
 0001:000144d8       __acrt_lowio_ensure_fh_exists$fin$0 00000001800154d8 f   libucrt:osfinfo.obj
 0001:000144f1       common_flush_all$fin$0     00000001800154f1 f   libucrt:fflush.obj
 0001:0001450b       common_flush_all$fin$1     000000018001550b f   libucrt:fflush.obj
 0001:00014524       _fcloseall$fin$0           0000000180015524 f   libucrt:closeall.obj
 0001:0001453d       ?fin$0@?0???$?RV<lambda_b521505b218e5242e90febf6bfebc422>@@AEAV<lambda_6978c1fb23f02e42e1d9e99668cc68aa>@@V<lambda_314360699dd331753a4119843814e9a7>@@@?$__crt_seh_guarded_call@H@@QEAAH$$QEAV<lambda_b521505b218e5242e90febf6bfebc422>@@AEAV<lambda_6978c1fb23f02e42e1d9e99668cc68aa>@@$$QEAV<lambda_314360699dd331753a4119843814e9a7>@@@Z@4HA 000000018001553d f   libucrt:commit.obj
 0001:0001453d       ?fin$0@?0???$?RV<lambda_bfedae4ebbf01fab1bb6dcc6a9e276e0>@@AEAV<lambda_2fe9b910cf3cbf4a0ab98a02ba45b3ec>@@V<lambda_237c231691f317818eb88cc1d5d642d6>@@@?$__crt_seh_guarded_call@H@@QEAAH$$QEAV<lambda_bfedae4ebbf01fab1bb6dcc6a9e276e0>@@AEAV<lambda_2fe9b910cf3cbf4a0ab98a02ba45b3ec>@@$$QEAV<lambda_237c231691f317818eb88cc1d5d642d6>@@@Z@4HA 000000018001553d f   libucrt:close.obj
 0001:00014557       _write$fin$0               0000000180015557 f   libucrt:write.obj
 0001:0001456e       fclose$fin$0               000000018001556e f   libucrt:fclose.obj
 0001:00014586       _ctrlfp$filt$0             0000000180015586 f   libucrt:fpctrl.obj
 0001:000145c0       _IsNonwritableInCurrentImage$filt$0 00000001800155c0 f   LIBCMT:pesect.obj
 0001:000145e0       $xdatasym                  00000001800155e0     chkstk.obj
 0001:000145e8       $unwind$__vcrt_freefls     00000001800155e8     libvcruntime:per_thread_data.obj
 0001:000145e8       $unwind$__dcrt_terminate_console_output 00000001800155e8     libucrt:initcon.obj
 0001:000145e8       $unwind$_msize             00000001800155e8     libucrt:msize.obj
 0001:000145e8       $unwind$__acrt_release_locale_ref 00000001800155e8     libucrt:locale_refcounting.obj
 0001:000145e8       $unwind$__doserrno         00000001800155e8     libucrt:errno.obj
 0001:000145e8       $unwind$__acrt_initialize_command_line 00000001800155e8     libucrt:argv_data.obj
 0001:000145e8       $unwind$??$uninitialize_environment_internal@_W@@YAXAEAPEAPEA_W@Z 00000001800155e8     libucrt:environment_initialization.obj
 0001:000145e8       $unwind$__acrt_initialize_ptd 00000001800155e8     libucrt:per_thread_data.obj
 0001:000145e8       $unwind$__acrt_initialize_multibyte 00000001800155e8     libucrt:mbctype.obj
 0001:000145e8       $unwind$??$uninitialize_environment_internal@D@@YAXAEAPEAPEAD@Z 00000001800155e8     libucrt:environment_initialization.obj
 0001:000145e8       $unwind$_errno             00000001800155e8     libucrt:errno.obj
 0001:000145e8       $unwind$?ItemWidth@?$DialogBuilderBase@UFarDialogItem@@@@IEAA_JAEBUFarDialogItem@@@Z 00000001800155e8     AutoWrap.obj
 0001:000145e8       $unwind$__dcrt_uninitialize_environments_nolock 00000001800155e8     libucrt:environment_initialization.obj
 0001:000145e8       $unwind$_set_errno_from_matherr 00000001800155e8     libucrt:fpexcept.obj
 0001:000145e8       $unwind$_invoke_watson     00000001800155e8     libucrt:invalid_parameter.obj
 0001:000145e8       $unwind$__scrt_dllmain_crt_thread_detach 00000001800155e8     LIBCMT:utility.obj
 0001:000145e8       $unwind$__GSHandlerCheck   00000001800155e8     LIBCMT:_gshandler_.obj
 0001:000145e8       $unwind$__acrt_uninitialize_ptd 00000001800155e8     libucrt:per_thread_data.obj
 0001:000145e8       $unwind$__scrt_dllmain_crt_thread_attach 00000001800155e8     LIBCMT:utility.obj
 0001:000145e8       $unwind$__vcrt_initialize_ptd 00000001800155e8     libvcruntime:per_thread_data.obj
 0001:000145e8       $unwind$__vcrt_thread_attach 00000001800155e8     libvcruntime:initialization.obj
 0001:000145e8       $unwind$__scrt_dllmain_uninitialize_critical 00000001800155e8     LIBCMT:utility.obj
 0001:000145e8       $unwind$?dllmain_crt_dispatch@@YAHQEAUHINSTANCE__@@KQEAX@Z 00000001800155e8     LIBCMT:dll_dllmain.obj
 0001:000145e8       $unwind$GetGlobalInfoW     00000001800155e8     AutoWrap.obj
 0001:000145e8       $unwind$__acrt_uninitialize_critical 00000001800155e8     libucrt:initialization.obj
 0001:000145e8       $unwind$__acrt_DownlevelLocaleNameToLCID 00000001800155e8     libucrt:lcidtoname_downlevel.obj
 0001:000145e8       $unwind$__vcrt_thread_detach 00000001800155e8     libvcruntime:initialization.obj
 0001:000145e8       $unwind$__acrt_thread_attach 00000001800155e8     libucrt:initialization.obj
 0001:000145e8       $unwind$_isatty            00000001800155e8     libucrt:isatty.obj
 0001:000145e8       $unwind$__acrt_thread_detach 00000001800155e8     libucrt:initialization.obj
 0001:000145e8       $unwind$_fileno            00000001800155e8     libucrt:fileno.obj
 0001:000145e8       $unwind$initialize_c       00000001800155e8     libucrt:initialization.obj
 0001:000145e8       $unwind$__vcrt_initialize  00000001800155e8     libvcruntime:initialization.obj
 0001:000145e8       $unwind$__scrt_initialize_default_local_stdio_options 00000001800155e8     LIBCMT:default_local_stdio_options.obj
 0001:000145e8       $unwind$_get_osfhandle     00000001800155e8     libucrt:osfinfo.obj
 0001:000145e8       $unwind$__pctype_func      00000001800155e8     libucrt:ctype.obj
 0001:000145e8       $unwind$atexit             00000001800155e8     LIBCMT:utility.obj
 0001:000145e8       $unwind$__scrt_dllmain_uninitialize_c 00000001800155e8     LIBCMT:utility.obj
 0001:000145e8       $unwind$uninitialize_environment 00000001800155e8     libucrt:initialization.obj
 0001:000145e8       $unwind$__scrt_dllmain_after_initialize_c 00000001800155e8     LIBCMT:utility.obj
 0001:000145e8       $unwind$_statfp            00000001800155e8     libucrt:fpctrl.obj
 0001:000145e8       $unwind$__vcrt_uninitialize_critical 00000001800155e8     libvcruntime:initialization.obj
 0001:000145e8       $unwind$__report_rangecheckfailure 00000001800155e8     LIBCMT:gs_report.obj
 0001:000145e8       $unwind$__vcrt_uninitialize_ptd 00000001800155e8     libvcruntime:per_thread_data.obj
 0001:000145e8       $unwind$__scrt_acquire_startup_lock 00000001800155e8     LIBCMT:utility.obj
 0001:000145e8       $unwind$__scrt_dllmain_before_initialize_c 00000001800155e8     LIBCMT:utility.obj
 0001:000145e8       $unwind$__acrt_initialize_heap 00000001800155e8     libucrt:heap_handle.obj
 0001:000145e8       $unwind$?initialize_multibyte@@YAHXZ 00000001800155e8     libucrt:multibyte_initializer.obj
 0001:000145e8       $unwind$__vcrt_uninitialize_telemetry_provider 00000001800155e8     libvcruntime:telemetry.obj
 0001:000145e8       $unwind$abort              00000001800155e8     libucrt:abort.obj
 0001:000145f0       $unwind$OpenW              00000001800155f0     AutoWrap.obj
 0001:00014610       $unwind$ProcessEditorInputW 0000000180015610     AutoWrap.obj
 0001:0001461c       $chain$4$ProcessEditorInputW 000000018001561c     AutoWrap.obj
 0001:00014640       $chain$6$ProcessEditorInputW 0000000180015640     AutoWrap.obj
 0001:00014664       $chain$7$ProcessEditorInputW 0000000180015664     AutoWrap.obj
 0001:00014678       $unwind$SetStartupInfoW    0000000180015678     AutoWrap.obj
 0001:0001468c       $unwind$__acrt_FlsGetValue 000000018001568c     libucrt:winapi_thunks.obj
 0001:0001468c       $unwind$__acrt_FlsFree     000000018001568c     libucrt:winapi_thunks.obj
 0001:0001468c       $unwind$__acrt_FlsAlloc    000000018001568c     libucrt:winapi_thunks.obj
 0001:0001468c       $unwind$__acrt_getptd      000000018001568c     libucrt:per_thread_data.obj
 0001:0001468c       $unwind$?replace_current_thread_locale_nolock@@YAXQEAU__acrt_ptd@@QEAU__crt_locale_data@@@Z 000000018001568c     libucrt:per_thread_data.obj
 0001:0001468c       $unwind$??0PluginIntEditFieldBinding@@QEAA@AEBUPluginStartupInfo@@PEAPEAXHPEAHH@Z 000000018001568c     AutoWrap.obj
 0001:0001468c       $unwind$_callnewh          000000018001568c     libucrt:new_handler.obj
 0001:0001468c       $unwind$_fclose_nolock     000000018001568c     libucrt:fclose.obj
 0001:0001468c       $unwind$??0_LocaleUpdate@@QEAA@QEAU__crt_locale_pointers@@@Z 000000018001568c     libucrt:_wctype.obj
 0001:0001468c       $unwind$__acrt_uninitialize_lowio 000000018001568c     libucrt:ioinit.obj
 0001:0001468c       $unwind$_updatetlocinfoEx_nolock 000000018001568c     libucrt:locale_refcounting.obj
 0001:0001468c       $unwind$?UpdateBorderSize@?$DialogBuilderBase@UFarDialogItem@@@@IEAAXXZ 000000018001568c     AutoWrap.obj
 0001:0001468c       $unwind$??_Gbad_alloc@std@@UEAAPEAXI@Z 000000018001568c     LIBCMT:throw_bad_alloc.obj
 0001:0001468c       $unwind$??$common_initialize_environment_nolock@D@@YAHXZ 000000018001568c     libucrt:environment_initialization.obj
 0001:0001468c       $unwind$_close_nolock      000000018001568c     libucrt:close.obj
 0001:0001468c       $unwind$?try_cor_exit_process@@YAXI@Z 000000018001568c     libucrt:exit.obj
 0001:0001468c       $unwind$??_Gexception@std@@UEAAPEAXI@Z 000000018001568c     LIBCMT:throw_bad_alloc.obj
 0001:0001468c       $unwind$__vcrt_FlsGetValue 000000018001568c     libvcruntime:winapi_downlevel.obj
 0001:0001468c       $unwind$__vcrt_FlsFree     000000018001568c     libvcruntime:winapi_downlevel.obj
 0001:0001468c       $unwind$??_G?$DialogBuilderBase@UFarDialogItem@@@@MEAAPEAXI@Z 000000018001568c     AutoWrap.obj
 0001:0001468c       $unwind$strncpy_s          000000018001568c     libucrt:strncpy_s.obj
 0001:0001468c       $unwind$??_Gbad_array_new_length@std@@UEAAPEAXI@Z 000000018001568c     LIBCMT:throw_bad_alloc.obj
 0001:0001468c       $unwind$__vcrt_FlsAlloc    000000018001568c     libvcruntime:winapi_downlevel.obj
 0001:0001468c       $unwind$?InitDialogItem@PluginDialogBuilder@@MEAAXPEAUFarDialogItem@@PEB_W@Z 000000018001568c     AutoWrap.obj
 0001:0001468c       $unwind$__vcrt_EventUnregister 000000018001568c     libvcruntime:winapi_downlevel.obj
 0001:0001468c       $unwind$?CreateRadioButtonBinding@PluginDialogBuilder@@MEAAPEAU?$DialogItemBinding@UFarDialogItem@@@@PEAH@Z 000000018001568c     AutoWrap.obj
 0001:0001468c       $unwind$??_GPluginDialogBuilder@@UEAAPEAXI@Z 000000018001568c     AutoWrap.obj
 0001:0001468c       $unwind$??0PluginUIntEditFieldBinding@@QEAA@AEBUPluginStartupInfo@@PEAPEAXHPEAIH@Z 000000018001568c     AutoWrap.obj
 0001:0001468c       $unwind$__acrt_invoke_user_matherr 000000018001568c     libucrt:matherr.obj
 0001:0001468c       $unwind$__acrt_errno_map_os_error 000000018001568c     libucrt:errno.obj
 0001:0001468c       $unwind$?SaveValue@PluginRadioButtonBinding@@UEAAXPEAUFarDialogItem@@H@Z 000000018001568c     AutoWrap.obj
 0001:0001468c       $unwind$_realloc_base      000000018001568c     libucrt:realloc_base.obj
 0001:00014698       $unwind$?ReallocDialogItems@?$DialogBuilderBase@UFarDialogItem@@@@IEAAXXZ 0000000180015698     AutoWrap.obj
 0001:000146a8       $unwind$?AddDialogItem@?$DialogBuilderBase@UFarDialogItem@@@@IEAAPEAUFarDialogItem@@W4FARDIALOGITEMTYPES@@PEB_W@Z 00000001800156a8     AutoWrap.obj
 0001:000146c0       $unwind$?MaxTextWidth@?$DialogBuilderBase@UFarDialogItem@@@@IEAA_JXZ 00000001800156c0     AutoWrap.obj
 0001:000146d0       $chain$1$?MaxTextWidth@?$DialogBuilderBase@UFarDialogItem@@@@IEAA_JXZ 00000001800156d0     AutoWrap.obj
 0001:000146e8       $chain$2$?MaxTextWidth@?$DialogBuilderBase@UFarDialogItem@@@@IEAA_JXZ 00000001800156e8     AutoWrap.obj
 0001:000146f8       $unwind$?SaveValues@?$DialogBuilderBase@UFarDialogItem@@@@IEAAXXZ 00000001800156f8     AutoWrap.obj
 0001:00014708       $chain$1$?SaveValues@?$DialogBuilderBase@UFarDialogItem@@@@IEAAXXZ 0000000180015708     AutoWrap.obj
 0001:00014720       $chain$2$?SaveValues@?$DialogBuilderBase@UFarDialogItem@@@@IEAAXXZ 0000000180015720     AutoWrap.obj
 0001:00014730       $unwind$??1?$DialogBuilderBase@UFarDialogItem@@@@MEAA@XZ 0000000180015730     AutoWrap.obj
 0001:00014730       $unwind$iswctype           0000000180015730     libucrt:iswctype.obj
 0001:00014730       $unwind$__acrt_is_packaged_app 0000000180015730     libucrt:winapi_thunks.obj
 0001:0001473c       $chain$0$??1?$DialogBuilderBase@UFarDialogItem@@@@MEAA@XZ 000000018001573c     AutoWrap.obj
 0001:00014750       $chain$1$??1?$DialogBuilderBase@UFarDialogItem@@@@MEAA@XZ 0000000180015750     AutoWrap.obj
 0001:00014760       $unwind$?AddButtons@?$DialogBuilderBase@UFarDialogItem@@@@QEAAXHPEBHHH@Z 0000000180015760     AutoWrap.obj
 0001:00014770       $chain$3$?AddButtons@?$DialogBuilderBase@UFarDialogItem@@@@QEAAXHPEBHHH@Z 0000000180015770     AutoWrap.obj
 0001:00014790       $chain$4$?AddButtons@?$DialogBuilderBase@UFarDialogItem@@@@QEAAXHPEBHHH@Z 0000000180015790     AutoWrap.obj
 0001:000147a0       $unwind$?DoShowDialog@PluginDialogBuilder@@MEAA_JXZ 00000001800157a0     AutoWrap.obj
 0001:000147ac       $unwind$?GetCommaWord@@YAPEB_WPEB_WPEA_W@Z 00000001800157ac     AutoWrap.obj
 0001:000147b8       $chain$4$?GetCommaWord@@YAPEB_WPEB_WPEA_W@Z 00000001800157b8     AutoWrap.obj
 0001:000147dc       $chain$6$?GetCommaWord@@YAPEB_WPEB_WPEA_W@Z 00000001800157dc     AutoWrap.obj
 0001:00014800       $unwind$?dllmain_crt_process_attach@@YAHQEAUHINSTANCE__@@QEAX@Z 0000000180015800     LIBCMT:dll_dllmain.obj
 0001:0001482c       $unwind$?dllmain_crt_process_detach@@YAH_N@Z 000000018001582c     LIBCMT:dll_dllmain.obj
 0001:00014854       $unwind$_query_new_handler$fin$0 0000000180015854     libucrt:new_handler.obj
 0001:00014854       $unwind$_IsNonwritableInCurrentImage$filt$0 0000000180015854     LIBCMT:pesect.obj
 0001:00014854       $unwind$common_flush_all$fin$1 0000000180015854     libucrt:fflush.obj
 0001:00014854       $unwind$?fin$0@?0???$?RV<lambda_bfedae4ebbf01fab1bb6dcc6a9e276e0>@@AEAV<lambda_2fe9b910cf3cbf4a0ab98a02ba45b3ec>@@V<lambda_237c231691f317818eb88cc1d5d642d6>@@@?$__crt_seh_guarded_call@H@@QEAAH$$QEAV<lambda_bfedae4ebbf01fab1bb6dcc6a9e276e0>@@AEAV<lambda_2fe9b910cf3cbf4a0ab98a02ba45b3ec>@@$$QEAV<lambda_237c231691f317818eb88cc1d5d642d6>@@@Z@4HA 0000000180015854     libucrt:close.obj
 0001:00014854       $unwind$?fin$0@?0???$?RV<lambda_fb3a7dec4e47f37f22dae91bb15c9095>@@AEAV<lambda_698284760c8add0bfb0756c19673e34b>@@V<lambda_dfb8eca1e75fef3034a8fb18dd509707>@@@?$__crt_seh_guarded_call@X@@QEAAX$$QEAV<lambda_fb3a7dec4e47f37f22dae91bb15c9095>@@AEAV<lambda_698284760c8add0bfb0756c19673e34b>@@$$QEAV<lambda_dfb8eca1e75fef3034a8fb18dd509707>@@@Z@4HA 0000000180015854     libucrt:per_thread_data.obj
 0001:00014854       $unwind$?fin$0@?0???$?RV<lambda_e24bbb7b643b32fcea6fa61b31d4c984>@@AEAV<lambda_275893d493268fdec8709772e3fcec0e>@@V<lambda_9d71df4d7cf3f480f8d633942495c3b0>@@@?$__crt_seh_guarded_call@H@@QEAAH$$QEAV<lambda_e24bbb7b643b32fcea6fa61b31d4c984>@@AEAV<lambda_275893d493268fdec8709772e3fcec0e>@@$$QEAV<lambda_9d71df4d7cf3f480f8d633942495c3b0>@@@Z@4HA 0000000180015854     libucrt:onexit.obj
 0001:00014854       $unwind$__acrt_uninitialize_locale$fin$0 0000000180015854     libucrt:wsetlocale.obj
 0001:00014854       $unwind$raise$fin$0        0000000180015854     libucrt:signal.obj
 0001:00014854       $unwind$?fin$0@?0???$?RV<lambda_c36588078e9f5dfd39652860aa6b3aaf>@@AEAV<lambda_ec61778202f4f5fc7e7711acc23c3bca>@@V<lambda_dc9d2797ccde5d239b4a0efae8ebd7db>@@@?$__crt_seh_guarded_call@P6AXH@Z@@QEAAP6AXH@Z$$QEAV<lambda_c36588078e9f5dfd39652860aa6b3aaf>@@AEAV<lambda_ec61778202f4f5fc7e7711acc23c3bca>@@$$QEAV<lambda_dc9d2797ccde5d239b4a0efae8ebd7db>@@@Z@4HA 0000000180015854     libucrt:signal.obj
 0001:00014854       $unwind$__acrt_update_thread_locale_data$fin$0 0000000180015854     libucrt:locale_refcounting.obj
 0001:00014854       $unwind$_ctrlfp$filt$0     0000000180015854     libucrt:fpctrl.obj
 0001:00014854       $unwind$?fin$0@?0???$?RV<lambda_b521505b218e5242e90febf6bfebc422>@@AEAV<lambda_6978c1fb23f02e42e1d9e99668cc68aa>@@V<lambda_314360699dd331753a4119843814e9a7>@@@?$__crt_seh_guarded_call@H@@QEAAH$$QEAV<lambda_b521505b218e5242e90febf6bfebc422>@@AEAV<lambda_6978c1fb23f02e42e1d9e99668cc68aa>@@$$QEAV<lambda_314360699dd331753a4119843814e9a7>@@@Z@4HA 0000000180015854     libucrt:commit.obj
 0001:00014854       $unwind$_fcloseall$fin$0   0000000180015854     libucrt:closeall.obj
 0001:00014854       $unwind$fclose$fin$0       0000000180015854     libucrt:fclose.obj
 0001:00014854       $unwind$?fin$0@?0???$?RV<lambda_5e887d1dcbef67a5eb4283622ba103bf>@@AEAV<lambda_4466841279450cc726390878d4a41900>@@V<lambda_341c25c0346d94847f1f3c463c57e077>@@@?$__crt_seh_guarded_call@X@@QEAAX$$QEAV<lambda_5e887d1dcbef67a5eb4283622ba103bf>@@AEAV<lambda_4466841279450cc726390878d4a41900>@@$$QEAV<lambda_341c25c0346d94847f1f3c463c57e077>@@@Z@4HA 0000000180015854     libucrt:per_thread_data.obj
 0001:00014854       $unwind$__acrt_lowio_ensure_fh_exists$fin$0 0000000180015854     libucrt:osfinfo.obj
 0001:00014854       $unwind$?fin$0@?0???$?RV<lambda_99476a1ad63dd22509b5d3e65b0ffc95>@@AEAV<lambda_ad1ced32f4ac17aa236e5ef05d6b3b7c>@@V<lambda_f7424dd8d45958661754dc4f2697e9c3>@@@?$__crt_seh_guarded_call@X@@QEAAX$$QEAV<lambda_99476a1ad63dd22509b5d3e65b0ffc95>@@AEAV<lambda_ad1ced32f4ac17aa236e5ef05d6b3b7c>@@$$QEAV<lambda_f7424dd8d45958661754dc4f2697e9c3>@@@Z@4HA 0000000180015854     libucrt:mbctype.obj
 0001:00014854       $unwind$common_flush_all$fin$0 0000000180015854     libucrt:fflush.obj
 0001:00014854       $unwind$?fin$0@?0??dllmain_crt_process_detach@@YAH_N@Z@4HA 0000000180015854     LIBCMT:dll_dllmain.obj
 0001:00014854       $unwind$_write$fin$0       0000000180015854     libucrt:write.obj
 0001:00014854       $unwind$?fin$0@?0???$?RV<lambda_b8c45f8f788dd370798f47cfe8ac3a86>@@AEAV<lambda_4e60a939b0d047cfe11ddc22648dfba9>@@V<lambda_332c3edc96d0294ec56c57d38c1cdfd5>@@@?$__crt_seh_guarded_call@H@@QEAAH$$QEAV<lambda_b8c45f8f788dd370798f47cfe8ac3a86>@@AEAV<lambda_4e60a939b0d047cfe11ddc22648dfba9>@@$$QEAV<lambda_332c3edc96d0294ec56c57d38c1cdfd5>@@@Z@4HA 0000000180015854     libucrt:onexit.obj
 0001:00014854       $unwind$?fin$0@?0???$?RV<lambda_72d1df2b273a38828b1ce30cbf4cdab5>@@AEAV<lambda_876a65b173b8412d3a47c70a915b0cf4>@@V<lambda_41932305e351933ebe8f8be3ed8bb5dc>@@@?$__crt_seh_guarded_call@X@@QEAAX$$QEAV<lambda_72d1df2b273a38828b1ce30cbf4cdab5>@@AEAV<lambda_876a65b173b8412d3a47c70a915b0cf4>@@$$QEAV<lambda_41932305e351933ebe8f8be3ed8bb5dc>@@@Z@4HA 0000000180015854     libucrt:per_thread_data.obj
 0001:00014854       $unwind$?fin$1@?0??common_exit@@YAXHW4_crt_exit_cleanup_mode@@W4_crt_exit_return_mode@@@Z@4HA 0000000180015854     libucrt:exit.obj
 0001:00014854       $unwind$__acrt_initialize_lowio$fin$0 0000000180015854     libucrt:ioinit.obj
 0001:00014854       $unwind$?fin$0@?0??dllmain_crt_process_attach@@YAHQEAUHINSTANCE__@@QEAX@Z@4HA 0000000180015854     LIBCMT:dll_dllmain.obj
 0001:00014854       $unwind$__acrt_update_thread_multibyte_data$fin$0 0000000180015854     libucrt:mbctype.obj
 0001:00014854       $unwind$?filt$0@?0??common_exit@@YAXHW4_crt_exit_cleanup_mode@@W4_crt_exit_return_mode@@@Z@4HA 0000000180015854     libucrt:exit.obj
 0001:00014854       $unwind$?fin$0@?0???$?RV<lambda_46352004c1216016012b18bd6f87e700>@@AEAV<lambda_3bd07e1a1191394380780325891bf33f>@@V<lambda_334532d3f185bcaa59b5be82d7d22bff>@@@?$__crt_seh_guarded_call@X@@QEAAX$$QEAV<lambda_46352004c1216016012b18bd6f87e700>@@AEAV<lambda_3bd07e1a1191394380780325891bf33f>@@$$QEAV<lambda_334532d3f185bcaa59b5be82d7d22bff>@@@Z@4HA 0000000180015854     libucrt:per_thread_data.obj
 0001:0001485c       $unwind$?dllmain_dispatch@@YAHQEAUHINSTANCE__@@KQEAX@Z 000000018001585c     LIBCMT:dll_dllmain.obj
 0001:00014884       $unwind$?filt$0@?0??dllmain_dispatch@@YAHQEAUHINSTANCE__@@KQEAX@Z@4HA 0000000180015884     LIBCMT:dll_dllmain.obj
 0001:0001488c       $unwind$__scrt_is_nonwritable_in_current_image 000000018001588c     LIBCMT:utility.obj
 0001:000148ac       $unwind$__scrt_is_nonwritable_in_current_image$filt$0 00000001800158ac     LIBCMT:utility.obj
 0001:000148b4       $unwind$__scrt_initialize_onexit_tables 00000001800158b4     LIBCMT:utility.obj
 0001:000148c0       $unwind$__scrt_dllmain_exception_filter 00000001800158c0     LIBCMT:utility.obj
 0001:000148c0       $unwind$?expand_if_necessary@?$argument_list@D@?A0xca0879c4@@AEAAHXZ 00000001800158c0     libucrt:argv_wildcards.obj
 0001:000148c0       $unwind$__acrt_lowio_create_handle_array 00000001800158c0     libucrt:osfinfo.obj
 0001:000148c0       $unwind$?dllmain_raw@@YAHQEAUHINSTANCE__@@KQEAX@Z 00000001800158c0     LIBCMT:dll_dllmain.obj
 0001:000148c0       $unwind$?AddTextAfter@?$DialogBuilderBase@UFarDialogItem@@@@QEAAPEAUFarDialogItem@@PEAU2@PEB_WH@Z 00000001800158c0     AutoWrap.obj
 0001:000148c0       $unwind$__vcrt_InitializeCriticalSectionEx 00000001800158c0     libvcruntime:winapi_downlevel.obj
 0001:000148c0       $unwind$?setSBCS@@YAXPEAU__crt_multibyte_data@@@Z 00000001800158c0     libucrt:mbctype.obj
 0001:000148c0       $unwind$__acrt_execute_initializers 00000001800158c0     libucrt:shared_initialization.obj
 0001:000148c0       $unwind$__acrt_InitializeCriticalSectionEx 00000001800158c0     libucrt:winapi_thunks.obj
 0001:000148c0       $unwind$__acrt_free_locale 00000001800158c0     libucrt:locale_refcounting.obj
 0001:000148c0       $unwind$_recalloc_base     00000001800158c0     libucrt:recalloc.obj
 0001:000148c0       $unwind$_seh_filter_exe    00000001800158c0     libucrt:exception_filter.obj
 0001:000148d4       $unwind$__security_init_cookie 00000001800158d4     LIBCMT:gs_support.obj
 0001:000148e0       $unwind$__scrt_fastfail    00000001800158e0     LIBCMT:utility_desktop.obj
 0001:000148f0       $unwind$__isa_available_init 00000001800158f0     LIBCMT:_cpu_disp_.obj
 0001:00014900       $xdatasym                  0000000180015900     LIBCMT:_guard_dispatch_.obj
 0001:00014904       $unwind$wcschr             0000000180015904     libvcruntime:wcschr.obj
 0001:00014910       $xdatasym                  0000000180015910     libvcruntime:memset.obj
 0001:00014914       $unwind$__telemetry_main_return_trigger 0000000180015914     libvcruntime:telemetry.obj
 0001:00014914       $unwind$__telemetry_main_invoke_trigger 0000000180015914     libvcruntime:telemetry.obj
 0001:0001492c       $unwind$?_TlgEnableCallback@__vcrt_trace_logging_provider@@YAXPEBU_GUID@@KE_K1PEAU_EVENT_FILTER_DESCRIPTOR@@PEAX@Z 000000018001592c     libvcruntime:telemetry.obj
 0001:00014948       $unwind$_isleadbyte_l      0000000180015948     libucrt:_wctype.obj
 0001:00014948       $unwind$?_TlgWrite@__vcrt_trace_logging_provider@@YAJPEBU_TlgProvider_t@1@PEFBXPEBU_GUID@@2IPEAU_EVENT_DATA_DESCRIPTOR@@@Z 0000000180015948     libvcruntime:telemetry.obj
 0001:00014948       $unwind$?getSystemCP@@YAHH@Z 0000000180015948     libucrt:mbctype.obj
 0001:00014950       $unwind$__C_specific_handler 0000000180015950     libvcruntime:_chandler_.obj
 0001:0001496c       $unwind$_CxxThrowException 000000018001596c     libvcruntime:throw.obj
 0001:00014980       $unwind$_invalid_parameter 0000000180015980     libucrt:invalid_parameter.obj
 0001:00014980       $unwind$__vcrt_EventWriteTransfer 0000000180015980     libvcruntime:winapi_downlevel.obj
 0001:00014998       $unwind$__vcrt_initialize_winapi_thunks 0000000180015998     libvcruntime:winapi_downlevel.obj
 0001:00014998       $unwind$__acrt_initialize_winapi_thunks 0000000180015998     libucrt:winapi_thunks.obj
 0001:000149a0       $unwind$__vcrt_uninitialize_winapi_thunks 00000001800159a0     libvcruntime:winapi_downlevel.obj
 0001:000149a8       $unwind$?try_get_function@@YAPEAXW4function_id@?A0x49c8dc86@@QEBDQEBW4module_id@2@2@Z 00000001800159a8     libvcruntime:winapi_downlevel.obj
 0001:000149a8       $unwind$?try_get_function@@YAPEAXW4function_id@?A0x63058377@@QEBDQEBW4module_id@2@2@Z 00000001800159a8     libucrt:winapi_thunks.obj
 0001:000149c8       $xdatasym                  00000001800159c8     libvcruntime:_jmpuwind_.obj
 0001:000149dc       $unwind$_query_new_handler 00000001800159dc     libucrt:new_handler.obj
 0001:000149fc       $unwind$__vcrt_EventRegister 00000001800159fc     libvcruntime:winapi_downlevel.obj
 0001:000149fc       $unwind$_initterm          00000001800159fc     libucrt:initterm.obj
 0001:000149fc       $unwind$__acrt_initialize_stdio 00000001800159fc     libucrt:_file.obj
 0001:000149fc       $unwind$__vcrt_EventSetInformation 00000001800159fc     libvcruntime:winapi_downlevel.obj
 0001:00014a14       $unwind$?common_exit@@YAXHW4_crt_exit_cleanup_mode@@W4_crt_exit_return_mode@@@Z 0000000180015a14     libucrt:exit.obj
 0001:00014a54       $unwind$_configure_narrow_argv 0000000180015a54     libucrt:argv_parsing.obj
 0001:00014a68       $unwind$??R<lambda_4e60a939b0d047cfe11ddc22648dfba9>@@QEBAHXZ 0000000180015a68     libucrt:onexit.obj
 0001:00014a68       $unwind$??$parse_command_line@D@@YAXPEADPEAPEAD0PEA_K2@Z 0000000180015a68     libucrt:argv_parsing.obj
 0001:00014a84       $unwind$??$free_environment@_W@@YAXQEAPEA_W@Z 0000000180015a84     libucrt:environment_initialization.obj
 0001:00014a84       $unwind$??$free_environment@D@@YAXQEAPEAD@Z 0000000180015a84     libucrt:environment_initialization.obj
 0001:00014a90       $unwind$?AddUIntEditField@PluginDialogBuilder@@UEAAPEAUFarDialogItem@@PEAIH@Z 0000000180015a90     AutoWrap.obj
 0001:00014a90       $unwind$?AddIntEditField@PluginDialogBuilder@@UEAAPEAUFarDialogItem@@PEAHH@Z 0000000180015a90     AutoWrap.obj
 0001:00014a90       $unwind$??$create_environment@D@@YAQEAPEADQEAD@Z 0000000180015a90     libucrt:environment_initialization.obj
 0001:00014aa8       $unwind$_register_onexit_function 0000000180015aa8     libucrt:onexit.obj
 0001:00014ab0       $unwind$_execute_onexit_table 0000000180015ab0     libucrt:onexit.obj
 0001:00014ab8       $unwind$??$?RV<lambda_b8c45f8f788dd370798f47cfe8ac3a86>@@AEAV<lambda_4e60a939b0d047cfe11ddc22648dfba9>@@V<lambda_332c3edc96d0294ec56c57d38c1cdfd5>@@@?$__crt_seh_guarded_call@H@@QEAAH$$QEAV<lambda_b8c45f8f788dd370798f47cfe8ac3a86>@@AEAV<lambda_4e60a939b0d047cfe11ddc22648dfba9>@@$$QEAV<lambda_332c3edc96d0294ec56c57d38c1cdfd5>@@@Z 0000000180015ab8     libucrt:onexit.obj
 0001:00014adc       $unwind$??$?RV<lambda_e24bbb7b643b32fcea6fa61b31d4c984>@@AEAV<lambda_275893d493268fdec8709772e3fcec0e>@@V<lambda_9d71df4d7cf3f480f8d633942495c3b0>@@@?$__crt_seh_guarded_call@H@@QEAAH$$QEAV<lambda_e24bbb7b643b32fcea6fa61b31d4c984>@@AEAV<lambda_275893d493268fdec8709772e3fcec0e>@@$$QEAV<lambda_9d71df4d7cf3f480f8d633942495c3b0>@@@Z 0000000180015adc     libucrt:onexit.obj
 0001:00014b0c       $unwind$terminate          0000000180015b0c     libucrt:terminate.obj
 0001:00014b2c       $unwind$_free_base         0000000180015b2c     libucrt:free_base.obj
 0001:00014b2c       $unwind$__acrt_locale_free_lc_time_if_unreferenced 0000000180015b2c     libucrt:locale_refcounting.obj
 0001:00014b2c       $unwind$?destroy_fls@@YAXPEAX@Z 0000000180015b2c     libucrt:per_thread_data.obj
 0001:00014b2c       $unwind$__acrt_locale_free_numeric 0000000180015b2c     libucrt:initnum.obj
 0001:00014b34       $unwind$?construct_ptd_array@@YAXQEAU__acrt_ptd@@@Z 0000000180015b34     libucrt:per_thread_data.obj
 0001:00014b3c       $unwind$?destroy_ptd_array@@YAXQEAU__acrt_ptd@@@Z 0000000180015b3c     libucrt:per_thread_data.obj
 0001:00014b44       $unwind$??$?RV<lambda_72d1df2b273a38828b1ce30cbf4cdab5>@@AEAV<lambda_876a65b173b8412d3a47c70a915b0cf4>@@V<lambda_41932305e351933ebe8f8be3ed8bb5dc>@@@?$__crt_seh_guarded_call@X@@QEAAX$$QEAV<lambda_72d1df2b273a38828b1ce30cbf4cdab5>@@AEAV<lambda_876a65b173b8412d3a47c70a915b0cf4>@@$$QEAV<lambda_41932305e351933ebe8f8be3ed8bb5dc>@@@Z 0000000180015b44     libucrt:per_thread_data.obj
 0001:00014b68       $unwind$??$?RV<lambda_5e887d1dcbef67a5eb4283622ba103bf>@@AEAV<lambda_4466841279450cc726390878d4a41900>@@V<lambda_341c25c0346d94847f1f3c463c57e077>@@@?$__crt_seh_guarded_call@X@@QEAAX$$QEAV<lambda_5e887d1dcbef67a5eb4283622ba103bf>@@AEAV<lambda_4466841279450cc726390878d4a41900>@@$$QEAV<lambda_341c25c0346d94847f1f3c463c57e077>@@@Z 0000000180015b68     libucrt:per_thread_data.obj
 0001:00014b8c       $unwind$??$?RV<lambda_46352004c1216016012b18bd6f87e700>@@AEAV<lambda_3bd07e1a1191394380780325891bf33f>@@V<lambda_334532d3f185bcaa59b5be82d7d22bff>@@@?$__crt_seh_guarded_call@X@@QEAAX$$QEAV<lambda_46352004c1216016012b18bd6f87e700>@@AEAV<lambda_3bd07e1a1191394380780325891bf33f>@@$$QEAV<lambda_334532d3f185bcaa59b5be82d7d22bff>@@@Z 0000000180015b8c     libucrt:per_thread_data.obj
 0001:00014bb0       $unwind$??$?RV<lambda_fb3a7dec4e47f37f22dae91bb15c9095>@@AEAV<lambda_698284760c8add0bfb0756c19673e34b>@@V<lambda_dfb8eca1e75fef3034a8fb18dd509707>@@@?$__crt_seh_guarded_call@X@@QEAAX$$QEAV<lambda_fb3a7dec4e47f37f22dae91bb15c9095>@@AEAV<lambda_698284760c8add0bfb0756c19673e34b>@@$$QEAV<lambda_dfb8eca1e75fef3034a8fb18dd509707>@@@Z 0000000180015bb0     libucrt:per_thread_data.obj
 0001:00014bd4       $unwind$__acrt_uninitialize_locale 0000000180015bd4     libucrt:wsetlocale.obj
 0001:00014bf4       $unwind$__raise_securityfailure 0000000180015bf4     LIBCMT:gs_report.obj
 0001:00014bf4       $unwind$_onexit            0000000180015bf4     LIBCMT:utility.obj
 0001:00014bf4       $unwind$__acrt_uninitialize_winapi_thunks 0000000180015bf4     libucrt:winapi_thunks.obj
 0001:00014bf4       $unwind$__acrt_stdio_free_buffer_nolock 0000000180015bf4     libucrt:_freebuf.obj
 0001:00014bf4       $unwind$_fflush_nolock     0000000180015bf4     libucrt:fflush.obj
 0001:00014bf4       $unwind$__acrt_initialize_locks 0000000180015bf4     libucrt:locks.obj
 0001:00014bf4       $unwind$__acrt_uninitialize_locks 0000000180015bf4     libucrt:locks.obj
 0001:00014bf4       $unwind$__scrt_uninitialize_crt 0000000180015bf4     LIBCMT:utility.obj
 0001:00014bf4       $unwind$strcpy_s           0000000180015bf4     libucrt:strcpy_s.obj
 0001:00014bf4       $unwind$_malloc_base       0000000180015bf4     libucrt:malloc_base.obj
 0001:00014bf4       $unwind$?exit_or_terminate_process@@YAXI@Z 0000000180015bf4     libucrt:exit.obj
 0001:00014bf4       $unwind$initialize_pointers 0000000180015bf4     libucrt:initialization.obj
 0001:00014bf4       $unwind$??0exception@std@@QEAA@AEBV01@@Z 0000000180015bf4     LIBCMT:throw_bad_alloc.obj
 0001:00014bf4       $unwind$??_G?$DialogItemBinding@UFarDialogItem@@@@UEAAPEAXI@Z 0000000180015bf4     AutoWrap.obj
 0001:00014bf4       $unwind$?SaveValue@PluginCheckBoxBinding@@UEAAXPEAUFarDialogItem@@H@Z 0000000180015bf4     AutoWrap.obj
 0001:00014bf4       $unwind$??2@YAPEAX_K@Z     0000000180015bf4     LIBCMT:new_scalar.obj
 0001:00014bf4       $unwind$__acrt_uninitialize_stdio 0000000180015bf4     libucrt:_file.obj
 0001:00014bf4       $unwind$?SaveValue@PluginUIntEditFieldBinding@@UEAAXPEAUFarDialogItem@@H@Z 0000000180015bf4     AutoWrap.obj
 0001:00014bf4       $unwind$??_Gtype_info@@UEAAPEAXI@Z 0000000180015bf4     LIBCMT:std_type_info_static.obj
 0001:00014bf4       $unwind$??_GPluginIntEditFieldBinding@@UEAAPEAXI@Z 0000000180015bf4     AutoWrap.obj
 0001:00014bf4       $unwind$??_GPluginCheckBoxBinding@@UEAAPEAXI@Z 0000000180015bf4     AutoWrap.obj
 0001:00014bf4       $unwind$?SaveValue@PluginIntEditFieldBinding@@UEAAXPEAUFarDialogItem@@H@Z 0000000180015bf4     AutoWrap.obj
 0001:00014bf4       $unwind$__vcrt_freeptd     0000000180015bf4     libvcruntime:per_thread_data.obj
 0001:00014bf4       $unwind$??0bad_array_new_length@std@@QEAA@AEBV01@@Z 0000000180015bf4     LIBCMT:throw_bad_alloc.obj
 0001:00014bf4       $unwind$__acrt_freeptd     0000000180015bf4     libucrt:per_thread_data.obj
 0001:00014bf4       $unwind$_set_statfp        0000000180015bf4     libucrt:fpctrl.obj
 0001:00014bf4       $unwind$__acrt_allocate_buffer_for_argv 0000000180015bf4     libucrt:argv_parsing.obj
 0001:00014bf4       $unwind$_clrfp             0000000180015bf4     libucrt:fpctrl.obj
 0001:00014bf4       $unwind$__acrt_update_locale_info 0000000180015bf4     libucrt:locale_update.obj
 0001:00014bf4       $unwind$__scrt_initialize_crt 0000000180015bf4     LIBCMT:utility.obj
 0001:00014bf4       $unwind$uninitialize_allocated_memory 0000000180015bf4     libucrt:initialization.obj
 0001:00014bf4       $unwind$_calloc_base       0000000180015bf4     libucrt:calloc_base.obj
 0001:00014bf4       $unwind$__std_exception_destroy 0000000180015bf4     libvcruntime:std_exception.obj
 0001:00014bf4       $unwind$__std_type_info_destroy_list 0000000180015bf4     libvcruntime:std_type_info.obj
 0001:00014bf4       $unwind$GetPluginInfoW     0000000180015bf4     AutoWrap.obj
 0001:00014bf4       $unwind$__scrt_release_startup_lock 0000000180015bf4     LIBCMT:utility.obj
 0001:00014bf4       $unwind$??_GPluginRadioButtonBinding@@UEAAPEAXI@Z 0000000180015bf4     AutoWrap.obj
 0001:00014bf4       $unwind$??_GPluginUIntEditFieldBinding@@UEAAPEAXI@Z 0000000180015bf4     AutoWrap.obj
 0001:00014bf4       $unwind$??0bad_alloc@std@@QEAA@AEBV01@@Z 0000000180015bf4     LIBCMT:throw_bad_alloc.obj
 0001:00014bf4       $unwind$??_GPluginEditFieldBinding@@UEAAPEAXI@Z 0000000180015bf4     AutoWrap.obj
 0001:00014bf4       $unwind$__vcrt_uninitialize_locks 0000000180015bf4     libvcruntime:locks.obj
 0001:00014bf4       $unwind$__vcrt_initialize_locks 0000000180015bf4     libvcruntime:locks.obj
 0001:00014bf4       $unwind$__vcrt_uninitialize 0000000180015bf4     libvcruntime:initialization.obj
 0001:00014bf4       $unwind$__acrt_update_multibyte_info 0000000180015bf4     libucrt:locale_update.obj
 0001:00014bf4       $unwind$?SaveValue@PluginEditFieldBinding@@UEAAXPEAUFarDialogItem@@H@Z 0000000180015bf4     AutoWrap.obj
 0001:00014bfc       $unwind$__acrt_LCMapStringEx 0000000180015bfc     libucrt:winapi_thunks.obj
 0001:00014bfc       $unwind$_mbtowc_l          0000000180015bfc     libucrt:mbtowc.obj
 0001:00014c14       $unwind$_log10_special     0000000180015c14     libucrt:log_special.obj
 0001:00014c14       $unwind$_invalid_parameter_noinfo 0000000180015c14     libucrt:invalid_parameter.obj
 0001:00014c1c       $unwind$__acrt_call_reportfault 0000000180015c1c     libucrt:invalid_parameter.obj
 0001:00014c3c       $unwind$??$common_expand_argv_wildcards@D@@YAHQEAPEADQEAPEAPEAD@Z 0000000180015c3c     libucrt:argv_wildcards.obj
 0001:00014c54       $unwind$??$copy_and_add_argument_to_buffer@D@@YAHQEBD0_KAEAV?$argument_list@D@?A0xca0879c4@@@Z 0000000180015c54     libucrt:argv_wildcards.obj
 0001:00014c70       $unwind$??$expand_argument_wildcards@D@@YAHQEAD0AEAV?$argument_list@D@?A0xca0879c4@@@Z 0000000180015c70     libucrt:argv_wildcards.obj
 0001:00014c90       $unwind$__acrt_update_thread_multibyte_data 0000000180015c90     libucrt:mbctype.obj
 0001:00014cb4       $unwind$_setmbcp_nolock    0000000180015cb4     libucrt:mbctype.obj
 0001:00014cd4       $unwind$?setSBUpLow@@YAXPEAU__crt_multibyte_data@@@Z 0000000180015cd4     libucrt:mbctype.obj
 0001:00014cf0       $unwind$?setmbcp_internal@@YAHH_N@Z 0000000180015cf0     libucrt:mbctype.obj
 0001:00014d00       $unwind$??$?RV<lambda_99476a1ad63dd22509b5d3e65b0ffc95>@@AEAV<lambda_ad1ced32f4ac17aa236e5ef05d6b3b7c>@@V<lambda_f7424dd8d45958661754dc4f2697e9c3>@@@?$__crt_seh_guarded_call@X@@QEAAX$$QEAV<lambda_99476a1ad63dd22509b5d3e65b0ffc95>@@AEAV<lambda_ad1ced32f4ac17aa236e5ef05d6b3b7c>@@$$QEAV<lambda_f7424dd8d45958661754dc4f2697e9c3>@@@Z 0000000180015d00     libucrt:mbctype.obj
 0001:00014d24       $unwind$?x_ismbbtype_l@@YAHPEAU__crt_locale_pointers@@IHH@Z 0000000180015d24     libucrt:ismbbyte.obj
 0001:00014d34       $unwind$__dcrt_get_narrow_environment_from_os 0000000180015d34     libucrt:get_environment_from_os.obj
 0001:00014d4c       $unwind$__acrt_initialize_lowio 0000000180015d4c     libucrt:ioinit.obj
 0001:00014d6c       $unwind$?initialize_inherited_file_handles_nolock@@YAXXZ 0000000180015d6c     libucrt:ioinit.obj
 0001:00014d88       $unwind$__acrt_get_sigabrt_handler 0000000180015d88     libucrt:signal.obj
 0001:00014d90       $unwind$raise              0000000180015d90     libucrt:signal.obj
 0001:00014dbc       $unwind$??$?RV<lambda_c36588078e9f5dfd39652860aa6b3aaf>@@AEAV<lambda_ec61778202f4f5fc7e7711acc23c3bca>@@V<lambda_dc9d2797ccde5d239b4a0efae8ebd7db>@@@?$__crt_seh_guarded_call@P6AXH@Z@@QEAAP6AXH@Z$$QEAV<lambda_c36588078e9f5dfd39652860aa6b3aaf>@@AEAV<lambda_ec61778202f4f5fc7e7711acc23c3bca>@@$$QEAV<lambda_dc9d2797ccde5d239b4a0efae8ebd7db>@@@Z 0000000180015dbc     libucrt:signal.obj
 0001:00014de0       $unwind$__acrt_update_thread_locale_data 0000000180015de0     libucrt:locale_refcounting.obj
 0001:00014e04       $unwind$__acrt_locale_free_monetary 0000000180015e04     libucrt:initmon.obj
 0001:00014e0c       $unwind$__acrt_locale_free_time 0000000180015e0c     libucrt:inittime.obj
 0001:00014e1c       $unwind$__acrt_GetStringTypeA 0000000180015e1c     libucrt:getstringtypea.obj
 0001:00014e44       $unwind$?GetTableIndexFromLocaleName@@YAHPEB_W@Z 0000000180015e44     libucrt:lcidtoname_downlevel.obj
 0001:00014e5c       $unwind$qsort              0000000180015e5c     libucrt:qsort.obj
 0001:00014e74       $chain$4$qsort             0000000180015e74     libucrt:qsort.obj
 0001:00014e98       $chain$5$qsort             0000000180015e98     libucrt:qsort.obj
 0001:00014ea8       $unwind$?shortsort@@YAXPEAD0_KP6AHPEBX2@Z@Z 0000000180015ea8     libucrt:qsort.obj
 0001:00014eb8       $chain$2$?shortsort@@YAXPEAD0_KP6AHPEBX2@Z@Z 0000000180015eb8     libucrt:qsort.obj
 0001:00014ed4       $chain$3$?shortsort@@YAXPEAD0_KP6AHPEBX2@Z@Z 0000000180015ed4     libucrt:qsort.obj
 0001:00014ee4       $unwind$strpbrk            0000000180015ee4     libucrt:strpbrk.obj
 0001:00014ef4       $unwind$_mbsdec_l          0000000180015ef4     libucrt:mbsdec.obj
 0001:00014f00       $unwind$__acrt_LCMapStringA 0000000180015f00     libucrt:lcmapstringa.obj
 0001:00014f10       $unwind$?__acrt_LCMapStringA_stat@@YAHPEAU__crt_locale_pointers@@PEB_WKPEBDHPEADHHH@Z 0000000180015f10     libucrt:lcmapstringa.obj
 0001:00014f38       $unwind$__std_exception_copy 0000000180015f38     libvcruntime:std_exception.obj
 0001:00014f38       $unwind$_free_osfhnd       0000000180015f38     libucrt:osfinfo.obj
 0001:00014f38       $unwind$?initialize_stdio_handles_nolock@@YAXXZ 0000000180015f38     libucrt:ioinit.obj
 0001:00014f4c       $unwind$__acrt_lowio_destroy_handle_array 0000000180015f4c     libucrt:osfinfo.obj
 0001:00014f5c       $unwind$__acrt_lowio_ensure_fh_exists 0000000180015f5c     libucrt:osfinfo.obj
 0001:00014f88       $unwind$common_flush_all   0000000180015f88     libucrt:fflush.obj
 0001:00014fc4       $unwind$_fcloseall         0000000180015fc4     libucrt:closeall.obj
 0001:00014fe8       $unwind$_commit            0000000180015fe8     libucrt:commit.obj
 0001:00014fe8       $unwind$_close             0000000180015fe8     libucrt:close.obj
 0001:00014ff0       $unwind$??$?RV<lambda_b521505b218e5242e90febf6bfebc422>@@AEAV<lambda_6978c1fb23f02e42e1d9e99668cc68aa>@@V<lambda_314360699dd331753a4119843814e9a7>@@@?$__crt_seh_guarded_call@H@@QEAAH$$QEAV<lambda_b521505b218e5242e90febf6bfebc422>@@AEAV<lambda_6978c1fb23f02e42e1d9e99668cc68aa>@@$$QEAV<lambda_314360699dd331753a4119843814e9a7>@@@Z 0000000180015ff0     libucrt:commit.obj
 0001:00015014       $unwind$_write             0000000180016014     libucrt:write.obj
 0001:00015044       $unwind$_write_nolock      0000000180016044     libucrt:write.obj
 0001:0001505c       $unwind$?write_double_translated_ansi_nolock@@YA?AUwrite_result@?A0x9c548279@@HQEBDI@Z 000000018001605c     libucrt:write.obj
 0001:0001507c       $unwind$?write_text_utf16le_nolock@@YA?AUwrite_result@?A0x9c548279@@HQEBDI@Z 000000018001607c     libucrt:write.obj
 0001:0001507c       $unwind$?write_text_ansi_nolock@@YA?AUwrite_result@?A0x9c548279@@HQEBDI@Z 000000018001607c     libucrt:write.obj
 0001:0001509c       $unwind$?write_text_utf8_nolock@@YA?AUwrite_result@?A0x9c548279@@HQEBDI@Z 000000018001609c     libucrt:write.obj
 0001:000150c0       $xdatasym                  00000001800160c0     libucrt:log10.obj
 0001:000150cc       $unwind$_initterm_e        00000001800160cc     libucrt:initterm.obj
 0001:000150cc       $unwind$__acrt_getptd_noexit 00000001800160cc     libucrt:per_thread_data.obj
 0001:000150cc       $unwind$?TraceLoggingRegister@__vcrt_trace_logging_provider@@YAJPEBU_TlgProvider_t@1@PEBU_GUID@@P6AX1KE_K2PEAU_EVENT_FILTER_DESCRIPTOR@@PEAX@Z4@Z 00000001800160cc     libvcruntime:telemetry.obj
 0001:000150cc       $unwind$__acrt_stdio_flush_nolock 00000001800160cc     libucrt:fflush.obj
 0001:000150cc       $unwind$_RTC_Initialize    00000001800160cc     LIBCMT:_initsect_.obj
 0001:000150cc       $unwind$__vcrt_getptd_noexit 00000001800160cc     libvcruntime:per_thread_data.obj
 0001:000150cc       $unwind$__vcrt_FlsSetValue 00000001800160cc     libvcruntime:winapi_downlevel.obj
 0001:000150cc       $unwind$__acrt_FlsSetValue 00000001800160cc     libucrt:winapi_thunks.obj
 0001:000150cc       $unwind$?free_crt_array_internal@@YAXQEAPEBX_K@Z 00000001800160cc     libucrt:inittime.obj
 0001:000150cc       $unwind$_DllMainCRTStartup 00000001800160cc     LIBCMT:dll_dllmain.obj
 0001:000150cc       $unwind$??$common_lseek_nolock@_J@@YA_JH_JH@Z 00000001800160cc     libucrt:lseek.obj
 0001:000150cc       $unwind$_RTC_Terminate     00000001800160cc     LIBCMT:_initsect_.obj
 0001:000150cc       $unwind$__acrt_execute_uninitializers 00000001800160cc     libucrt:shared_initialization.obj
 0001:000150cc       $unwind$?CreateCheckBoxBinding@PluginDialogBuilder@@MEAAPEAU?$DialogItemBinding@UFarDialogItem@@@@PEAHH@Z 00000001800160cc     AutoWrap.obj
 0001:000150cc       $unwind$??R<lambda_ad1ced32f4ac17aa236e5ef05d6b3b7c>@@QEBAXXZ 00000001800160cc     libucrt:mbctype.obj
 0001:000150cc       $unwind$_exception_enabled 00000001800160cc     libucrt:libm_error.obj
 0001:000150cc       $unwind$__acrt_LocaleNameToLCID 00000001800160cc     libucrt:winapi_thunks.obj
 0001:000150dc       $unwind$fclose             00000001800160dc     libucrt:fclose.obj
 0001:00015100       $unwind$_call_matherr      0000000180016100     libucrt:libm_error.obj
 0001:00015108       $unwind$_handle_error      0000000180016108     libucrt:libm_error.obj
 0001:00015128       $unwind$__acrt_initialize_fma3 0000000180016128     libucrt:fma3_available.obj
 0001:00015130       $unwind$_log_special_common 0000000180016130     libucrt:log_special.obj
 0001:0001513c       $unwind$??$?RV<lambda_bfedae4ebbf01fab1bb6dcc6a9e276e0>@@AEAV<lambda_2fe9b910cf3cbf4a0ab98a02ba45b3ec>@@V<lambda_237c231691f317818eb88cc1d5d642d6>@@@?$__crt_seh_guarded_call@H@@QEAAH$$QEAV<lambda_bfedae4ebbf01fab1bb6dcc6a9e276e0>@@AEAV<lambda_2fe9b910cf3cbf4a0ab98a02ba45b3ec>@@$$QEAV<lambda_237c231691f317818eb88cc1d5d642d6>@@@Z 000000018001613c     libucrt:close.obj
 0001:00015160       $unwind$_raise_exc         0000000180016160     libucrt:fpexcept.obj
 0001:00015160       $unwind$?__scrt_throw_std_bad_alloc@@YAXXZ 0000000180016160     LIBCMT:throw_bad_alloc.obj
 0001:00015160       $unwind$?__scrt_throw_std_bad_array_new_length@@YAXXZ 0000000180016160     LIBCMT:throw_bad_alloc.obj
 0001:00015160       $unwind$__dcrt_lowio_initialize_console_output 0000000180016160     libucrt:initcon.obj
 0001:00015168       $xdatasym                  0000000180016168     libucrt:fpsr.obj
 0001:00015170       $unwind$_raise_exc_ex      0000000180016170     libucrt:fpexcept.obj
 0001:00015184       $unwind$_ctrlfp            0000000180016184     libucrt:fpctrl.obj
 0001:000151ac       $unwind$__GSHandlerCheckCommon 00000001800161ac     LIBCMT:_gshandler_.obj
 0001:000151b8       $xdatasym                  00000001800161b8     LIBCMT:_amdsecgs_.obj
 0001:000151bc       $unwind$_IsNonwritableInCurrentImage 00000001800161bc     LIBCMT:pesect.obj
 0001:000151e0       $unwind$__report_securityfailure 00000001800161e0     LIBCMT:gs_report.obj
 0001:000151e8       $unwind$_putwch_nolock     00000001800161e8     libucrt:putwch.obj
 0001:000151e8       $unwind$__report_gsfailure 00000001800161e8     LIBCMT:gs_report.obj
 0001:000151f0       $unwind$capture_current_context 00000001800161f0     LIBCMT:gs_report.obj
 0001:000151fc       $unwind$capture_previous_context 00000001800161fc     LIBCMT:gs_report.obj
 0001:00015208       $xdatasym                  0000000180016208     libvcruntime:memcpy.obj
 0001:00015210       $xdatasym                  0000000180016210     libvcruntime:memcmp.obj
 0001:00015310       .edata                     0000000180016310     AutoWrap.exp
 0001:00015338       rgpv                       0000000180016338     AutoWrap.exp
 0001:0001534c       rgszName                   000000018001634c     AutoWrap.exp
 0001:00015360       rgwOrd                     0000000180016360     AutoWrap.exp
 0001:0001536a       szName                     000000018001636a     AutoWrap.exp
 0001:00015377       $N00001                    0000000180016377     AutoWrap.exp
 0001:00015386       $N00002                    0000000180016386     AutoWrap.exp
 0001:00015395       $N00003                    0000000180016395     AutoWrap.exp
 0001:0001539b       $N00004                    000000018001639b     AutoWrap.exp
 0001:000153af       $N00005                    00000001800163af     AutoWrap.exp
 0002:00000030       ?_Tlg_Microsoft_CRTProviderProv@@3U_TlgProvider_t@__vcrt_trace_logging_provider@@A 0000000180017030     libvcruntime:telemetry.obj
 0002:00000080       ?__vcrt_flsindex@@3KA      0000000180017080     libvcruntime:per_thread_data.obj
 0002:00000088       __acrt_flsindex            0000000180017088     libucrt:per_thread_data.obj
 0002:000001fc       errno_no_memory            00000001800171fc     libucrt:errno.obj
 0002:00000200       doserrno_no_memory         0000000180017200     libucrt:errno.obj
 0002:00000440       __rgctypeflag              0000000180017440     libucrt:mbctype.obj
 0002:00000450       __rgcode_page_info         0000000180017450     libucrt:mbctype.obj
 0002:00000920       ?dazSupported@?1??_ctrlfp@@9@9 0000000180017920     libucrt:fpctrl.obj
 0002:000011f0       ?Info@@3UPluginStartupInfo@@A 00000001800181f0     AutoWrap.obj
 0002:00001300       ?FSF@@3UFarStandardFunctions@@A 0000000180018300     AutoWrap.obj
 0002:00001480       ?PluginMenuStrings@?1??GetPluginInfoW@@9@4PAPEB_WA 0000000180018480     AutoWrap.obj
 0002:00001488       ?Reenter@?1??ProcessEditorInputW@@9@4HA 0000000180018488     AutoWrap.obj
 0002:0000148c       ?__proc_attached@@3HA      000000018001848c     LIBCMT:dll_dllmain.obj
 0002:000014a0       ?module_local_atexit_table@@3U_onexit_table_t@@A 00000001800184a0     LIBCMT:utility.obj
 0002:000014b8       ?module_local_at_quick_exit_table@@3U_onexit_table_t@@A 00000001800184b8     LIBCMT:utility.obj
 0002:000014d0       ?is_initialized_as_dll@@3_NA 00000001800184d0     LIBCMT:utility.obj
 0002:00001510       ?module_handles@@3PAPEAUHINSTANCE__@@A 0000000180018510     libvcruntime:winapi_downlevel.obj
 0002:00001530       ?encoded_function_pointers@@3PAPEAXA 0000000180018530     libvcruntime:winapi_downlevel.obj
 0002:00001580       ?__vcrt_startup_thread_ptd@@3U__vcrt_ptd@@A 0000000180018580     libvcruntime:per_thread_data.obj
 0002:000015f8       __vcrt_lock_table          00000001800185f8     libvcruntime:locks.obj
 0002:00001620       __vcrt_locks_initialized   0000000180018620     libvcruntime:locks.obj
 0002:00001678       ?heap@@3V_HeapManager@@A   0000000180018678     libvcruntime:undname.obj
 0002:000016a0       __acrt_new_handler         00000001800186a0     libucrt:new_handler.obj
 0002:000016a8       c_termination_complete     00000001800186a8     libucrt:exit.obj
 0002:000016b0       thread_local_exit_callback_func 00000001800186b0     libucrt:exit.obj
 0002:000016b8       ?c_exit_complete@?5??common_exit@@YAXHW4_crt_exit_cleanup_mode@@W4_crt_exit_return_mode@@@Z@4_NA 00000001800186b8     libucrt:exit.obj
 0002:000016c0       ?program_name@?5???$common_configure_argv@D@@YAHW4_crt_argv_mode@@@Z@4PADA 00000001800186c0     libucrt:argv_parsing.obj
 0002:00001830       __acrt_lock_table          0000000180018830     libucrt:locks.obj
 0002:00001a38       __acrt_locks_initialized   0000000180018a38     libucrt:locks.obj
 0002:00001a40       module_handles             0000000180018a40     libucrt:winapi_thunks.obj
 0002:00001ae0       encoded_function_pointers  0000000180018ae0     libucrt:winapi_thunks.obj
 0002:00001be0       ?state_cache@?1??__acrt_is_packaged_app@@9@4JA 0000000180018be0     libucrt:winapi_thunks.obj
 0002:00001be8       __acrt_invalid_parameter_handler 0000000180018be8     libucrt:invalid_parameter.obj
 0002:00001c04       fSystemSet                 0000000180018c04     libucrt:mbctype.obj
 0002:00001c10       ?initialized@?1??__acrt_initialize_multibyte@@9@4_NA 0000000180018c10     libucrt:mbctype.obj
 0002:00002058       ctrlc_action               0000000180019058     libucrt:signal.obj
 0002:00002060       ctrlbreak_action           0000000180019060     libucrt:signal.obj
 0002:00002068       abort_action               0000000180019068     libucrt:signal.obj
 0002:00002070       term_action                0000000180019070     libucrt:signal.obj
 0002:00002078       user_matherr               0000000180019078     libucrt:matherr.obj
 0002:00002090       __acrt_global_new_mode     0000000180019090     libucrt:new_mode.obj
 0002:000020b0       __acrt_app_type            00000001800190b0     libucrt:report_runtime_error.obj
 0002:000020c0       GS_ExceptionRecord         00000001800190c0     LIBCMT:gs_report.obj
 0002:00002160       GS_ContextRecord           0000000180019160     LIBCMT:gs_report.obj
 0003:00000000       $pdata$?TraceLoggingRegister@__vcrt_trace_logging_provider@@YAJPEBU_TlgProvider_t@1@PEBU_GUID@@P6AX1KE_K2PEAU_EVENT_FILTER_DESCRIPTOR@@PEAX@Z4@Z 000000018001a000     libvcruntime:telemetry.obj
 0003:0000000c       $pdata$?_TlgEnableCallback@__vcrt_trace_logging_provider@@YAXPEBU_GUID@@KE_K1PEAU_EVENT_FILTER_DESCRIPTOR@@PEAX@Z 000000018001a00c     libvcruntime:telemetry.obj
 0003:00000018       $pdata$?_TlgWrite@__vcrt_trace_logging_provider@@YAJPEBU_TlgProvider_t@1@PEFBXPEBU_GUID@@2IPEAU_EVENT_DATA_DESCRIPTOR@@@Z 000000018001a018     libvcruntime:telemetry.obj
 0003:00000030       $pdata$??0PluginIntEditFieldBinding@@QEAA@AEBUPluginStartupInfo@@PEAPEAXHPEAHH@Z 000000018001a030     AutoWrap.obj
 0003:0000003c       $pdata$??0PluginUIntEditFieldBinding@@QEAA@AEBUPluginStartupInfo@@PEAPEAXHPEAIH@Z 000000018001a03c     AutoWrap.obj
 0003:00000048       $pdata$??1?$DialogBuilderBase@UFarDialogItem@@@@MEAA@XZ 000000018001a048     AutoWrap.obj
 0003:00000054       $pdata$0$??1?$DialogBuilderBase@UFarDialogItem@@@@MEAA@XZ 000000018001a054     AutoWrap.obj
 0003:00000060       $pdata$1$??1?$DialogBuilderBase@UFarDialogItem@@@@MEAA@XZ 000000018001a060     AutoWrap.obj
 0003:0000006c       $pdata$??_G?$DialogBuilderBase@UFarDialogItem@@@@MEAAPEAXI@Z 000000018001a06c     AutoWrap.obj
 0003:00000078       $pdata$??_G?$DialogItemBinding@UFarDialogItem@@@@UEAAPEAXI@Z 000000018001a078     AutoWrap.obj
 0003:00000084       $pdata$??_GPluginCheckBoxBinding@@UEAAPEAXI@Z 000000018001a084     AutoWrap.obj
 0003:00000084       $pdata$??_GPluginEditFieldBinding@@UEAAPEAXI@Z 000000018001a084     AutoWrap.obj
 0003:00000090       $pdata$??_GPluginDialogBuilder@@UEAAPEAXI@Z 000000018001a090     AutoWrap.obj
 0003:0000009c       $pdata$??_GPluginIntEditFieldBinding@@UEAAPEAXI@Z 000000018001a09c     AutoWrap.obj
 0003:0000009c       $pdata$??_GPluginUIntEditFieldBinding@@UEAAPEAXI@Z 000000018001a09c     AutoWrap.obj
 0003:000000a8       $pdata$??_GPluginRadioButtonBinding@@UEAAPEAXI@Z 000000018001a0a8     AutoWrap.obj
 0003:000000b4       $pdata$?AddButtons@?$DialogBuilderBase@UFarDialogItem@@@@QEAAXHPEBHHH@Z 000000018001a0b4     AutoWrap.obj
 0003:000000c0       $pdata$3$?AddButtons@?$DialogBuilderBase@UFarDialogItem@@@@QEAAXHPEBHHH@Z 000000018001a0c0     AutoWrap.obj
 0003:000000cc       $pdata$4$?AddButtons@?$DialogBuilderBase@UFarDialogItem@@@@QEAAXHPEBHHH@Z 000000018001a0cc     AutoWrap.obj
 0003:000000d8       $pdata$?AddDialogItem@?$DialogBuilderBase@UFarDialogItem@@@@IEAAPEAUFarDialogItem@@W4FARDIALOGITEMTYPES@@PEB_W@Z 000000018001a0d8     AutoWrap.obj
 0003:000000e4       $pdata$?AddIntEditField@PluginDialogBuilder@@UEAAPEAUFarDialogItem@@PEAHH@Z 000000018001a0e4     AutoWrap.obj
 0003:000000f0       $pdata$?AddTextAfter@?$DialogBuilderBase@UFarDialogItem@@@@QEAAPEAUFarDialogItem@@PEAU2@PEB_WH@Z 000000018001a0f0     AutoWrap.obj
 0003:000000fc       $pdata$?AddUIntEditField@PluginDialogBuilder@@UEAAPEAUFarDialogItem@@PEAIH@Z 000000018001a0fc     AutoWrap.obj
 0003:00000108       $pdata$?CreateCheckBoxBinding@PluginDialogBuilder@@MEAAPEAU?$DialogItemBinding@UFarDialogItem@@@@PEAHH@Z 000000018001a108     AutoWrap.obj
 0003:00000114       $pdata$?CreateRadioButtonBinding@PluginDialogBuilder@@MEAAPEAU?$DialogItemBinding@UFarDialogItem@@@@PEAH@Z 000000018001a114     AutoWrap.obj
 0003:00000120       $pdata$?DoShowDialog@PluginDialogBuilder@@MEAA_JXZ 000000018001a120     AutoWrap.obj
 0003:0000012c       $pdata$?GetCommaWord@@YAPEB_WPEB_WPEA_W@Z 000000018001a12c     AutoWrap.obj
 0003:00000138       $pdata$4$?GetCommaWord@@YAPEB_WPEB_WPEA_W@Z 000000018001a138     AutoWrap.obj
 0003:00000144       $pdata$6$?GetCommaWord@@YAPEB_WPEB_WPEA_W@Z 000000018001a144     AutoWrap.obj
 0003:00000150       $pdata$?InitDialogItem@PluginDialogBuilder@@MEAAXPEAUFarDialogItem@@PEB_W@Z 000000018001a150     AutoWrap.obj
 0003:0000015c       $pdata$?ItemWidth@?$DialogBuilderBase@UFarDialogItem@@@@IEAA_JAEBUFarDialogItem@@@Z 000000018001a15c     AutoWrap.obj
 0003:00000168       $pdata$?MaxTextWidth@?$DialogBuilderBase@UFarDialogItem@@@@IEAA_JXZ 000000018001a168     AutoWrap.obj
 0003:00000174       $pdata$1$?MaxTextWidth@?$DialogBuilderBase@UFarDialogItem@@@@IEAA_JXZ 000000018001a174     AutoWrap.obj
 0003:00000180       $pdata$2$?MaxTextWidth@?$DialogBuilderBase@UFarDialogItem@@@@IEAA_JXZ 000000018001a180     AutoWrap.obj
 0003:0000018c       $pdata$?ReallocDialogItems@?$DialogBuilderBase@UFarDialogItem@@@@IEAAXXZ 000000018001a18c     AutoWrap.obj
 0003:00000198       $pdata$?SaveValue@PluginCheckBoxBinding@@UEAAXPEAUFarDialogItem@@H@Z 000000018001a198     AutoWrap.obj
 0003:000001a4       $pdata$?SaveValue@PluginEditFieldBinding@@UEAAXPEAUFarDialogItem@@H@Z 000000018001a1a4     AutoWrap.obj
 0003:000001b0       $pdata$?SaveValue@PluginIntEditFieldBinding@@UEAAXPEAUFarDialogItem@@H@Z 000000018001a1b0     AutoWrap.obj
 0003:000001bc       $pdata$?SaveValue@PluginRadioButtonBinding@@UEAAXPEAUFarDialogItem@@H@Z 000000018001a1bc     AutoWrap.obj
 0003:000001c8       $pdata$?SaveValue@PluginUIntEditFieldBinding@@UEAAXPEAUFarDialogItem@@H@Z 000000018001a1c8     AutoWrap.obj
 0003:000001d4       $pdata$?SaveValues@?$DialogBuilderBase@UFarDialogItem@@@@IEAAXXZ 000000018001a1d4     AutoWrap.obj
 0003:000001e0       $pdata$1$?SaveValues@?$DialogBuilderBase@UFarDialogItem@@@@IEAAXXZ 000000018001a1e0     AutoWrap.obj
 0003:000001ec       $pdata$2$?SaveValues@?$DialogBuilderBase@UFarDialogItem@@@@IEAAXXZ 000000018001a1ec     AutoWrap.obj
 0003:000001f8       $pdata$?UpdateBorderSize@?$DialogBuilderBase@UFarDialogItem@@@@IEAAXXZ 000000018001a1f8     AutoWrap.obj
 0003:00000204       $pdata$GetGlobalInfoW      000000018001a204     AutoWrap.obj
 0003:00000210       $pdata$GetPluginInfoW      000000018001a210     AutoWrap.obj
 0003:0000021c       $pdata$OpenW               000000018001a21c     AutoWrap.obj
 0003:00000228       $pdata$ProcessEditorInputW 000000018001a228     AutoWrap.obj
 0003:00000234       $pdata$4$ProcessEditorInputW 000000018001a234     AutoWrap.obj
 0003:00000240       $pdata$6$ProcessEditorInputW 000000018001a240     AutoWrap.obj
 0003:0000024c       $pdata$7$ProcessEditorInputW 000000018001a24c     AutoWrap.obj
 0003:00000258       $pdata$SetStartupInfoW     000000018001a258     AutoWrap.obj
 0003:00000264       $pdata$??2@YAPEAX_K@Z      000000018001a264     LIBCMT:new_scalar.obj
 0003:00000270       $pdata$?dllmain_crt_dispatch@@YAHQEAUHINSTANCE__@@KQEAX@Z 000000018001a270     LIBCMT:dll_dllmain.obj
 0003:0000027c       $pdata$?dllmain_crt_process_attach@@YAHQEAUHINSTANCE__@@QEAX@Z 000000018001a27c     LIBCMT:dll_dllmain.obj
 0003:00000288       $pdata$?dllmain_crt_process_detach@@YAH_N@Z 000000018001a288     LIBCMT:dll_dllmain.obj
 0003:00000294       $pdata$?dllmain_dispatch@@YAHQEAUHINSTANCE__@@KQEAX@Z 000000018001a294     LIBCMT:dll_dllmain.obj
 0003:000002a0       $pdata$?dllmain_raw@@YAHQEAUHINSTANCE__@@KQEAX@Z 000000018001a2a0     LIBCMT:dll_dllmain.obj
 0003:000002ac       $pdata$_DllMainCRTStartup  000000018001a2ac     LIBCMT:dll_dllmain.obj
 0003:000002b8       $pdata$??0bad_alloc@std@@QEAA@AEBV01@@Z 000000018001a2b8     LIBCMT:throw_bad_alloc.obj
 0003:000002c4       $pdata$??0bad_array_new_length@std@@QEAA@AEBV01@@Z 000000018001a2c4     LIBCMT:throw_bad_alloc.obj
 0003:000002d0       $pdata$??0exception@std@@QEAA@AEBV01@@Z 000000018001a2d0     LIBCMT:throw_bad_alloc.obj
 0003:000002dc       $pdata$??_Gexception@std@@UEAAPEAXI@Z 000000018001a2dc     LIBCMT:throw_bad_alloc.obj
 0003:000002dc       $pdata$??_Gbad_array_new_length@std@@UEAAPEAXI@Z 000000018001a2dc     LIBCMT:throw_bad_alloc.obj
 0003:000002dc       $pdata$??_Gbad_alloc@std@@UEAAPEAXI@Z 000000018001a2dc     LIBCMT:throw_bad_alloc.obj
 0003:000002e8       $pdata$?__scrt_throw_std_bad_alloc@@YAXXZ 000000018001a2e8     LIBCMT:throw_bad_alloc.obj
 0003:000002f4       $pdata$?__scrt_throw_std_bad_array_new_length@@YAXXZ 000000018001a2f4     LIBCMT:throw_bad_alloc.obj
 0003:00000300       $pdata$__scrt_acquire_startup_lock 000000018001a300     LIBCMT:utility.obj
 0003:0000030c       $pdata$__scrt_dllmain_after_initialize_c 000000018001a30c     LIBCMT:utility.obj
 0003:00000318       $pdata$__scrt_dllmain_before_initialize_c 000000018001a318     LIBCMT:utility.obj
 0003:00000324       $pdata$__scrt_dllmain_crt_thread_attach 000000018001a324     LIBCMT:utility.obj
 0003:00000330       $pdata$__scrt_dllmain_crt_thread_detach 000000018001a330     LIBCMT:utility.obj
 0003:0000033c       $pdata$__scrt_dllmain_exception_filter 000000018001a33c     LIBCMT:utility.obj
 0003:00000348       $pdata$__scrt_dllmain_uninitialize_c 000000018001a348     LIBCMT:utility.obj
 0003:00000354       $pdata$__scrt_dllmain_uninitialize_critical 000000018001a354     LIBCMT:utility.obj
 0003:00000360       $pdata$__scrt_initialize_crt 000000018001a360     LIBCMT:utility.obj
 0003:0000036c       $pdata$__scrt_initialize_onexit_tables 000000018001a36c     LIBCMT:utility.obj
 0003:00000378       $pdata$__scrt_is_nonwritable_in_current_image 000000018001a378     LIBCMT:utility.obj
 0003:00000384       $pdata$__scrt_release_startup_lock 000000018001a384     LIBCMT:utility.obj
 0003:00000390       $pdata$__scrt_uninitialize_crt 000000018001a390     LIBCMT:utility.obj
 0003:0000039c       $pdata$_onexit             000000018001a39c     LIBCMT:utility.obj
 0003:000003a8       $pdata$atexit              000000018001a3a8     LIBCMT:utility.obj
 0003:000003b4       $pdata$__security_init_cookie 000000018001a3b4     LIBCMT:gs_support.obj
 0003:000003c0       $pdata$__scrt_initialize_default_local_stdio_options 000000018001a3c0     LIBCMT:default_local_stdio_options.obj
 0003:000003cc       $pdata$__scrt_fastfail     000000018001a3cc     LIBCMT:utility_desktop.obj
 0003:000003d8       $pdata$_RTC_Initialize     000000018001a3d8     LIBCMT:_initsect_.obj
 0003:000003e4       $pdata$_RTC_Terminate      000000018001a3e4     LIBCMT:_initsect_.obj
 0003:000003f0       $pdata$??_Gtype_info@@UEAAPEAXI@Z 000000018001a3f0     LIBCMT:std_type_info_static.obj
 0003:000003fc       $pdata$__isa_available_init 000000018001a3fc     LIBCMT:_cpu_disp_.obj
 0003:00000408       $pdata$wcschr              000000018001a408     libvcruntime:wcschr.obj
 0003:00000420       $pdata$__telemetry_main_invoke_trigger 000000018001a420     libvcruntime:telemetry.obj
 0003:0000042c       $pdata$__telemetry_main_return_trigger 000000018001a42c     libvcruntime:telemetry.obj
 0003:00000438       $pdata$__vcrt_uninitialize_telemetry_provider 000000018001a438     libvcruntime:telemetry.obj
 0003:00000444       $pdata$__C_specific_handler 000000018001a444     libvcruntime:_chandler_.obj
 0003:00000450       $pdata$__std_exception_copy 000000018001a450     libvcruntime:std_exception.obj
 0003:0000045c       $pdata$__std_exception_destroy 000000018001a45c     libvcruntime:std_exception.obj
 0003:00000468       $pdata$_CxxThrowException  000000018001a468     libvcruntime:throw.obj
 0003:00000474       $pdata$__vcrt_initialize   000000018001a474     libvcruntime:initialization.obj
 0003:00000480       $pdata$__vcrt_thread_attach 000000018001a480     libvcruntime:initialization.obj
 0003:0000048c       $pdata$__vcrt_thread_detach 000000018001a48c     libvcruntime:initialization.obj
 0003:00000498       $pdata$__vcrt_uninitialize 000000018001a498     libvcruntime:initialization.obj
 0003:000004a4       $pdata$__vcrt_uninitialize_critical 000000018001a4a4     libvcruntime:initialization.obj
 0003:000004b0       $pdata$__std_type_info_destroy_list 000000018001a4b0     libvcruntime:std_type_info.obj
 0003:000004bc       $pdata$?try_get_function@@YAPEAXW4function_id@?A0x49c8dc86@@QEBDQEBW4module_id@2@2@Z 000000018001a4bc     libvcruntime:winapi_downlevel.obj
 0003:000004c8       $pdata$__vcrt_EventRegister 000000018001a4c8     libvcruntime:winapi_downlevel.obj
 0003:000004d4       $pdata$__vcrt_EventSetInformation 000000018001a4d4     libvcruntime:winapi_downlevel.obj
 0003:000004e0       $pdata$__vcrt_EventUnregister 000000018001a4e0     libvcruntime:winapi_downlevel.obj
 0003:000004ec       $pdata$__vcrt_EventWriteTransfer 000000018001a4ec     libvcruntime:winapi_downlevel.obj
 0003:000004f8       $pdata$__vcrt_FlsAlloc     000000018001a4f8     libvcruntime:winapi_downlevel.obj
 0003:00000504       $pdata$__vcrt_FlsFree      000000018001a504     libvcruntime:winapi_downlevel.obj
 0003:00000510       $pdata$__vcrt_FlsGetValue  000000018001a510     libvcruntime:winapi_downlevel.obj
 0003:0000051c       $pdata$__vcrt_FlsSetValue  000000018001a51c     libvcruntime:winapi_downlevel.obj
 0003:00000528       $pdata$__vcrt_InitializeCriticalSectionEx 000000018001a528     libvcruntime:winapi_downlevel.obj
 0003:00000534       $pdata$__vcrt_initialize_winapi_thunks 000000018001a534     libvcruntime:winapi_downlevel.obj
 0003:00000540       $pdata$__vcrt_uninitialize_winapi_thunks 000000018001a540     libvcruntime:winapi_downlevel.obj
 0003:0000057c       $pdata$__vcrt_freefls      000000018001a57c     libvcruntime:per_thread_data.obj
 0003:00000588       $pdata$__vcrt_freeptd      000000018001a588     libvcruntime:per_thread_data.obj
 0003:00000594       $pdata$__vcrt_getptd_noexit 000000018001a594     libvcruntime:per_thread_data.obj
 0003:000005a0       $pdata$__vcrt_initialize_ptd 000000018001a5a0     libvcruntime:per_thread_data.obj
 0003:000005ac       $pdata$__vcrt_uninitialize_ptd 000000018001a5ac     libvcruntime:per_thread_data.obj
 0003:000005b8       $pdata$__vcrt_initialize_locks 000000018001a5b8     libvcruntime:locks.obj
 0003:000005c4       $pdata$__vcrt_uninitialize_locks 000000018001a5c4     libvcruntime:locks.obj
 0003:000005d0       $pdata$??0_LocaleUpdate@@QEAA@QEAU__crt_locale_pointers@@@Z 000000018001a5d0     libucrt:_wctype.obj
 0003:000005dc       $pdata$_isleadbyte_l       000000018001a5dc     libucrt:_wctype.obj
 0003:000005e8       $pdata$_callnewh           000000018001a5e8     libucrt:new_handler.obj
 0003:000005f4       $pdata$_query_new_handler  000000018001a5f4     libucrt:new_handler.obj
 0003:00000600       $pdata$_initterm           000000018001a600     libucrt:initterm.obj
 0003:0000060c       $pdata$_initterm_e         000000018001a60c     libucrt:initterm.obj
 0003:00000618       $pdata$_seh_filter_exe     000000018001a618     libucrt:exception_filter.obj
 0003:00000624       $pdata$?common_exit@@YAXHW4_crt_exit_cleanup_mode@@W4_crt_exit_return_mode@@@Z 000000018001a624     libucrt:exit.obj
 0003:00000630       $pdata$?exit_or_terminate_process@@YAXI@Z 000000018001a630     libucrt:exit.obj
 0003:0000063c       $pdata$?try_cor_exit_process@@YAXI@Z 000000018001a63c     libucrt:exit.obj
 0003:00000648       $pdata$??$parse_command_line@D@@YAXPEADPEAPEAD0PEA_K2@Z 000000018001a648     libucrt:argv_parsing.obj
 0003:00000654       $pdata$__acrt_allocate_buffer_for_argv 000000018001a654     libucrt:argv_parsing.obj
 0003:00000660       $pdata$_configure_narrow_argv 000000018001a660     libucrt:argv_parsing.obj
 0003:0000066c       $pdata$??$common_initialize_environment_nolock@D@@YAHXZ 000000018001a66c     libucrt:environment_initialization.obj
 0003:00000678       $pdata$??$create_environment@D@@YAQEAPEADQEAD@Z 000000018001a678     libucrt:environment_initialization.obj
 0003:00000684       $pdata$??$free_environment@_W@@YAXQEAPEA_W@Z 000000018001a684     libucrt:environment_initialization.obj
 0003:00000684       $pdata$??$free_environment@D@@YAXQEAPEAD@Z 000000018001a684     libucrt:environment_initialization.obj
 0003:00000690       $pdata$??$uninitialize_environment_internal@D@@YAXAEAPEAPEAD@Z 000000018001a690     libucrt:environment_initialization.obj
 0003:0000069c       $pdata$??$uninitialize_environment_internal@_W@@YAXAEAPEAPEA_W@Z 000000018001a69c     libucrt:environment_initialization.obj
 0003:000006a8       $pdata$__dcrt_uninitialize_environments_nolock 000000018001a6a8     libucrt:environment_initialization.obj
 0003:000006b4       $pdata$??$?RV<lambda_b8c45f8f788dd370798f47cfe8ac3a86>@@AEAV<lambda_4e60a939b0d047cfe11ddc22648dfba9>@@V<lambda_332c3edc96d0294ec56c57d38c1cdfd5>@@@?$__crt_seh_guarded_call@H@@QEAAH$$QEAV<lambda_b8c45f8f788dd370798f47cfe8ac3a86>@@AEAV<lambda_4e60a939b0d047cfe11ddc22648dfba9>@@$$QEAV<lambda_332c3edc96d0294ec56c57d38c1cdfd5>@@@Z 000000018001a6b4     libucrt:onexit.obj
 0003:000006c0       $pdata$??$?RV<lambda_e24bbb7b643b32fcea6fa61b31d4c984>@@AEAV<lambda_275893d493268fdec8709772e3fcec0e>@@V<lambda_9d71df4d7cf3f480f8d633942495c3b0>@@@?$__crt_seh_guarded_call@H@@QEAAH$$QEAV<lambda_e24bbb7b643b32fcea6fa61b31d4c984>@@AEAV<lambda_275893d493268fdec8709772e3fcec0e>@@$$QEAV<lambda_9d71df4d7cf3f480f8d633942495c3b0>@@@Z 000000018001a6c0     libucrt:onexit.obj
 0003:000006cc       $pdata$??R<lambda_4e60a939b0d047cfe11ddc22648dfba9>@@QEBAHXZ 000000018001a6cc     libucrt:onexit.obj
 0003:000006d8       $pdata$_execute_onexit_table 000000018001a6d8     libucrt:onexit.obj
 0003:000006e4       $pdata$_register_onexit_function 000000018001a6e4     libucrt:onexit.obj
 0003:000006f0       $pdata$initialize_c        000000018001a6f0     libucrt:initialization.obj
 0003:000006fc       $pdata$uninitialize_environment 000000018001a6fc     libucrt:initialization.obj
 0003:00000708       $pdata$initialize_pointers 000000018001a708     libucrt:initialization.obj
 0003:00000714       $pdata$uninitialize_allocated_memory 000000018001a714     libucrt:initialization.obj
 0003:00000720       $pdata$__acrt_thread_attach 000000018001a720     libucrt:initialization.obj
 0003:0000072c       $pdata$__acrt_thread_detach 000000018001a72c     libucrt:initialization.obj
 0003:00000738       $pdata$__acrt_uninitialize_critical 000000018001a738     libucrt:initialization.obj
 0003:00000744       $pdata$terminate           000000018001a744     libucrt:terminate.obj
 0003:00000750       $pdata$strcpy_s            000000018001a750     libucrt:strcpy_s.obj
 0003:0000075c       $pdata$_free_base          000000018001a75c     libucrt:free_base.obj
 0003:00000768       $pdata$_malloc_base        000000018001a768     libucrt:malloc_base.obj
 0003:00000774       $pdata$abort               000000018001a774     libucrt:abort.obj
 0003:00000780       $pdata$_calloc_base        000000018001a780     libucrt:calloc_base.obj
 0003:0000078c       $pdata$iswctype            000000018001a78c     libucrt:iswctype.obj
 0003:00000798       $pdata$??$?RV<lambda_46352004c1216016012b18bd6f87e700>@@AEAV<lambda_3bd07e1a1191394380780325891bf33f>@@V<lambda_334532d3f185bcaa59b5be82d7d22bff>@@@?$__crt_seh_guarded_call@X@@QEAAX$$QEAV<lambda_46352004c1216016012b18bd6f87e700>@@AEAV<lambda_3bd07e1a1191394380780325891bf33f>@@$$QEAV<lambda_334532d3f185bcaa59b5be82d7d22bff>@@@Z 000000018001a798     libucrt:per_thread_data.obj
 0003:000007a4       $pdata$??$?RV<lambda_5e887d1dcbef67a5eb4283622ba103bf>@@AEAV<lambda_4466841279450cc726390878d4a41900>@@V<lambda_341c25c0346d94847f1f3c463c57e077>@@@?$__crt_seh_guarded_call@X@@QEAAX$$QEAV<lambda_5e887d1dcbef67a5eb4283622ba103bf>@@AEAV<lambda_4466841279450cc726390878d4a41900>@@$$QEAV<lambda_341c25c0346d94847f1f3c463c57e077>@@@Z 000000018001a7a4     libucrt:per_thread_data.obj
 0003:000007b0       $pdata$??$?RV<lambda_72d1df2b273a38828b1ce30cbf4cdab5>@@AEAV<lambda_876a65b173b8412d3a47c70a915b0cf4>@@V<lambda_41932305e351933ebe8f8be3ed8bb5dc>@@@?$__crt_seh_guarded_call@X@@QEAAX$$QEAV<lambda_72d1df2b273a38828b1ce30cbf4cdab5>@@AEAV<lambda_876a65b173b8412d3a47c70a915b0cf4>@@$$QEAV<lambda_41932305e351933ebe8f8be3ed8bb5dc>@@@Z 000000018001a7b0     libucrt:per_thread_data.obj
 0003:000007bc       $pdata$??$?RV<lambda_fb3a7dec4e47f37f22dae91bb15c9095>@@AEAV<lambda_698284760c8add0bfb0756c19673e34b>@@V<lambda_dfb8eca1e75fef3034a8fb18dd509707>@@@?$__crt_seh_guarded_call@X@@QEAAX$$QEAV<lambda_fb3a7dec4e47f37f22dae91bb15c9095>@@AEAV<lambda_698284760c8add0bfb0756c19673e34b>@@$$QEAV<lambda_dfb8eca1e75fef3034a8fb18dd509707>@@@Z 000000018001a7bc     libucrt:per_thread_data.obj
 0003:000007c8       $pdata$?construct_ptd_array@@YAXQEAU__acrt_ptd@@@Z 000000018001a7c8     libucrt:per_thread_data.obj
 0003:000007d4       $pdata$?destroy_fls@@YAXPEAX@Z 000000018001a7d4     libucrt:per_thread_data.obj
 0003:000007e0       $pdata$?destroy_ptd_array@@YAXQEAU__acrt_ptd@@@Z 000000018001a7e0     libucrt:per_thread_data.obj
 0003:000007ec       $pdata$?replace_current_thread_locale_nolock@@YAXQEAU__acrt_ptd@@QEAU__crt_locale_data@@@Z 000000018001a7ec     libucrt:per_thread_data.obj
 0003:000007f8       $pdata$__acrt_freeptd      000000018001a7f8     libucrt:per_thread_data.obj
 0003:00000804       $pdata$__acrt_getptd       000000018001a804     libucrt:per_thread_data.obj
 0003:00000810       $pdata$__acrt_getptd_noexit 000000018001a810     libucrt:per_thread_data.obj
 0003:0000081c       $pdata$__acrt_initialize_ptd 000000018001a81c     libucrt:per_thread_data.obj
 0003:00000828       $pdata$__acrt_uninitialize_ptd 000000018001a828     libucrt:per_thread_data.obj
 0003:00000834       $pdata$__acrt_update_locale_info 000000018001a834     libucrt:locale_update.obj
 0003:00000840       $pdata$__acrt_update_multibyte_info 000000018001a840     libucrt:locale_update.obj
 0003:0000084c       $pdata$__acrt_uninitialize_locale 000000018001a84c     libucrt:wsetlocale.obj
 0003:00000858       $pdata$__acrt_initialize_locks 000000018001a858     libucrt:locks.obj
 0003:00000864       $pdata$__acrt_uninitialize_locks 000000018001a864     libucrt:locks.obj
 0003:00000870       $pdata$?try_get_function@@YAPEAXW4function_id@?A0x63058377@@QEBDQEBW4module_id@2@2@Z 000000018001a870     libucrt:winapi_thunks.obj
 0003:0000087c       $pdata$__acrt_FlsAlloc     000000018001a87c     libucrt:winapi_thunks.obj
 0003:00000888       $pdata$__acrt_FlsFree      000000018001a888     libucrt:winapi_thunks.obj
 0003:00000894       $pdata$__acrt_FlsGetValue  000000018001a894     libucrt:winapi_thunks.obj
 0003:000008a0       $pdata$__acrt_FlsSetValue  000000018001a8a0     libucrt:winapi_thunks.obj
 0003:000008ac       $pdata$__acrt_InitializeCriticalSectionEx 000000018001a8ac     libucrt:winapi_thunks.obj
 0003:000008b8       $pdata$__acrt_LCMapStringEx 000000018001a8b8     libucrt:winapi_thunks.obj
 0003:000008c4       $pdata$__acrt_LocaleNameToLCID 000000018001a8c4     libucrt:winapi_thunks.obj
 0003:000008d0       $pdata$__acrt_initialize_winapi_thunks 000000018001a8d0     libucrt:winapi_thunks.obj
 0003:000008dc       $pdata$__acrt_is_packaged_app 000000018001a8dc     libucrt:winapi_thunks.obj
 0003:000008e8       $pdata$__acrt_uninitialize_winapi_thunks 000000018001a8e8     libucrt:winapi_thunks.obj
 0003:000008f4       $pdata$__acrt_call_reportfault 000000018001a8f4     libucrt:invalid_parameter.obj
 0003:00000900       $pdata$_invalid_parameter  000000018001a900     libucrt:invalid_parameter.obj
 0003:0000090c       $pdata$_invalid_parameter_noinfo 000000018001a90c     libucrt:invalid_parameter.obj
 0003:00000918       $pdata$_invoke_watson      000000018001a918     libucrt:invalid_parameter.obj
 0003:00000924       $pdata$__acrt_errno_map_os_error 000000018001a924     libucrt:errno.obj
 0003:00000930       $pdata$__doserrno          000000018001a930     libucrt:errno.obj
 0003:0000093c       $pdata$_errno              000000018001a93c     libucrt:errno.obj
 0003:00000948       $pdata$??$common_expand_argv_wildcards@D@@YAHQEAPEADQEAPEAPEAD@Z 000000018001a948     libucrt:argv_wildcards.obj
 0003:00000954       $pdata$??$copy_and_add_argument_to_buffer@D@@YAHQEBD0_KAEAV?$argument_list@D@?A0xca0879c4@@@Z 000000018001a954     libucrt:argv_wildcards.obj
 0003:00000960       $pdata$??$expand_argument_wildcards@D@@YAHQEAD0AEAV?$argument_list@D@?A0xca0879c4@@@Z 000000018001a960     libucrt:argv_wildcards.obj
 0003:0000096c       $pdata$?expand_if_necessary@?$argument_list@D@?A0xca0879c4@@AEAAHXZ 000000018001a96c     libucrt:argv_wildcards.obj
 0003:00000978       $pdata$??$?RV<lambda_99476a1ad63dd22509b5d3e65b0ffc95>@@AEAV<lambda_ad1ced32f4ac17aa236e5ef05d6b3b7c>@@V<lambda_f7424dd8d45958661754dc4f2697e9c3>@@@?$__crt_seh_guarded_call@X@@QEAAX$$QEAV<lambda_99476a1ad63dd22509b5d3e65b0ffc95>@@AEAV<lambda_ad1ced32f4ac17aa236e5ef05d6b3b7c>@@$$QEAV<lambda_f7424dd8d45958661754dc4f2697e9c3>@@@Z 000000018001a978     libucrt:mbctype.obj
 0003:00000984       $pdata$??R<lambda_ad1ced32f4ac17aa236e5ef05d6b3b7c>@@QEBAXXZ 000000018001a984     libucrt:mbctype.obj
 0003:00000990       $pdata$?getSystemCP@@YAHH@Z 000000018001a990     libucrt:mbctype.obj
 0003:0000099c       $pdata$?setSBCS@@YAXPEAU__crt_multibyte_data@@@Z 000000018001a99c     libucrt:mbctype.obj
 0003:000009a8       $pdata$?setSBUpLow@@YAXPEAU__crt_multibyte_data@@@Z 000000018001a9a8     libucrt:mbctype.obj
 0003:000009b4       $pdata$?setmbcp_internal@@YAHH_N@Z 000000018001a9b4     libucrt:mbctype.obj
 0003:000009c0       $pdata$__acrt_initialize_multibyte 000000018001a9c0     libucrt:mbctype.obj
 0003:000009cc       $pdata$__acrt_update_thread_multibyte_data 000000018001a9cc     libucrt:mbctype.obj
 0003:000009d8       $pdata$_setmbcp_nolock     000000018001a9d8     libucrt:mbctype.obj
 0003:000009e4       $pdata$?x_ismbbtype_l@@YAHPEAU__crt_locale_pointers@@IHH@Z 000000018001a9e4     libucrt:ismbbyte.obj
 0003:000009f0       $pdata$__acrt_initialize_command_line 000000018001a9f0     libucrt:argv_data.obj
 0003:000009fc       $pdata$__dcrt_get_narrow_environment_from_os 000000018001a9fc     libucrt:get_environment_from_os.obj
 0003:00000a08       $pdata$_recalloc_base      000000018001aa08     libucrt:recalloc.obj
 0003:00000a14       $pdata$__acrt_initialize_heap 000000018001aa14     libucrt:heap_handle.obj
 0003:00000a20       $pdata$?initialize_inherited_file_handles_nolock@@YAXXZ 000000018001aa20     libucrt:ioinit.obj
 0003:00000a2c       $pdata$?initialize_stdio_handles_nolock@@YAXXZ 000000018001aa2c     libucrt:ioinit.obj
 0003:00000a38       $pdata$__acrt_initialize_lowio 000000018001aa38     libucrt:ioinit.obj
 0003:00000a44       $pdata$__acrt_uninitialize_lowio 000000018001aa44     libucrt:ioinit.obj
 0003:00000a50       $pdata$__acrt_execute_initializers 000000018001aa50     libucrt:shared_initialization.obj
 0003:00000a5c       $pdata$__acrt_execute_uninitializers 000000018001aa5c     libucrt:shared_initialization.obj
 0003:00000a68       $pdata$??$?RV<lambda_c36588078e9f5dfd39652860aa6b3aaf>@@AEAV<lambda_ec61778202f4f5fc7e7711acc23c3bca>@@V<lambda_dc9d2797ccde5d239b4a0efae8ebd7db>@@@?$__crt_seh_guarded_call@P6AXH@Z@@QEAAP6AXH@Z$$QEAV<lambda_c36588078e9f5dfd39652860aa6b3aaf>@@AEAV<lambda_ec61778202f4f5fc7e7711acc23c3bca>@@$$QEAV<lambda_dc9d2797ccde5d239b4a0efae8ebd7db>@@@Z 000000018001aa68     libucrt:signal.obj
 0003:00000a74       $pdata$__acrt_get_sigabrt_handler 000000018001aa74     libucrt:signal.obj
 0003:00000a80       $pdata$raise               000000018001aa80     libucrt:signal.obj
 0003:00000a8c       $pdata$__acrt_invoke_user_matherr 000000018001aa8c     libucrt:matherr.obj
 0003:00000a98       $pdata$_mbtowc_l           000000018001aa98     libucrt:mbtowc.obj
 0003:00000aa4       $pdata$_fileno             000000018001aaa4     libucrt:fileno.obj
 0003:00000ab0       $pdata$__acrt_initialize_stdio 000000018001aab0     libucrt:_file.obj
 0003:00000abc       $pdata$__acrt_uninitialize_stdio 000000018001aabc     libucrt:_file.obj
 0003:00000ac8       $pdata$__pctype_func       000000018001aac8     libucrt:ctype.obj
 0003:00000ad4       $pdata$__acrt_free_locale  000000018001aad4     libucrt:locale_refcounting.obj
 0003:00000ae0       $pdata$__acrt_locale_free_lc_time_if_unreferenced 000000018001aae0     libucrt:locale_refcounting.obj
 0003:00000aec       $pdata$__acrt_release_locale_ref 000000018001aaec     libucrt:locale_refcounting.obj
 0003:00000af8       $pdata$__acrt_update_thread_locale_data 000000018001aaf8     libucrt:locale_refcounting.obj
 0003:00000b04       $pdata$_updatetlocinfoEx_nolock 000000018001ab04     libucrt:locale_refcounting.obj
 0003:00000b10       $pdata$__acrt_locale_free_monetary 000000018001ab10     libucrt:initmon.obj
 0003:00000b1c       $pdata$__acrt_locale_free_numeric 000000018001ab1c     libucrt:initnum.obj
 0003:00000b28       $pdata$?free_crt_array_internal@@YAXQEAPEBX_K@Z 000000018001ab28     libucrt:inittime.obj
 0003:00000b34       $pdata$__acrt_locale_free_time 000000018001ab34     libucrt:inittime.obj
 0003:00000b40       $pdata$__acrt_GetStringTypeA 000000018001ab40     libucrt:getstringtypea.obj
 0003:00000b4c       $pdata$?GetTableIndexFromLocaleName@@YAHPEB_W@Z 000000018001ab4c     libucrt:lcidtoname_downlevel.obj
 0003:00000b58       $pdata$__acrt_DownlevelLocaleNameToLCID 000000018001ab58     libucrt:lcidtoname_downlevel.obj
 0003:00000b64       $pdata$?shortsort@@YAXPEAD0_KP6AHPEBX2@Z@Z 000000018001ab64     libucrt:qsort.obj
 0003:00000b70       $pdata$2$?shortsort@@YAXPEAD0_KP6AHPEBX2@Z@Z 000000018001ab70     libucrt:qsort.obj
 0003:00000b7c       $pdata$3$?shortsort@@YAXPEAD0_KP6AHPEBX2@Z@Z 000000018001ab7c     libucrt:qsort.obj
 0003:00000b88       $pdata$qsort               000000018001ab88     libucrt:qsort.obj
 0003:00000b94       $pdata$4$qsort             000000018001ab94     libucrt:qsort.obj
 0003:00000ba0       $pdata$5$qsort             000000018001aba0     libucrt:qsort.obj
 0003:00000bac       $pdata$strncpy_s           000000018001abac     libucrt:strncpy_s.obj
 0003:00000bb8       $pdata$strpbrk             000000018001abb8     libucrt:strpbrk.obj
 0003:00000bc4       $pdata$_mbsdec_l           000000018001abc4     libucrt:mbsdec.obj
 0003:00000bd0       $pdata$?initialize_multibyte@@YAHXZ 000000018001abd0     libucrt:multibyte_initializer.obj
 0003:00000bdc       $pdata$?__acrt_LCMapStringA_stat@@YAHPEAU__crt_locale_pointers@@PEB_WKPEBDHPEADHHH@Z 000000018001abdc     libucrt:lcmapstringa.obj
 0003:00000be8       $pdata$__acrt_LCMapStringA 000000018001abe8     libucrt:lcmapstringa.obj
 0003:00000bf4       $pdata$_msize              000000018001abf4     libucrt:msize.obj
 0003:00000c00       $pdata$_realloc_base       000000018001ac00     libucrt:realloc_base.obj
 0003:00000c0c       $pdata$__acrt_lowio_create_handle_array 000000018001ac0c     libucrt:osfinfo.obj
 0003:00000c18       $pdata$__acrt_lowio_destroy_handle_array 000000018001ac18     libucrt:osfinfo.obj
 0003:00000c24       $pdata$__acrt_lowio_ensure_fh_exists 000000018001ac24     libucrt:osfinfo.obj
 0003:00000c30       $pdata$_free_osfhnd        000000018001ac30     libucrt:osfinfo.obj
 0003:00000c3c       $pdata$_get_osfhandle      000000018001ac3c     libucrt:osfinfo.obj
 0003:00000c48       $pdata$_isatty             000000018001ac48     libucrt:isatty.obj
 0003:00000c54       $pdata$__acrt_stdio_flush_nolock 000000018001ac54     libucrt:fflush.obj
 0003:00000c60       $pdata$_fflush_nolock      000000018001ac60     libucrt:fflush.obj
 0003:00000c6c       $pdata$common_flush_all    000000018001ac6c     libucrt:fflush.obj
 0003:00000c78       $pdata$_fcloseall          000000018001ac78     libucrt:closeall.obj
 0003:00000c84       $pdata$__acrt_stdio_free_buffer_nolock 000000018001ac84     libucrt:_freebuf.obj
 0003:00000c90       $pdata$??$?RV<lambda_b521505b218e5242e90febf6bfebc422>@@AEAV<lambda_6978c1fb23f02e42e1d9e99668cc68aa>@@V<lambda_314360699dd331753a4119843814e9a7>@@@?$__crt_seh_guarded_call@H@@QEAAH$$QEAV<lambda_b521505b218e5242e90febf6bfebc422>@@AEAV<lambda_6978c1fb23f02e42e1d9e99668cc68aa>@@$$QEAV<lambda_314360699dd331753a4119843814e9a7>@@@Z 000000018001ac90     libucrt:commit.obj
 0003:00000c9c       $pdata$_commit             000000018001ac9c     libucrt:commit.obj
 0003:00000ca8       $pdata$?write_double_translated_ansi_nolock@@YA?AUwrite_result@?A0x9c548279@@HQEBDI@Z 000000018001aca8     libucrt:write.obj
 0003:00000cb4       $pdata$?write_text_ansi_nolock@@YA?AUwrite_result@?A0x9c548279@@HQEBDI@Z 000000018001acb4     libucrt:write.obj
 0003:00000cc0       $pdata$?write_text_utf16le_nolock@@YA?AUwrite_result@?A0x9c548279@@HQEBDI@Z 000000018001acc0     libucrt:write.obj
 0003:00000ccc       $pdata$?write_text_utf8_nolock@@YA?AUwrite_result@?A0x9c548279@@HQEBDI@Z 000000018001accc     libucrt:write.obj
 0003:00000cd8       $pdata$_write              000000018001acd8     libucrt:write.obj
 0003:00000ce4       $pdata$_write_nolock       000000018001ace4     libucrt:write.obj
 0003:00000cfc       $pdata$??$common_lseek_nolock@_J@@YA_JH_JH@Z 000000018001acfc     libucrt:lseek.obj
 0003:00000d08       $pdata$_fclose_nolock      000000018001ad08     libucrt:fclose.obj
 0003:00000d14       $pdata$fclose              000000018001ad14     libucrt:fclose.obj
 0003:00000d20       $pdata$_putwch_nolock      000000018001ad20     libucrt:putwch.obj
 0003:00000d2c       $pdata$_call_matherr       000000018001ad2c     libucrt:libm_error.obj
 0003:00000d38       $pdata$_exception_enabled  000000018001ad38     libucrt:libm_error.obj
 0003:00000d44       $pdata$_handle_error       000000018001ad44     libucrt:libm_error.obj
 0003:00000d50       $pdata$__acrt_initialize_fma3 000000018001ad50     libucrt:fma3_available.obj
 0003:00000d5c       $pdata$_log10_special      000000018001ad5c     libucrt:log_special.obj
 0003:00000d68       $pdata$_log_special_common 000000018001ad68     libucrt:log_special.obj
 0003:00000d74       $pdata$??$?RV<lambda_bfedae4ebbf01fab1bb6dcc6a9e276e0>@@AEAV<lambda_2fe9b910cf3cbf4a0ab98a02ba45b3ec>@@V<lambda_237c231691f317818eb88cc1d5d642d6>@@@?$__crt_seh_guarded_call@H@@QEAAH$$QEAV<lambda_bfedae4ebbf01fab1bb6dcc6a9e276e0>@@AEAV<lambda_2fe9b910cf3cbf4a0ab98a02ba45b3ec>@@$$QEAV<lambda_237c231691f317818eb88cc1d5d642d6>@@@Z 000000018001ad74     libucrt:close.obj
 0003:00000d80       $pdata$_close              000000018001ad80     libucrt:close.obj
 0003:00000d8c       $pdata$_close_nolock       000000018001ad8c     libucrt:close.obj
 0003:00000d98       $pdata$__dcrt_lowio_initialize_console_output 000000018001ad98     libucrt:initcon.obj
 0003:00000da4       $pdata$__dcrt_terminate_console_output 000000018001ada4     libucrt:initcon.obj
 0003:00000dbc       $pdata$_raise_exc          000000018001adbc     libucrt:fpexcept.obj
 0003:00000dc8       $pdata$_raise_exc_ex       000000018001adc8     libucrt:fpexcept.obj
 0003:00000dd4       $pdata$_set_errno_from_matherr 000000018001add4     libucrt:fpexcept.obj
 0003:00000de0       $pdata$_clrfp              000000018001ade0     libucrt:fpctrl.obj
 0003:00000dec       $pdata$_ctrlfp             000000018001adec     libucrt:fpctrl.obj
 0003:00000df8       $pdata$_set_statfp         000000018001adf8     libucrt:fpctrl.obj
 0003:00000e04       $pdata$_statfp             000000018001ae04     libucrt:fpctrl.obj
 0003:00000e10       $pdata$__GSHandlerCheck    000000018001ae10     LIBCMT:_gshandler_.obj
 0003:00000e1c       $pdata$__GSHandlerCheckCommon 000000018001ae1c     LIBCMT:_gshandler_.obj
 0003:00000e34       $pdata$_IsNonwritableInCurrentImage 000000018001ae34     LIBCMT:pesect.obj
 0003:00000e40       $pdata$__raise_securityfailure 000000018001ae40     LIBCMT:gs_report.obj
 0003:00000e4c       $pdata$__report_gsfailure  000000018001ae4c     LIBCMT:gs_report.obj
 0003:00000e58       $pdata$__report_rangecheckfailure 000000018001ae58     LIBCMT:gs_report.obj
 0003:00000e64       $pdata$__report_securityfailure 000000018001ae64     LIBCMT:gs_report.obj
 0003:00000e70       $pdata$capture_current_context 000000018001ae70     LIBCMT:gs_report.obj
 0003:00000e7c       $pdata$capture_previous_context 000000018001ae7c     LIBCMT:gs_report.obj
 0003:00000eac       $pdata$?fin$0@?0??dllmain_crt_process_attach@@YAHQEAUHINSTANCE__@@QEAX@Z@4HA 000000018001aeac     LIBCMT:dll_dllmain.obj
 0003:00000eb8       $pdata$?fin$0@?0??dllmain_crt_process_detach@@YAH_N@Z@4HA 000000018001aeb8     LIBCMT:dll_dllmain.obj
 0003:00000ec4       $pdata$?filt$0@?0??dllmain_dispatch@@YAHQEAUHINSTANCE__@@KQEAX@Z@4HA 000000018001aec4     LIBCMT:dll_dllmain.obj
 0003:00000ed0       $pdata$__scrt_is_nonwritable_in_current_image$filt$0 000000018001aed0     LIBCMT:utility.obj
 0003:00000edc       $pdata$_query_new_handler$fin$0 000000018001aedc     libucrt:new_handler.obj
 0003:00000ee8       $pdata$?filt$0@?0??common_exit@@YAXHW4_crt_exit_cleanup_mode@@W4_crt_exit_return_mode@@@Z@4HA 000000018001aee8     libucrt:exit.obj
 0003:00000ef4       $pdata$?fin$1@?0??common_exit@@YAXHW4_crt_exit_cleanup_mode@@W4_crt_exit_return_mode@@@Z@4HA 000000018001aef4     libucrt:exit.obj
 0003:00000f00       $pdata$?fin$0@?0???$?RV<lambda_e24bbb7b643b32fcea6fa61b31d4c984>@@AEAV<lambda_275893d493268fdec8709772e3fcec0e>@@V<lambda_9d71df4d7cf3f480f8d633942495c3b0>@@@?$__crt_seh_guarded_call@H@@QEAAH$$QEAV<lambda_e24bbb7b643b32fcea6fa61b31d4c984>@@AEAV<lambda_275893d493268fdec8709772e3fcec0e>@@$$QEAV<lambda_9d71df4d7cf3f480f8d633942495c3b0>@@@Z@4HA 000000018001af00     libucrt:onexit.obj
 0003:00000f0c       $pdata$__acrt_uninitialize_locale$fin$0 000000018001af0c     libucrt:wsetlocale.obj
 0003:00000f0c       $pdata$__acrt_update_thread_locale_data$fin$0 000000018001af0c     libucrt:locale_refcounting.obj
 0003:00000f18       $pdata$__acrt_update_thread_multibyte_data$fin$0 000000018001af18     libucrt:mbctype.obj
 0003:00000f24       $pdata$?fin$0@?0???$?RV<lambda_5e887d1dcbef67a5eb4283622ba103bf>@@AEAV<lambda_4466841279450cc726390878d4a41900>@@V<lambda_341c25c0346d94847f1f3c463c57e077>@@@?$__crt_seh_guarded_call@X@@QEAAX$$QEAV<lambda_5e887d1dcbef67a5eb4283622ba103bf>@@AEAV<lambda_4466841279450cc726390878d4a41900>@@$$QEAV<lambda_341c25c0346d94847f1f3c463c57e077>@@@Z@4HA 000000018001af24     libucrt:per_thread_data.obj
 0003:00000f24       $pdata$?fin$0@?0???$?RV<lambda_72d1df2b273a38828b1ce30cbf4cdab5>@@AEAV<lambda_876a65b173b8412d3a47c70a915b0cf4>@@V<lambda_41932305e351933ebe8f8be3ed8bb5dc>@@@?$__crt_seh_guarded_call@X@@QEAAX$$QEAV<lambda_72d1df2b273a38828b1ce30cbf4cdab5>@@AEAV<lambda_876a65b173b8412d3a47c70a915b0cf4>@@$$QEAV<lambda_41932305e351933ebe8f8be3ed8bb5dc>@@@Z@4HA 000000018001af24     libucrt:per_thread_data.obj
 0003:00000f24       $pdata$?fin$0@?0???$?RV<lambda_fb3a7dec4e47f37f22dae91bb15c9095>@@AEAV<lambda_698284760c8add0bfb0756c19673e34b>@@V<lambda_dfb8eca1e75fef3034a8fb18dd509707>@@@?$__crt_seh_guarded_call@X@@QEAAX$$QEAV<lambda_fb3a7dec4e47f37f22dae91bb15c9095>@@AEAV<lambda_698284760c8add0bfb0756c19673e34b>@@$$QEAV<lambda_dfb8eca1e75fef3034a8fb18dd509707>@@@Z@4HA 000000018001af24     libucrt:per_thread_data.obj
 0003:00000f24       $pdata$?fin$0@?0???$?RV<lambda_99476a1ad63dd22509b5d3e65b0ffc95>@@AEAV<lambda_ad1ced32f4ac17aa236e5ef05d6b3b7c>@@V<lambda_f7424dd8d45958661754dc4f2697e9c3>@@@?$__crt_seh_guarded_call@X@@QEAAX$$QEAV<lambda_99476a1ad63dd22509b5d3e65b0ffc95>@@AEAV<lambda_ad1ced32f4ac17aa236e5ef05d6b3b7c>@@$$QEAV<lambda_f7424dd8d45958661754dc4f2697e9c3>@@@Z@4HA 000000018001af24     libucrt:mbctype.obj
 0003:00000f24       $pdata$?fin$0@?0???$?RV<lambda_b8c45f8f788dd370798f47cfe8ac3a86>@@AEAV<lambda_4e60a939b0d047cfe11ddc22648dfba9>@@V<lambda_332c3edc96d0294ec56c57d38c1cdfd5>@@@?$__crt_seh_guarded_call@H@@QEAAH$$QEAV<lambda_b8c45f8f788dd370798f47cfe8ac3a86>@@AEAV<lambda_4e60a939b0d047cfe11ddc22648dfba9>@@$$QEAV<lambda_332c3edc96d0294ec56c57d38c1cdfd5>@@@Z@4HA 000000018001af24     libucrt:onexit.obj
 0003:00000f24       $pdata$?fin$0@?0???$?RV<lambda_46352004c1216016012b18bd6f87e700>@@AEAV<lambda_3bd07e1a1191394380780325891bf33f>@@V<lambda_334532d3f185bcaa59b5be82d7d22bff>@@@?$__crt_seh_guarded_call@X@@QEAAX$$QEAV<lambda_46352004c1216016012b18bd6f87e700>@@AEAV<lambda_3bd07e1a1191394380780325891bf33f>@@$$QEAV<lambda_334532d3f185bcaa59b5be82d7d22bff>@@@Z@4HA 000000018001af24     libucrt:per_thread_data.obj
 0003:00000f24       $pdata$?fin$0@?0???$?RV<lambda_c36588078e9f5dfd39652860aa6b3aaf>@@AEAV<lambda_ec61778202f4f5fc7e7711acc23c3bca>@@V<lambda_dc9d2797ccde5d239b4a0efae8ebd7db>@@@?$__crt_seh_guarded_call@P6AXH@Z@@QEAAP6AXH@Z$$QEAV<lambda_c36588078e9f5dfd39652860aa6b3aaf>@@AEAV<lambda_ec61778202f4f5fc7e7711acc23c3bca>@@$$QEAV<lambda_dc9d2797ccde5d239b4a0efae8ebd7db>@@@Z@4HA 000000018001af24     libucrt:signal.obj
 0003:00000f30       $pdata$raise$fin$0         000000018001af30     libucrt:signal.obj
 0003:00000f3c       $pdata$__acrt_initialize_lowio$fin$0 000000018001af3c     libucrt:ioinit.obj
 0003:00000f3c       $pdata$__acrt_lowio_ensure_fh_exists$fin$0 000000018001af3c     libucrt:osfinfo.obj
 0003:00000f48       $pdata$common_flush_all$fin$0 000000018001af48     libucrt:fflush.obj
 0003:00000f54       $pdata$common_flush_all$fin$1 000000018001af54     libucrt:fflush.obj
 0003:00000f60       $pdata$_fcloseall$fin$0    000000018001af60     libucrt:closeall.obj
 0003:00000f6c       $pdata$?fin$0@?0???$?RV<lambda_b521505b218e5242e90febf6bfebc422>@@AEAV<lambda_6978c1fb23f02e42e1d9e99668cc68aa>@@V<lambda_314360699dd331753a4119843814e9a7>@@@?$__crt_seh_guarded_call@H@@QEAAH$$QEAV<lambda_b521505b218e5242e90febf6bfebc422>@@AEAV<lambda_6978c1fb23f02e42e1d9e99668cc68aa>@@$$QEAV<lambda_314360699dd331753a4119843814e9a7>@@@Z@4HA 000000018001af6c     libucrt:commit.obj
 0003:00000f6c       $pdata$?fin$0@?0???$?RV<lambda_bfedae4ebbf01fab1bb6dcc6a9e276e0>@@AEAV<lambda_2fe9b910cf3cbf4a0ab98a02ba45b3ec>@@V<lambda_237c231691f317818eb88cc1d5d642d6>@@@?$__crt_seh_guarded_call@H@@QEAAH$$QEAV<lambda_bfedae4ebbf01fab1bb6dcc6a9e276e0>@@AEAV<lambda_2fe9b910cf3cbf4a0ab98a02ba45b3ec>@@$$QEAV<lambda_237c231691f317818eb88cc1d5d642d6>@@@Z@4HA 000000018001af6c     libucrt:close.obj
 0003:00000f78       $pdata$_write$fin$0        000000018001af78     libucrt:write.obj
 0003:00000f84       $pdata$fclose$fin$0        000000018001af84     libucrt:fclose.obj
 0003:00000f90       $pdata$_ctrlfp$filt$0      000000018001af90     libucrt:fpctrl.obj
 0003:00000f9c       $pdata$_IsNonwritableInCurrentImage$filt$0 000000018001af9c     LIBCMT:pesect.obj
 0004:000004e8       .idata$6                   000000018001b4e8     kernel32:KERNEL32.dll
 0004:00000a08       .idata$6                   000000018001ba08     advapi32:ADVAPI32.dll
 0005:00000000       __guard_fids__             000000018001c000     libucrt:initialization.obj
 0005:00000060       __guard_fids___acrt_initialize_ptd 000000018001c060     libucrt:per_thread_data.obj
 0005:00000064       __guard_fids_??$expand_argument_wildcards@D@@YAHQEAD0AEAV?$argument_list@D@?A0xca0879c4@@@Z 000000018001c064     libucrt:argv_wildcards.obj
 0005:00000068       __guard_fids__             000000018001c068     libucrt:locale_initializer.obj
 0005:0000006c       __guard_fids__             000000018001c06c     libucrt:multibyte_initializer.obj
 0005:00000070       __guard_fids__             000000018001c070     libucrt:stdio_initializer.obj
 0005:00000074       __guard_fids__             000000018001c074     libucrt:stdio_initializer.obj
 0005:00000078       __guard_fids__             000000018001c078     libucrt:fma3_initializer.obj
 0005:0000007c       __guard_fids__             000000018001c07c     libucrt:console_output_initializer.obj
 0005:00000080       __guard_fids_?dllmain_crt_process_attach@@YAHQEAUHINSTANCE__@@QEAX@Z 000000018001c080     LIBCMT:dll_dllmain.obj
 0005:00000088       __guard_fids_?dllmain_dispatch@@YAHQEAUHINSTANCE__@@KQEAX@Z 000000018001c088     LIBCMT:dll_dllmain.obj
 0005:0000008c       __guard_fids__             000000018001c08c     LIBCMT:throw_bad_alloc.obj
 0005:00000094       __guard_fids__             000000018001c094     LIBCMT:throw_bad_alloc.obj
 0005:0000009c       __guard_fids__             000000018001c09c     LIBCMT:throw_bad_alloc.obj
 0005:000000a4       __guard_fids__             000000018001c0a4     LIBCMT:std_type_info_static.obj
 0005:000000a8       __guard_fids__             000000018001c0a8     LIBCMT:guard_support.obj
 0005:000000ac       __guard_fids__             000000018001c0ac     libvcruntime:telemetry.obj
 0005:000000b0       __guard_fids_?TraceLoggingRegister@__vcrt_trace_logging_provider@@YAJPEBU_TlgProvider_t@1@PEBU_GUID@@P6AX1KE_K2PEAU_EVENT_FILTER_DESCRIPTOR@@PEAX@Z4@Z 000000018001c0b0     libvcruntime:telemetry.obj
 0005:000000b4       __guard_fids___vcrt_initialize_ptd 000000018001c0b4     libvcruntime:per_thread_data.obj
 0006:00000060       $R000000                   000000018001d060     AutoWrap.res
